:020000040800F2
:10000000008000201D4E0008A15A0008C1240008ED
:10001000A35A0008A55A0008A75A000800000000CB
:10002000000000000000000000000000B1A5000872
:10003000A95A00080000000041A6000885A6000893
:10004000AB5A0008AD5A0008AF5A0008B15A000870
:10005000B35A0008B55A0008355A00083B5A000840
:10006000415A0008475A00084D5A0008B75A00087C
:10007000B95A0008BB5A0008BD5A0008BF5A000808
:10008000C15A0008C35A0008C55A0008C75A0008D8
:10009000C95A0008CB5A0008CD5A0008535A000824
:1000A000CF5A0008D15A0008D35A0008D55A000880
:1000B000D75A0008D95A0008DB5A0008DD5A000850
:1000C000DF5A0008E15A0008E35A0008E55A000820
:1000D000E75A00085962000839640008E95A000824
:1000E000775A0008215B0008EB5A0008ED5A000817
:1000F000EF5A0008000000000000000000000000AF
:1001000000000000000000005FF808F110B5054C89
:10011000237833B9044B13B10448AFF300800123B3
:10012000237010BD780400200000000038FA010898
:1001300008B5034B1BB103490348AFF3008008BD6A
:10014000000000007C04002038FA010808B501F026
:10015000DFF8BDE8084001F011B908B501F0D8F8A2
:1001600008BD08B501F0D4F8503008BD004870470C
:100170004D01000808B501F0CBF8643008BD10B59A
:1001800001F0C6F8044603680121DB68984723683C
:1001900020461B694FF4FA71984723682046BDE852
:1001A0001040DB680021184708B501F0B1F8BDE840
:1001B000084001F05FB908B501F0AAF8BDE80840B1
:1001C00001F01CBA10B5044601F0A2F80146204621
:1001D00001F080FB204610BD08B5034808F02AF95D
:1001E000BDE8084006F058B931AE010806F054B930
:1001F00010B50446C06910B1012114F05DF9206901
:1002000010B1012114F058F9204610BDF8B50025B1
:10021000C0E901120570C0E90335C0E90555C0E920
:100220000755456206990446164600F11C0712F070
:1002300067F838B93146074808F0FCF8202106482D
:1002400002F0BAF8069A3946204612F043F82046E2
:10025000F8BD00BF4FAE01087AAE0108F8B5002521
:10026000C0E901120570C0E90335C0E90555C0E9D0
:100270000755456206990446164600F11C0712F020
:1002800023F938B93146074808F0D4F82021064848
:1002900002F092F8069A3946204612F0DDF8204620
:1002A000F8BD00BF4FAE01087AAE01082DE9F0415C
:1002B00000259DF81860C0E901120570C0E90335FA
:1002C000C0E90555C0E90755456231460446174661
:1002D00000F11C0811F014FF38B93946074808F03E
:1002E000A9F82021064802F067F832464146204628
:1002F00011F0F4FE2046BDE8F08100BF4FAE0108CA
:100300007AAE010870B5AEB013F03EF9054600268E
:1003100012A808ACFFF756FF12A928460DF0AEFF51
:10032000674B684A009602212046FFF76FFF21467F
:10033000284613F0CFF92046FFF75AFF3223624ACE
:1003400000930221614B2046FFF760FF21462846BB
:1003500013F0C0F92046FFF74BFF5D4B5D4A1B6869
:100360000321009320465C4BFFF778FF2146284687
:1003700013F0B0F92046FFF73BFF3C23574A0093A8
:100380000221574B2046FFF741FF2146284613F034
:10039000A1F92046FFF72CFF524B534A009601214A
:1003A0002046FFF783FF2146284613F093F92046A5
:1003B000FFF71EFF4D4B4E4A009602212046FFF7E5
:1003C00025FF2146284613F085F92046FFF710FF48
:1003D000484B494A009601212046FFF767FF214616
:1003E000284613F077F92046FFF702FF434B444AB3
:1003F000009602212046FFF709FF2146284613F008
:1004000069F92046FFF7F4FE4FF416733D4A009356
:1004100002213D4B2046FFF7F9FE2146284613F006
:1004200059F92046FFF7E4FE384B394A1B6803218F
:1004300000932046374BFFF711FF2146284613F063
:1004400049F92046FFF7D4FE334B344A1B68032199
:1004500000932046324BFFF701FF2146284613F058
:1004600039F92046FFF7C4FE2E4B2F4A0093032193
:100470002E4B2046FFF7F2FE2146284613F02AF9BC
:100480002046FFF7B5FE2846294B2A4A2A4912F092
:10049000E9FF0121294B2A4A08932A4BCDE905128D
:1004A0000993294B07960A9305AB93E807008DE85B
:1004B00007000B9694E80F0013F004FB2EB070BDFC
:1004C00068AA0108BBAA0108F1AA0108C9AA010883
:1004D0000400002044AB010800AB01088FAB010809
:1004E0004FAB01089BAB0108DAAB0108EDAB01088B
:1004F0002DAC010839AC010864AC010871AC0108ED
:10050000B9AC0108ECAC0108CAAC01080800002035
:1005100043AD0108FDAC01080C0000209BAD0108B3
:100520004BAD01080BE40108FDAD0108A5AD0108C4
:10053000ED01000807AE01082BAE0108A153000829
:100540000000080829530008D901000810B5084C1C
:1005500022681AB99421074801F02EFF064B1A6849
:100560002368B2FBF3F003FB102303B1013010BD8D
:10057000B4060020F7B00108B0060020F8B5FFF778
:10058000F0FD03681B6898470E4B1B78B3B90E4B00
:10059000D3E90023B3F1004F08BF002A10D0002791
:1005A0000A4E841A61EB0305A64277EB050407DBCC
:1005B000904271EB0303B4BF012300231846F8BD3A
:1005C0000123FBE7CC050020280000204351010057
:1005D00038B503F072F804F0DBF8022104F0E6F815
:1005E00004460D4603F0C4FC012C75F100030ADB40
:1005F00002F040F905492B462246097802F043FEF5
:10060000034B187838BD034BFBE700BFD80600202A
:100610001308002010080020F8B54FF0004700260E
:10062000184C15F0CFFD01F0F5FDD4E90023BB42D5
:1006300008BFB24223D002F01DF930CC1249621C2F
:1006400045F10003097802F02CFEB94208BFB04220
:1006500004460D4613D0FFF784FD03681B689847D6
:10066000A04271EB05030ADB2946204607F062FE33
:100670000146064807F0DEFE054B1878F8BD054B2D
:10068000FBE700BF30000020D006002080AF01084B
:10069000130800201008002010B50020002103F0EE
:1006A000ABFA044628B90F4807F0C4FE0E4B187881
:1006B00010BD41790D4807F0BDFE617980290DD14B
:1006C0000B4B22792168186812F0FEFA204603F0DD
:1006D000FBFD0821204613F0EFFEE7E7054807F091
:1006E000A9FEF3E7DBAF010810080020E3AF010823
:1006F000D4060020ECAF010810B5CCB004F048F8E7
:1007000004A903F04BFF204C00283AD04FF4967216
:100710001E49684613F033FE01238DF80C301C4B44
:100720001B78012B1ED1059A0023684613F06EFE3C
:100730000CA90B9A684613F02FFE684613F057FE7B
:100740000022144B206068461A6013F04EFE0446E7
:10075000684613F04CFE214602460F4813F0C6FDD2
:100760004CB010BD022BE3D16846059A002313F06C
:100770004DFE9DF8241068464942C9B213F02AFE86
:10078000D6E72060ECE700BFB0060020A004002000
:10079000AB060020AC0600201000002010B5FFF7CB
:1007A00003FD0B49044616F0D5FE17F0BFF8094BC0
:1007B0001880FFF700FD084B084A18804FF0804171
:1007C00020460EF04DFCBDE810400EF073BC00BF9B
:1007D00000007A443A00002038000020CDCC4C4084
:1007E00008B5084807F026FEFFF7BBFC03681B6846
:1007F0009847054BC3E90001FFF7D0FF034B18787A
:1008000008BD00BFAEAF0108300000201008002076
:1008100070B54A4C94B02368DB0708D412F0CEFEC2
:1008200080220146464811F0ABFF01232360454B6F
:10083000434A454D1A602B68444C13F0010F04D114
:10084000FFF798FC012320602B60206803681B6879
:100850009847054620B940F217113D4801F0ACFD1C
:100860003C4B0C933C4B0A933C4B09933C4B0B93F6
:100870003C4B06933C4B08933C4B079312F09EFE77
:1008800004461C2200210DA817F0A1FB3849204680
:1008900012F022FD37498DF83400204612F036FD63
:1008A0003549ADF83600204612F030FD3349ADF839
:1008B0003800204612F02AFD1090FFF752FC064641
:1008C00002AB06AA07CA83E807000BAB93E8030054
:1008D0008DE8030009AB0CCB2946304603F022FF1C
:1008E0000DA904F0C5F803F053FF054615F06AFCA6
:1008F0002349204612F013FD05F52C7501462846C4
:1009000015F086F81F49204612F009FD01462846D9
:1009100015F0F8F81C49204612F001FD0146284662
:1009200015F066F91949204612F0D6FC0DF038FB97
:10093000FFF734FF164B187814B070BD94040020F4
:10094000B8060020D406002098040020C806002025
:10095000F7B001083584000895090008B1090008BE
:10096000CD09000875E1000815E10008D9E100088B
:1009700064AC01088FAB01082DAC0108ECAC010898
:1009800043AD01089BAD0108FDAD0108DAAB0108DC
:1009900010080020054B30B41C6823689D6813467E
:1009A000AC460A460146204630BC6047C8060020D7
:1009B000054B30B41C6823685D681346AC460A4694
:1009C0000146204630BC6047C8060020034B014664
:1009D0001B681A6818461269104700BFC806002035
:1009E00038B502F06AFE03F0D3FE012103F0DEFE0B
:1009F00004460D4603F0BCFA012C75F100030ADB36
:100A000001F038FF09492B462246097802F03BFCE9
:100A1000074B187838BD15F056FE28B9054807F081
:100A200009FD0122044B1A70044BF2E7D80600209E
:100A30001308002027AF0108CC0500201008002073
:100A400038B5134B1B685B680BB1012038BDFFF74D
:100A500095FD0028F9D10F4C23683BB915F01FFE16
:100A6000002801DDFFF748FE236863B115F02BFE77
:100A7000054615F014FE2D1A15F025FE29460246EE
:100A8000054807F0D7FC2068003018BF0120DDE7DB
:100A9000D4060020B0060020BEAF01081FB56123B8
:100AA000CDE9013101A9039201F0FEFE05B05DF828
:100AB00004FB07B58DF8041001A98DF805208DF809
:100AC000063001F0B1FF03B05DF804FB2DE9F04FF3
:100AD00087B0FFF742FB044614F0BEFC204614F03A
:100AE000D1FCFFF70FFCFA200BF08AF812F066FD3C
:100AF000044612F05BF9204603F032F9A349204680
:100B000012F004FC022800F230810025A04B18707E
:100B1000A049204612F0FAFBA0F10A03282B00F2AC
:100B200029819D4B1860002D40F027819B4D9C48EA
:100B300007F080FC2B689B4C13F0010F04D101F0EF
:100B400099FE012320602B602568FFF70AFB014610
:100B5000284601F05BFD2568FFF708FB01462846A3
:100B600001F056FD12F02AFD8F49256812F0D7FBDF
:100B70008E49024603A801F033FD03A9284601F07F
:100B800089FD8B4B2568187000220023894903A832
:100B900001F0D8FC03A9284601F07CFD864A87496C
:100BA0001070874A2068FFF779FF8DF807002068EA
:100BB00002F0A2FD834A824683492068FFF76EFF58
:100BC0004FF000097025814B064603A92068049365
:100BD00003958DF8149001F067FE7D4A8DF80500AD
:100BE0007C492068FFF75AFF7B4B804603A92068A9
:100BF000049303958DF8149001F056FE774A8DF812
:100C0000060077492068FFF749FF764B8346764A0E
:100C10007649206803F062FA754A074675492068EC
:100C2000FFF73CFF744A8DF8020074492068FFF713
:100C300035FF5F4B8DF803001A787149206802F088
:100C40009DFE9DF807508DF804002068534680F8FB
:100C500028506C4D9DF807102A78FFF72AFF6A4A42
:100C60005146DFF8BCA1334620681278FFF721FF18
:100C70009DF805309AF8002031462068FFF719FFEB
:100C80004D4933460A7820689DF80510FFF711FF9B
:100C900043462A7831462068FFF70BFF9DF806305F
:100CA0009AF8002041462068FFF703FF4249434677
:100CB0000A7820689DF80610FFF7FBFE3B462A786D
:100CC00041462068DFF85C81FFF7F3FE3B462A7857
:100CD0009DF802102068FFF7ECFE9DF8023098F8AE
:100CE000002039462068FFF7E4FE9DF803302A789B
:100CF00039462068FFF7DDFE5B469AF800209DF834
:100D000003102068FFF7D5FE9DF804302A789DF87F
:100D100003102068FFF7CDFE9DF8023098F8002000
:100D20009DF804102068FFF7C4FE214A5B469DF839
:100D3000041020681278FFF7BCFE33462A78594623
:100D40002068FFF7B6FE206802F016F82F4807F07B
:100D500071FB01224FF49671206801F0A7FF48460D
:100D60000AF0CAFC07B0BDE8F08F294807F062FB23
:100D70000125CDE6274807F05DFB274807F05AFB21
:100D800040F2E311254801F017FBCFE6BBAA0108AA
:100D9000AB060020F1AA0108B40600209C04002044
:100DA00069B00108CC06002044AB010886B00108F8
:100DB000D00600208BB00108D8060020E4BB010853
:100DC00011080008D105000895B001089FB001087E
:100DD000E1090008AAB00108B4B00108E107000861
:100DE000BFB00108C90F0008410A0008C6B00108D9
:100DF000990600086EBA010819060008D3B0010868
:100E0000B9BB01081008002014080020DDB001085B
:100E10000CB0010833B0010856B00108F7B0010862
:100E200013080020D908002030B5012585B00A46F6
:100E300004461949684613F0A2FA022168468DF863
:100E40000C5013F0C7FA0421684613F0C3FA0021CE
:100E5000684613F0BFFA114B6846198813F0E2FA9E
:100E60000F4B6846B3F9001013F0C3FA0D4B197815
:100E700011B1002229461A70684613F0ABFA684691
:100E800013F0B3FA0546684613F0B1FA0123256062
:100E90006371207105B030BDCD0500203A000020FF
:100EA00038000020CC0500202DE9F7433C4B0446D8
:100EB0001B780A46012B5CD008D3022B67D0E121B6
:100EC000384803B0BDE8F04301F076BAFFF73EFBC7
:100ED000354D364F2B68984244D93968344A01FB66
:100EE0000328344B1E68FFF731FB2A68904292BFFB
:100EF00000233B685343F61A3B689E4228BF1E46B8
:100F00001EB9B921274801F057FA0A272B6803FBBD
:100F10000777FFF71BFB2968074401F10109FFF779
:100F200015FBFBB20246009349463346224807F0C0
:100F300081FA3146404607F0E3FA204807F07AFA92
:100F40002B6867710133C4F8008026712B60FFF7AE
:100F5000FDFA2B68984202D10022164B1A6003B0AA
:100F6000BDE8F083B7210F4801F026FA4FF00008E2
:100F7000B7E7134E134D3146284613F089F9652320
:100F800063712071D5E9022326609A42E3E70C4E93
:100F90000C4D3146284613F07BF96623F0E700BF7D
:100FA000AB060020F7B00108AC060020B406002014
:100FB000A0040020B006002045AF01080AE40108A3
:100FC000CD05002010000020F7B5194F04463B68FE
:100FD0000D465B688BB1174E174807F02BFA0DF1E1
:100FE00007032A463146386811F024FC9DF8073083
:100FF00026606371207103B0F0BDFFF7BFFA78B1CE
:101000000E4807F017FAFFF7ACF803681B6898471B
:101010000B4BC3E9000129462046FFF705FFEAE72D
:10102000084807F007FA29462046FFF73DFFE2E7A8
:10103000D4060020CD050020C9AE0108EFAE01089E
:10104000280000200CAF010813B5FFF786F80368ED
:1010500000249B689847FFF792F801234FF496729B
:101060000B49CDE900340B4823460AF057FA0A48E9
:1010700007F0E0F9094807F0DDF90AF029FC40F231
:101080000F21074801F098F9204602B010BD00BFBB
:1010900043B10108CD0A00084CB101085FB1010855
:1010A000F7B00108FF23024A1370024A1370704719
:1010B000D8060020D00600207047000038B50A4C42
:1010C00005460121204604F0B3FB002320461A46C2
:1010D000012104F0EBFA85F001022046BDE838401A
:1010E000012104F0B1BB00BF0000024008B501209F
:1010F000FFF7E4FFBDE80840032005F0DDB908462E
:10110000FFF7DCBF10B50446682113F0D5F920467F
:1011100010BD0000024B0121186803681B681847C6
:10112000E8060020021C18BF01220321014804F038
:101130008BBB00BF0004024010B50C460AF0C8FF8C
:10114000022808D14FF47A704443B4FBF0F0BDE8B4
:1011500010400AF055BD2046BDE8104004F0C2B86A
:101160000321014804F079BB0004024010B5094C8A
:10117000094807F05FF920460B2104F059FB0023D2
:1011800020461A460B2104F091FABDE8104004F005
:101190008FB800BF00000240CEB4010808B502209D
:1011A00003F0EAFF04F04CF800F046FC04F072F89B
:1011B00000F054FE04F0D6FD0C4801F0C7F84FF4DF
:1011C000E13005F02DF90A4B1A680AB9094A1A608C
:1011D000094B1A680AB9074A1A60084807F02AF941
:1011E000BDE80840064807F025B900BFED1000082B
:1011F000B40C0020C1620008B80C0020F8B101084E
:1012000010B201082DE9F347044625464FF01B0AAA
:1012100014F018F9254B04F1210945F8113B10226F
:101220000021284616F0D3FE52460021484616F00B
:10123000CEFE00231E4AC4E90F3362641D4A84F8BF
:101240004C30A2641C4AC4E91633226584F860302D
:101250001A4A1B4B1B4F626563661B4807F0EAF88E
:101260003B68DFF870800193D8F80030174E009388
:101270003368174A5146484617F018FD316828462A
:1012800007F0E2F9D8F8001004F1150007F0DCF9D6
:10129000396804F1190007F0D7F9316804F11D002D
:1012A00007F0D2F9204602B0BDE8F08734B5010856
:1012B00028B60108C4B60108F4B60108E0B6010872
:1012C00060B601086400F81F02B501085000F81F5D
:1012D00017B501085400F81F10B5094CFFF75EFF61
:1012E0002368DB0709D40748FFF78CFF0123064A70
:1012F00006490448236015F0F8F9024810BD00BF04
:10130000E0060020EC06002000000020B9100008D4
:1013100038B5064D064C2B6813F0010F04D1FFF7CA
:10132000DBFF012320602B60206838BDE40600202D
:101330005407002008B50B21054804F093FA28B1A2
:10134000BDE808400B21024804F0A0BA08BD00BF68
:101350000000024008B519B1BDE80840FFF706BF1C
:10136000044807F067F8BDE8084002220B21024854
:1013700004F0DAB9EAB4010800000240F8B5044606
:10138000374804F1440507F055F82846002100F0DD
:101390008DFD0021284600F09FFD324D204614F0BF
:1013A00081F80CF0B7FE0DF05DFB20460021FFF741
:1013B000D1FF0BF07DFC13F045FB012228460C21E8
:1013C00004F0B2F904F0ECFD23682046DB6804F178
:1013D000540600219847244F0021304600F080FE3B
:1013E00004F0B2FA214807F025F804F007FF03F0F3
:1013F00051FF384601220D2104F096F901223846AA
:101400000E2104F091F90021084604F087FD04F153
:10141000480000F0F5FD0121304600F061FE4FF478
:10142000E13004F0FDFF124807F004F828460C21D3
:1014300004F0FEF9002328461A460C2104F036F980
:101440000120002104F0D0FD13F00EFB0BF056FB41
:1014500004F0A4FD2046BDE8F84014F033B800BF06
:101460009CB401080004024000000240C0B401081E
:1014700018B7010838B50546FFF75CFF044628B1E8
:1014800000212846FFF766FF03F012FF03F018FE65
:1014900005460CB1FFF76AFE284638BD70B50C460C
:1014A00006461549204616F011FA20B900212046BB
:1014B00016F0EEF970B11149204616F04BF816F00F
:1014C0000FFA01460E4806F0B5FF40F27D110D48B7
:1014D00000F072FF3046FFF72DFF054648B9304651
:1014E000FFF7C8FF0146204616F0F0F908B1FFF7F4
:1014F0003DFE284670BD00BF3333534000007A44A0
:1015000026B2010855B2010870B52D4AD6B013684D
:101510000546DB0705D42B4900F154030B6001237A
:10152000136029492846FFF7B9FF0646274806F009
:1015300081FF002105F1440000F0CEFC244C254B36
:10154000E360254B2361254BA360254B6360254B4E
:101550002360254B6361254BA361254BE36104F1B7
:1015600010030FCB8DE80F0094E80F0013F0A6FCDA
:10157000002305A8EB632B6413F02CFC9DF81430BA
:1015800005F13C04012B14D1DDF8153005A8EB63FF
:10159000DDF819302B6413F0EDFB164806F04AFF16
:1015A0000821204606F0ACFFBDF91611124806F0DE
:1015B00041FF31462846FFF7CDFE56B070BD00BF53
:1015C000DC060020E80600200000404091B1010840
:1015D00024560020E55200086D520008151100083D
:1015E000611100082511000835840008D5A5000800
:1015F00015A60008B2B10108D8B1010870B50749B5
:101600000546FFF74BFF064613F07CFB04463146C8
:101610002846FFF79FFE204670BD00BF00004040F7
:101620007FB5F82300F1480504AC0646284604F8C7
:10163000013D00F0EBFC0223214600930122A1238F
:10164000284600F0E7FC4FF400430822009306F11F
:101650005801A1230446284600F006FD0440E4B2E8
:10166000284600F0D5FC204604B070BD30B58BB0E4
:10167000044604F04FFF0146514806F0DBFE514896
:1016800006F0D8FE204600F09FFB00F0B1FA00F013
:101690005BFA4D4806F0CEFE04F148054B484C4934
:1016A00006F0C8FE284600F0ABFC38B9494806F001
:1016B000C1FE4FF49D71484800F07EFE03F0F8FD36
:1016C0002046FFF7ADFF20B940F23F11424800F03D
:1016D00073FE94F85F0094F85A30049094F85E001A
:1016E00094F85920039094F85D0094F858100290F3
:1016F00094F85C00019094F85B000090374806F085
:1017000099FE284600F022FA284600F083FA04F1F8
:10171000440584F8600004F1640000F023FC00211B
:10172000284600F0C3FB012000F038FD00212846C8
:1017300000F0D2FB012000F04FFD2046FFF7E4FE51
:1017400000F0B4FA264806F075FE4FF4FA7016F071
:10175000DBFB054660BB234806F06CFE224806F022
:1017600069FE224806F066FE214A2249224806F018
:1017700061FE2249224806F05DFE224806F05AFE2C
:1017800004F12101204806F055FE2049204806F0CA
:1017900051FE07A804F07EFA07A806F0A1FD014655
:1017A0001C4806F047FE114806F044FE0BB030BD61
:1017B000194806F03FFE284616F0AEFBCEE700BF04
:1017C0009DB20108B3B20108CAB20108DFB2010834
:1017D000A0860100FAB2010855B2010810B3010851
:1017E00045B3010878B3010809E40108B6B301085C
:1017F000E7B30108F1B301081DB401082DB40108D5
:1018000034B401083FB401085FB401086AB40108A8
:1018100070B401088AB40108ACB301082DE9FF4196
:1018200000F14805284600F0F1FB04240226284F69
:10183000013C14F0FF0433D0A12301223946009665
:10184000284600F0E7FB4FF4004380460093042253
:10185000A12302A9284600F007FCB8F1000F01D12E
:101860000028E5D09DF80830442B20D19DF80930A0
:101870006E2B1CD10DF10A0006F0C7FE02230130C9
:1018800084B221460DF109008DF8083006F0E5FE1E
:10189000002303220093A02302A9284600F0BAFBEC
:1018A000284600F0B5FB204604B0BDE8F0814FF4B7
:1018B00088430024ADF808306E2300210DF10B00A1
:1018C0008DF80A3006F0C9FE0094A0230522E3E754
:1018D00090B1010838B50C46113105460CF094FF63
:1018E000214651F8583F28462B604B686B6038BD45
:1018F000024B186803685B68184700BF6407002044
:10190000024B186803689B68184700BF64070020F3
:101910002DE9FF41002315461370022206460D4FA4
:1019200004AC386804F8011D03680092D3F80C80F9
:10193000012233462146C04748B14FF4004238687F
:101940002946036800921C6901223346A04704B06F
:10195000BDE8F0816407002030B585B08DF80D201A
:101960000022074B8DF80C101C6803A92368009215
:10197000DD68022203462046A84705B030BD00BFFF
:101980006407002037B54FF40045064B1C682368F8
:1019900000951D6913460A4601462046A84703B034
:1019A00030BD00BF6007002037B50025054B1C681F
:1019B00023680095DD6813460A4601462046A8477D
:1019C00003B030BD6007002037B50225054B1C6809
:1019D00023680095DD6813460A4601462046A8475D
:1019E00003B030BD60070020024B186803681B6815
:1019F000184700BF60070020024B186803685B6847
:101A0000184700BF60070020024B186803689B68F6
:101A1000184700BF600700204FF47A735843B0FBAB
:101A2000F3F00AF0EDB810B50446FFF771FC21465B
:101A3000BDE81040FFF7F2BE10B5424C0BF08AF93A
:101A400020460222002103F06FFE012220461146AB
:101A500003F06AFE20460122022103F065FE2046C3
:101A60000222032103F060FE20460022042103F03D
:101A70005BFE20460222082103F056FE204601228A
:101A8000092103F051FE204601220A2103F04CFEF9
:101A9000204602220B2103F047FE03F0FBFB00234C
:101AA00020461A460C2103F001FE204600220C219C
:101AB00003F0CAFE2046002204F580640F2103F0E3
:101AC00033FE20460122002103F02EFE2046002294
:101AD000022103F029FE20460022032103F024FE08
:101AE00020460222062103F01FFE20460022082184
:101AF00003F01AFE20460022092103F015FE2046BD
:101B000001220C2103F010FE204602220D2103F0D9
:101B10000BFE204602220E2103F006FE2046022282
:101B20000F2103F001FE002304F5806420461A46CD
:101B30000D2103F0BBFD2046BDE8104000220D2121
:101B400003F082BE0000024004F00CB91D4B00B54A
:101B50001A6889B0D2075FBF1B4A106001221A6061
:101B60001A4B1B4A04931B4B05931B4B03931B4BB4
:101B700002931B4B079308AB43F8082D93E803002F
:101B80008DE8030002AB0FCB13F04CF890B1154871
:101B900006F050FC00221448114603F0C5FD0F2347
:101BA00002220021104803F05FFC09B05DF804EB4D
:101BB00012F0D2BF69210D4809B05DF804EB00F0C6
:101BC000FBBB00BF5C07002064070020F118000881
:101BD000191A0008011900081119000859190008FC
:101BE00035840008C6B5010800000240D7B50108D9
:101BF000002307B5ADF8043001238DF806300198B5
:101C00000BF004F803F046FB03B05DF804EB0BF0B7
:101C10004FB80000194B10B51A688CB0D2075FBFDF
:101C2000174A106001221A60164B0793164B059352
:101C3000164B0693164B0893164B0993164B0A93B3
:101C4000164B0B930CAB13E907008DE8070005ABAF
:101C50000FCB12F0CDFC044601220F21104803F0F7
:101C600063FD3CB10F4806F0E5FB12F09FFC2046F7
:101C70000CB010BD0C4806F0DDFBF8E7580700205B
:101C80006007002085190008A9190008C919000873
:101C9000E9190008F9190008091A00083584000834
:101CA0000000024048B501087BB501082DE9F04F5E
:101CB000A9B00BF045FBDFF80C9168B9384B394AF5
:101CC000CDE923332292384A0093CDF880902192B7
:101CD00020AB0FCB0BF03AFB344B00251993344B60
:101CE0004FF0010A1893334B4FF003081A93324B0D
:101CF0002B4C1B93314B2C4F1C930423294E09A9C9
:101D000018A8CDE909351D941E971F968DF829A0B6
:101D100007F054F807F046F816F060FF2946142241
:101D200023A80C95CDF82C8016F051F9EE460DF154
:101D3000A00C4CF8186DBCE80F00CDE92047AEE8C8
:101D40000F009CE803008EE803000DF1800B0BA947
:101D50009BE80C0003C90CF029F9294610220EA8B3
:101D600016F035F9164BCDE91244CDF834808DF8D4
:101D70003EA002AC0DADCDE915761793CDF850908D
:101D80000FCD0FC42B68236016AB93E803008DE8DA
:101D9000030012AB0FCB0CF061FD29B0BDE8F08F52
:101DA00035840008418500086D85000835CC0008A1
:101DB000FDCA00080DCA0008A5C90008B9C9000875
:101DC000271A0008515D00082DE9F047044603F08A
:101DD00077F91E49054615F0BDFB15F081FD01465A
:101DE0001B4806F027FB4FF08041284615F050FDB8
:101DF00048B30025DFF86090DFF85080154E03F0FF
:101E00005FF94946074615F057FDA8B941463846DF
:101E100015F0A0FB15F064FD0146304606F00AFB04
:101E2000236885F001052046DB68294698474FF472
:101E30007A7003F057FAE2E723682046BDE8F047DE
:101E4000DB6800211847BDE8F08700BF00007A4436
:101E500099B50108ABB501080000204008B50D494F
:101E6000012003F0D5FD0C490B2003F0D1FD0B49F7
:101E70000A2003F0CDFD0A49042003F0C9FD0949F9
:101E8000072003F0C5FDBDE808400749052003F021
:101E9000BFBD00BFB9A0000801A4000871A20008DE
:101EA00021A5000875A40008FDA40008002310B5B2
:101EB0000C461A460D21074803F0F8FB14B1012C1B
:101EC00000D010BD2246BDE810400D21014803F0AE
:101ED000BBBC00BF00080240002310B50C461A46E8
:101EE0000C21074803F0E2FB14B1012C00D010BD17
:101EF0002246BDE810400C21014803F0A5BC00BFFC
:101F00000000024012F0C4BC084611461A4612F006
:101F10005DBD084611461A4612F0DABC0846114665
:101F20001A4612F00FBD00000C2110B1024803F058
:101F30007FBC014803F082BC0004024010B561B1CF
:101F4000FFF7E6F9044612F077FC01462046FFF75A
:101F5000A5FABDE8104012F087BDBDE8104012F0B0
:101F600071BD000070B588B0FFF7D2F91D49054674
:101F7000FFF794FA0C2106461B4803F059FC002396
:101F80000C211A46184803F091FB0021012004F0AF
:101F90002BF8102200210DEB020016F018F8134B5D
:101FA00002AC0293124B0693124B039308AB13E956
:101FB00003008DE8030094E80F0012F06DFD60B19E
:101FC00012F066FC01460C4806F034FA3146284609
:101FD00008B0BDE87040FFF7BDB9084806F02AFA1E
:101FE000F4E700BF0000404000040240291F000841
:101FF000E55200089D60000830B6010846B60108A9
:10200000014803F08FBC00BFA086010003F05ABC5A
:1020100003F074BC2DE9F041069F1E4607F0030350
:10202000032B80460C46154603D12F210D4800F0A6
:10203000C3F92046BC07324629460AD503F0ACFC5A
:1020400010B10120BDE8F0810123002088F80430A0
:10205000F8E7FB0702D503F0ADFCF1E703F08EFCD7
:10206000EEE700BF74B601082DE9F041069C0D466D
:10207000E107804616461F4603D54C210D4800F067
:102080009BF9A20703D54F210A4800F095F92304D4
:102090003A46314628460AD503F09AFC10B1012091
:1020A000BDE8F0810123002088F80430F8E703F050
:1020B00057FCF3E774B6010808B50321034803F0A1
:1020C000CCFB003018BF012008BD00BF0004024057
:1020D0000A460248032103F0B7BB00BF00040240D8
:1020E00008B581B1012303211A460A4803F0DEFA3C
:1020F0000321084803F09CFBBDE808400322054883
:10210000114603F0B3BA0122BDE80840032101489B
:1021100003F00ABB0004024003F01ABE1FB501A879
:1021200006F0A0F801A803F0A5FD05B05DF804FBDA
:102130001FB501A806F096F801A803F0E9FE05B066
:102140005DF804FB03F052BE03F06ABE084603F0DC
:10215000E1BCDFB50023CDE90133ADF80C3001233C
:102160008DF807308DF808306FF01D038DF80930B9
:102170000723044601A88DF80A3006F098F8236872
:1021800006461B6820460F469847864277EB0103B8
:10219000B4BF0120002004B0D0BD0000042817D82F
:1021A000DFE800F00309100E1200002303211A4695
:1021B000084803F07BBA00220321064803F0B4BAB2
:1021C0000222F9E70122F7E70321024803F0D2BA1D
:1021D000704700BF00000240042817D8DFE800F075
:1021E0000309100E1200002302211A46084803F0CA
:1021F0005DBA00220221064803F096BA0222F9E7EE
:102200000122F7E70221024803F0B4BA704700BF89
:10221000000002402DE9F04742488AB006F00AF972
:1022200009F0A4FB2425079007993F4806F002F91E
:102230000798684306F09AF904463C4806F0FAF815
:1022400094B107990DEB0502204609F0E9FE002341
:10225000DFF8F4A0364F07900893089A079B9A423C
:102260001DD3204606F06CF908F0BAFB044608F0CE
:10227000BDFB214602462F4806F0DCF82E4B2F48C6
:1022800019889A888B1A06F0D5F82D4B1B6803B174
:1022900098472C4806F0CEF80AB0BDE8F087089BB6
:1022A00005FB03431B7B013BDBB2032B98BF1AF8F2
:1022B0000320099B88BF3F22642B83BF6420B3FBAC
:1022C000F0F30899002382BF05FB01418969B1FB46
:1022D000F3F308990898DDF820C0DDF820E0DDF878
:1022E0002080DDF8209005FB004005FB0949D9F866
:1022F0001C6005FB0141CDE9033605FB08439B69E2
:10230000029305FB0E439B68019305FB0C431B8C5A
:10231000009303694968384606F08CF8089B01333E
:1023200008939AE714B7010820B701082BB70108F2
:1023300060B7010892B7010872550020B1B70108D3
:10234000E007002084B1010810B70108014B1860B4
:10235000704700BFFC07002073B5124C0646237877
:102360000D46114A1BB913780BB172B6FEE7012373
:10237000002113700D48642215F029FE2B460096AB
:102380000B4A6421094816F091FC0A4B1B6803B103
:1023900098470125054E304606F090F872B6257034
:1023A000F9E700BFD80700206C0700206E07002067
:1023B000E8B70108FC070020F7B5164C064623785D
:1023C0000D46154A1BB913780BB172B6FEE701230F
:1023D000002113701148642215F0F9FD2B46009678
:1023E0000F4A64210D4816F061FC0E4B1B680BB1BF
:1023F0000A4898470C4B1B6803B198470125074FC3
:102400000A4E384606F05AF8304606F057F872B6CB
:102410002570F6E7D90700206D0700206E07002021
:1024200010B8010868070020FC0700201FB8010849
:102430000368DFF888C080B5CCF80030164F4368D9
:10244000164E3B608368164D3360C36815492B6098
:102450000369154A0B604369144C13608369C069B2
:102460002360134B1860DCF8000038683068286877
:102470000968104812680021226864221B6815F060
:10248000A6FD23680C4A64210A4816F00FFC09488F
:1024900006F014F8FEE700BFEC070020F407002068
:1024A000F8070020F0070020D4070020DC070020F8
:1024B000E40700206E070020D5B70108E8070020D8
:1024C000074B1B6803B198471EF0040F0CBFEFF3D6
:1024D0000880EFF309808169004A10473124000821
:1024E000FC07002010B50446C06908B106F028F8C2
:1024F000206908B106F024F8606808B106F020F8F9
:10250000204610BD10B50446006808F027FF20469D
:1025100010BD0000CB210148FFF74EBF3BB80108BA
:10252000FE2307B502A901F8043D054B18680023F6
:1025300000681A4608F002FC03B05DF804FB00BF17
:102540000C080020D0B51F467423C0E900310023D9
:10255000044683600820164611F08EFFC0E900672C
:10256000A0602046D0BD00002DE9D043DDE906671C
:1025700099467223C0E9003100239642836077EBCD
:1025800009030446904603DA2B210748FFF714FF9E
:10259000102011F071FFC0E90089C0E90267A06056
:1025A0002046BDE8D08300BF85B80108036837B571
:1025B000632B04460D4601D0FFF7ACFF002302AAAF
:1025C00042F8043DA168284605F01AFD019B1BB1A5
:1025D00038210248FFF7F0FE03B030BD85B801088E
:1025E00070B563230025C0E90031044685601A20D8
:1025F000164611F041FF1A22294615F0E8FC314633
:10260000A0602046FFF7D2FF204670BD816470476E
:10261000C16470472DE9F843D0E90173884600256D
:102620004FF00C09DB1B0A4E9B105E43ECB2B44228
:102630000BD209FB04724146506816F08BFB013542
:102640000028F3D12046BDE8F8834FF0FF30FAE7C9
:10265000ABAAAAAA2DE9F843D0E90473884600255D
:102660004FF00C09DB1B0A4E9B105E43ECB2B442E8
:102670000BD209FB04724146506816F06BFB013522
:102680000028F3D12046BDE8F8834FF0FF30FAE789
:10269000ABAAAAAA2DE9F0410E4649680446FFF705
:1026A000B9FFC0B2FF2803D07C212948FFF784FE80
:1026B000D4E90123274F9B1A9B107B437E2B03D920
:1026C0007F212348FFF778FED4E901120C25E0684A
:1026D000531A9B10121A7B4392107A430133934290
:1026E00005FB03F80ED84144A160D4E9013496E813
:1026F0000700E31A04E9070016489B105843013805
:10270000BDE8F081404605F031FF054618B9692162
:102710001148FFF751FED4E901C30027A3EB0C03D6
:102720009A100C4B5343002B09DD05EB070E0CEB05
:10273000070207CA013B8EE807000C37F3E7604643
:1027400005F0FEFE65604544C4E90255CDE700BFD3
:1027500085B80108ABAAAAAAEEB801081FB56E2376
:10276000CDE90131002301A90393FFF793FF05B0E1
:102770005DF804FBFF2270B5002380F828204FF09D
:1027800000424FF0FF31C0E90D23C2636FF07F427A
:10279000C0E910120522C0E90033C0E91423C0E9E2
:1027A00002330022C0E90433C0E90633C0E908332C
:1027B0000363C0E9123383654FF000431E4DC0E947
:1027C00018232A68044612F0010213D101211B4E7E
:1027D00008463260716008F0D7F9306018B91221EC
:1027E0001748FFF7E9FD0123164A174913482B60E4
:1027F00013F07BFF154B1A680AB9104A1A60144986
:102800002046FFF7ABFF134B134918702046FFF724
:10281000A5FF124B124918702046FFF79FFF114B7E
:10282000114918702046FFF799FFFE220F4B1870D0
:102830000F4B20461A7070BD080800209008002039
:1028400041B9010800000020052500080C080020FF
:1028500083B90108140800208BB901081208002070
:1028600093B901081008002098B901081308002046
:102870001108002010B5084C2368DB0709D407486D
:10288000FFF778FF0123064A06490448236013F046
:102890002CFF024810BD00BF0408002028080020BB
:1028A00000000020E52400082DE9F0410E464968AB
:1028B0000446FFF7CFFEC0B2FF2803D08721294886
:1028C000FFF77AFDD4E90423274F9B1A9B107B4323
:1028D0007E2B03D98A212348FFF76EFDD4E9041229
:1028E0000C25A069531A9B10121A7B4392107A434D
:1028F0000133934205FB03F80ED841446161D4E9EA
:10290000043496E80700E31A04E9070016489B1010
:1029100058430138BDE8F081404605F027FE0546E2
:1029200018B969211148FFF747FDD4E904C300270E
:10293000A3EB0C039A100C4B5343002B09DD05EB62
:10294000070E0CEB070207CA013B8EE807000C37A5
:10295000F3E7604605F0F4FD25614544C4E90555FB
:10296000CDE700BF85B80108ABAAAAAAEEB8010856
:1029700038B5D0E901239B1A074A9B105343CDB2C7
:102980009D42044603D3A6210448FFF715FD0C2001
:10299000636800FB053038BDABAAAAAA85B8010858
:1029A00038B5CCB2114905460B6813F0010307D1C5
:1029B0000F4A70201372012310600E480B605060A4
:1029C000FF2C10D0D5E904239B1A0B4A9B105343CC
:1029D0009C4203D3B2210948FFF7EEFC0C2328697F
:1029E00003FB040038BD0248FCE700BF00080020DC
:1029F00018080020CFB80108ABAAAAAA85B8010818
:102A000010B5D0E90730C9B2D2B2834209D01C78E0
:102A10008C4204D15C78944201D1987810BD033384
:102A2000F3E74FF0FF30F9E72DE9F041D0E9042357
:102A30009B1A484A9B1053430D4609780446994215
:102A400003D393214448FFF7B7FCD4E901239B1A31
:102A5000404A9B1053436978994203D394213E48DE
:102A6000FFF7AAFCD4E904239B1A3A4A9B1053436C
:102A7000A978994205D3FE2903D095213648FFF75E
:102A80009BFC6A7829782046FFF7BAFFC3B2FF2B78
:102A900006461BD029782046FFF782FF697820463A
:102AA000FFF766FF31462046FFF77AFF2978204678
:102AB000FFF776FF69782046FFF75AFFA97820468E
:102AC000FFF76EFF9C212448FFF776FCD4E907232B
:102AD000204F9B1A7B437E2B03D99F211E48FFF773
:102AE0006BFCD4E90762616A931B7B43521A57431C
:102AF0000133BB4203EB43080AD8464426622A88C6
:102B0000236A23F8032CAA7803F8012CBDE8F0818E
:102B1000404605F02BFD064618B969210F48FFF71E
:102B20004BFCD4E90702131A0A4A5A430023002A2D
:102B30000ADDC118B1F800C0F71826F803C089787B
:102B4000013AB9700333F2E705F0FAFCE661464456
:102B50006662D3E7ABAAAAAA85B80108EEB8010855
:102B600013B5FF24084A02AB106803F8044D0A4667
:102B70000068194608F086F9012814BF20469DF820
:102B8000040002B010BD00BF0C08002038B58168F9
:102B900000681D46144605F099FD0346201845EBD4
:102BA000E37138BD08682DE9F04172281F461FD037
:102BB00074280FD0632820D1886805F0E1FA002836
:102BC00071F1000304460D460EDADD210D48FFF7D2
:102BD000F3FB09E08B68D3E90045B5F1004F08BF6E
:102BE000002C01D0A4187D4120462946BDE8F08183
:102BF0008868BDE8F041FFF7C9BF00244FF00045E9
:102C0000F2E700BF85B801082DE9F0410F460646FE
:102C10000024FFB2FFF7C4FED6E90758454511D09E
:102C20002B78BB420CD169783046FFF7A1FE0368D0
:102C3000692B05D183681B6803B198470134E4B25E
:102C40000335EBE72046BDE8F0812DE9F3418046EE
:102C50000F460025FFF7A4FED8F81C40D8F82060E6
:102C600003340336FFB2A6421BD0234633F8032DAC
:102C70009B78ADF804208DF8063014F8033C9F4291
:102C80000DD19DF805104046FFF772FE0368692BD1
:102C900005D183685B6803B198470135EDB2033411
:102CA000E1E7284602B0BDE8F0810000836C73B50F
:102CB00004460D46164623B94FF48C710B48FFF7B6
:102CC0007BFBCDE9006423462A460949094808F000
:102CD00025FC012807D04FF48F71044802B0BDE8ED
:102CE0007040FFF769BB02B070BD00BF85B8010836
:102CF000E3B801087D32000838B590F84730044643
:102D0000032B0D4604D940F231110648FFF754FB5E
:102D100094F847305A1C84F847201C4484F84250E9
:102D200038BD00BF85B8010810B590F8473004469B
:102D300023B94FF49B710648FFF73EFB94F84730E8
:102D4000013BDBB284F847301C4494F8420010BDCC
:102D500085B80108CBB2FE2B10B504460AD0FFF7A8
:102D60001FFE03686D2B05D1017A2046BDE8104097
:102D7000FFF716BE10BD00002DE9F84304460026FB
:102D8000114FD4E904239B1A9B107B435FFA86F80A
:102D9000434516D941462046FFF7DCFFD4E90759E1
:102DA000A9450CD02B78434507D169782046FFF719
:102DB000DFFDA9782046FFF7CDFF0335F0E70136A8
:102DC000DFE7BDE8F88300BFABAAAAAA38B505467D
:102DD000002495F84730A34207DD2B1993F84210E1
:102DE0002846FFF7DDFD0134F3E738BD00232DE968
:102DF000F74FC0E9083388461946D8E907594FF01C
:102E000000430446C0E90613C0E90013C0E90213F9
:102E1000C0E90413FF208A469B46D2B284F8200002
:102E200001924D45D4E9006720D02B78019A934256
:102E30001AD169784046FFF79BFDDDE90C23014676
:102E40004046FFF7AFFE594508BF50450CD05F45DF
:102E500008BF564503D0B04271EB070304DA6B7824
:102E6000C4E9000184F820300335DAE7B7F1004FF8
:102E700008BF002E08D0DDE90C23B21A67EB03036C
:102E800016461F46C4E90467204603B0BDE8F08F2C
:102E9000F8B50D460B4B896906464B434FF47A71E2
:102EA000B3FBF1F1FFF75CFE0446C7B2B06C0368F8
:102EB0001B689847FF2FC6E90E010CBF95F820004C
:102EC0002046F8BD40420F0038B5C36C04460D469D
:102ED0001BB9BDE83840FFF7DBBF806C17490368BA
:102EE0005B699847A06C0368DB689847D5E90201E5
:102EF00005F020FA0146124805F09CFAA06C036820
:102F00009968D5E902238847A06C03681B69984734
:102F1000E36C9847A06C0368DB689847A06C036873
:102F20001B689847C4E90E0100212046FFF718FEF0
:102F3000C0B2FE2808BF95F8200038BD2125000842
:102F40002EB90108F8B5D1E90667B7F1004F08BFFF
:102F5000002E05460C4608D11AB1BDE8F840FFF72F
:102F600097BFBDE8F840FFF7AFBF012E77F1000330
:102F700002DA91F82000F8BD92B121462846FFF709
:102F800087FF94F82030C0B28342F4D1D5E90E67B0
:102F9000D4E90023964277EB0303B8BFFF20EAE7AA
:102FA000D0E91423964277EB0303E6DBFFF78CFFAF
:102FB000E7E700002DE9F04F8FB004460D46FFF71C
:102FC000EFFC03680646702B04D04FF49E714F4807
:102FD000FFF7F2F9A06C03681B6898472A46C4E91A
:102FE0000C01CDE90001214604A8FFF7FFFE2946A8
:102FF0002046FFF709FE9DF83030FF2B05D120B9A0
:1030000040F247114148FFF7D7F99DF83010FF29EA
:1030100065D100224FF00043CDE90823DDE9042308
:10302000CDE90623DDE90823CDE90A23A36DEBB141
:103030009847DDE90423D4E91889B3F1004F08BFAC
:10304000002A09D0DDE9082318F10B0049F100013D
:10305000904271EB030309DAD4E90C2312EB080068
:1030600043EB0901CDE90A89CDE90601327A04A9C9
:103070002046FFF767FFA36D074603B19847FBB2F1
:10308000FF2B3BD1DDE90401D4E90EABA36DB0EB1E
:103090000A0861EB0B09CDE90889CDE90601CDE904
:1030A0000A89002BE2D0D4E91823B1F1004F08BF00
:1030B0000028CDE9022307D012F10B0043F10001F3
:1030C000404571EB0903D1DADDE90223CDE90A239A
:1030D00012EB0A0243EB0B03CDE90623C6E72046B9
:1030E000FFF746FCD4E90C01DDE90423121A63EB77
:1030F000010317469846CDE908788FE72946204610
:10310000FFF7A3FD38460FB0BDE8F08F85B8010882
:1031100070B504460D46FFF743FC03686D2B11D0D4
:10312000702B09D0612B14D1836894F8411094F866
:103130004000BDE87040184729462046BDE8704071
:10314000FFF738BF034840F22B11FFF735F94FF076
:10315000FF3070BD85B80108F8B590F828300446F6
:10316000FF2B04D14FF4E3714148FFF725F994F8A0
:1031700028102046FFF714FC94F8283084F84630D5
:1031800094F846102046FFF70BFC036805466D2BAC
:10319000204694F846100BD1FFF7AEFD297A204661
:1031A00084F84610FFF7FCFB2046FFF70FFEE7E729
:1031B000FFF7AEFFC3B2FF2B06460BD140F2DB1187
:1031C0002B48FFF7F9F840F2DB112A4B2A4A28482E
:1031D00014F086FD024694F846102046FFF710FCD6
:1031E000C5B2FF2D09D140F2E1112148FFF7E4F803
:1031F000204B214A40F2E111E9E794F84610FE2DF8
:10320000204621D1FFF790FD074601462046FFF7F3
:10321000C7FB324639462046FFF7F2FBC5B2FF2D09
:103220000DD131462046FFF7A3FB40F2ED111048C7
:10323000FFF7C2F80F4B104A40F2ED11C7E72046E6
:10324000FFF7C4FD3946DAE7FFF7AAFB314620460F
:10325000FFF78EFB29462046FFF7A2FB94F8463085
:1032600084F8416084F8403084F8465088E700BF15
:1032700085B80108DDB80108A0B9010808B5FFF755
:10328000F9FAFFF769FFD0B51F461646FFF770FB46
:1032900003688468742B01D0FFF73CF9C4E9006728
:1032A000D0BDD0B5044616461F46FFF761FB324637
:1032B0003B4601462046BDE8D040FFF773BC000006
:1032C000836C10B5044623B940F297210248FFF7FA
:1032D00073F8A06C10BD00BF85B80108FF23054A34
:1032E0001370054A1370054A1370054A1370054A96
:1032F00013707047140800201208002010080020E6
:103300001308002011080020014B1878704700BFF7
:103310001008002010B50446006808F01FF8204689
:1033200010BD00002DE9FF480BF0E2FB4FF6FF71E6
:103330002B4A13888B421CBF01331380FFF79AFA84
:10334000FFF7BEFF03681B689847264B5A78EAB917
:10335000254AD288D2B1254CD4E900BCBCF1004F3B
:1033600008BFBBF1000F0FD083457CEB01040DDAE1
:103370001F4CB0EB0B0604FB02F461EB0C07E517E6
:10338000A64277EB050201DB01225A700022ADF85C
:103390000C205A782AB101228DF80C20134AC2E978
:1033A00000011B78134CBBB1012513488DF80D505B
:1033B00005F040F82570114B11481A78114B197817
:1033C000002300930068039B0BF0D4FC30B10E4B3C
:1033D000187804B0BDE8F0882370ECE70B4BF7E7F2
:1033E000DA080020BC080020C80800205000002097
:1033F00080510100C508002019BA0108BF0800204B
:10340000B8080020BE080020100800201208002084
:1034100008B5184BDB8813B9174B187808BD174B44
:10342000D3E90023B3F1004F08BF002AF4D1144AB6
:1034300013780133DBB2032B1370EDD8012B0BD9BA
:103440000A21002005F042F90E4B58434FF47A73DD
:10345000B0FBF3F008F0D4FB00230B4A13700B4AC7
:1034600013700B4A13600B4A1370012353700A4BFD
:10347000D3E700BFC8080020100800204800002043
:10348000F008002040420F00BF080020BE080020C6
:10349000B8080020BC0800201308002008B500234D
:1034A0001A4607F04BFC431E5842584108BD000025
:1034B00007B50B78012B0FD004D3022B10D003B02B
:1034C0005DF804FB002302A941F8043D064B1B688C
:1034D0001868FFF7E3FFF2E702A94FF0FF33F3E7C5
:1034E000014B04311B68F3E7A80800201FB57023C7
:1034F000CDE90131002301A98DF80C30FFF7D4F993
:1035000005B05DF804FB00002DE9F04F4A4B85B093
:103510001A780446002A40F08B80012747491F7023
:10352000FFF71CF9464B474918702046FFF716F97C
:10353000DFF868A144498AF800002046FFF70EF939
:10354000DFF85C910A22002389F800003F4901A8B6
:10355000FEF7F8FF01A92046FFF79CF83C4E3D49D5
:1035600030702046FFF7FAF83B4B3C491870204674
:10357000FFF7F4F83A4B3B4918702046FFF7EEF896
:10358000394B3A4918702046FFF7E8F8384B394A6A
:10359000187039492046FDF781FADFF808B1374A3B
:1035A0008BF8000036492046FDF778FA3549054684
:1035B0002046FFF79BFF70230193334B804601A900
:1035C000204602938DF80C70FFF76EF907462F4ADC
:1035D0002B4612789BF800102046FDF76AFA434606
:1035E0009AF8002029462046FDF763FA3B4699F8F1
:1035F000002029462046FDF75CFA2B4632784146EA
:103600002046FDF756FA2B46327839462046FDF71C
:1036100050FA1F4A2B46127829462046FDF749FAF0
:103620001C4B1D4A1B78127829462046FDF741FAAB
:1036300005B0BDE8F08F00BFF10800203BBA0108DB
:10364000C008002045BA010850BA01085CBA010858
:10365000A108002069BA0108D908002077BA01083A
:10366000D808002083BA0108DC08002090BA0108BD
:10367000DD080020253300089EBA01082D4400080B
:10368000A8BA0108BCBA0108CFBA01081008002086
:10369000130800201108002014080020C40800208E
:1036A000A0080020C208002008B50BF0FFF918B1EF
:1036B000BDE808400BF01CBA08BD08B50BF0F6F9E0
:1036C00018B9BDE808400BF0CDB908BD30B50446C7
:1036D00085B00D46FFF718FF6D22064B01A91B7838
:1036E0002046CDE901258DF80C30FFF7DDF805B057
:1036F00030BD00BFC20800202DE9F84F424B434DBA
:103700001A68044612F0010F01BFFF222A7001223D
:103710001A602B78FF2B73D1FFF7F6FE3C4A3D4928
:103720002046FDF7BBF93C4A28703C492046FDF78E
:10373000B5F93B4F3B4A38703B492046FDF7AEF99F
:103740003A4E3B4930702046FFF7C0FF3949824668
:103750002046FFF7CBFE384983462046FFF7C6FEDA
:103760008146364A3B78127829782046FDF7A1F940
:10377000334ADFF8E0803378127829782046FDF765
:1037800098F9337898F8002039782046FDF791F9B8
:103790002B7898F8002031782046FDF78AF9294ADD
:1037A0005B46127839782046FDF783F926493B7845
:1037B0000A7820465946FDF77CF9244A4B46127890
:1037C00039782046FDF775F91F493B780A7820467D
:1037D0004946FDF76EF91A4A534612783178204669
:1037E000FDF767F9337898F8002051462046FDF739
:1037F00060F9174A2B78127831782046FDF759F98D
:103800002878BDE8F88F00BF9C080020F30800204E
:103810009D3E0008DFBB0108413A0008E9BB0108F2
:10382000C108002011340008F3BB0108C3080020C0
:10383000FDBB010809BC010817BC0108C008002035
:1038400013080020C4080020A1080020120800204E
:10385000100800201408002038B504460D46FFF774
:1038600053FE034A29462046FDF718F938BD00BF2C
:10387000593C0008344B2DE9F04F1A8900230446C7
:1038800089B0CDE900230391002300222F4905A828
:10389000FEF76AFE05A92046FEF7FCFE2C4982468B
:1038A0002046FFF723FE2B4983462046FFF7D4FF2F
:1038B000294A804629492046FDF7F0F8284A05465E
:1038C00028492046FDF7EAF80646274FDFF8A8907A
:1038D0003B7899F8002029462046FDF7EAF8234A6C
:1038E0005B46294620461278FDF7E3F8204A434616
:1038F000294620461278FDF7DCF8334652465946F1
:103900002046FDF7D6F83346524641462046FDF79D
:10391000D0F8184A3B78414620461278FDF7C9F89E
:103920003B7899F8002031462046FDF7C2F86D2318
:103930000593039B05A9204606938DF81C50FEF7BE
:10394000B3FF09B0BDE8F08FC808002026BC01080D
:1039500033BC010843BC0108BD3F000854BC01084A
:103960000933000863BC010811080020DC080020AE
:10397000DD080020D9080020100800202DE9FF47AD
:1039800090468A461E4A1F490446FDF787F81E499D
:1039900005462046FFF7AAFD1C4981462046FFF751
:1039A0005BFF06461A4A4B46294620461278FDF729
:1039B00080F8184A184F3346294620461278FDF7FA
:1039C00078F83B78424649462046FDF772F83B7846
:1039D000424631462046FDF76CF8104A3B78127893
:1039E00031462046FDF765F86D2301A92046CDE953
:1039F000013A8DF80C50FEF757FF04B0BDE8F08790
:103A0000E13F0008B4BB0108BEBB0108CEBB010802
:103A1000DC080020DD08002011080020D908002063
:103A200070B50D460446FEF725FF044922462B4695
:103A3000BDE870400978FFF726BC00BFA108002050
:103A4000F7B5504C2668A6B9082010F015FD0546BC
:103A50000660012032466860042107F095F828606E
:103A600018B912214848FEF7A7FC484825600BF01A
:103A700055F8474D474F2B6801332B600BF038F852
:103A80003B781BB901233B700BF05EF8002302A9C1
:103A900041F8043D2368404A186807F0F3F901280B
:103AA00004D04FF4C7713D48FEF786FC019E731C9D
:103AB00042D12B68042B0CD90FF080FD037843B161
:103AC0004FF47A7008F09CF840F299113348FEF7F1
:103AD00073FC00233B702B681E22013BDBB21E2BC4
:103AE00028BF1E2302FA03F32D4A93421DD8B3F5D3
:103AF000616F1C464FF0000519D2B3F5167F75F1C2
:103B0000000317DA3C2C75F10003ACBF1E210A211B
:103B1000002004F0DBFD0346201845EBE371FFF7BE
:103B20007FFF204B187803B0F0BD00251C4C4FF4EC
:103B30001671EDE73C21EBE72EB130460021FFF78F
:103B40006FFF194BEEE72E600AF08CFFFEF792FE36
:103B5000FFF7B6FB03681B689847144BC3E90001E5
:103B600023686BB130460AF0D9FF256835B1286863
:103B700007F0F4FB0821284610F09EFC0023236088
:103B80000B4BCFE7A808002041B90108B134000869
:103B9000EC080020E8080020A0860100C5B9010853
:103BA00000A3020012080020C408002040000020EA
:103BB00014080020054B1870054B1A700022054BA5
:103BC0001960054B1A705A70704700BFBF0800207B
:103BD000BE080020B8080020BC0800200279016857
:103BE0004079FFF7E7BF08B50BF0BCF8C0B2DE289C
:103BF00028BFDE2008BD00004FF47A7337B50024DB
:103C000003FB00F2074802A9056841F8044DB2FB26
:103C1000F3F2286807F036F9012814BF204601980E
:103C200003B030BDA40800204FF47A7337B50024E8
:103C300003FB00F2074802A9056841F8044DB2FBF6
:103C4000F3F2286807F060FA012814BF20460198B3
:103C500003B030BDA40800202DE9F04F99B0FEF765
:103C600009FE90F84630044603930026FFF71CFD3A
:103C70004FF00009214DDFF89080A06C0EAF036873
:103C80001B6898479DF80C20CDE9000121460EA83D
:103C9000FFF7ACF80FCFDDE912AB0DF1100CACE87B
:103CA0000F000FCFACE80F003B688CF80030DDE967
:103CB0000E23B3F1004F08BF002A03D0D04579EBA3
:103CC0000B0313DAAA46B34601274FF47A73AAFB13
:103CD000030103FB0B11FFF7A7FF48B10122084BBB
:103CE0005A72084B187819B0BDE8F08F0027ECE73E
:103CF000002FC2D19DF83000F5E700BF80510100D0
:103D0000AC080020D90800208551010010B5002022
:103D10000021FFF789FF10B1084B187810BD084C3F
:103D20002368984720B9074B1B780BB9064BF4E77B
:103D3000637A0BB1054BF0E7054BEEE7D90800209D
:103D4000AC080020DE080020100800201408002025
:103D500013080020022818BF00200BF0B1B90000A2
:103D6000F8B53B4B05461E78002E6FD101271F701A
:103D70000AF090FB374928460FF0C8FAC31F052BFD
:103D8000354C42D820710E233449284663710FF018
:103D9000C6FA3349074614F0DDFF00283AD1E06047
:103DA000304928460FF098FA2F49607028460FF0E6
:103DB000ADFAB0F57A7F3AD8E0802C4928460FF06A
:103DC000A5FA42F21073984236D820812849284635
:103DD0000FF082FA2749A07028460FF097FAB0F545
:103DE0007A7F2ED26081244928460FF075FAE07060
:103DF00036B1224804F01EFB71212148FEF7DCFA9F
:103E0000E068BDE8F840FFF7A5BF1E4804F012FBCC
:103E10003E46B8E71C49384614F09CFF10B902230F
:103E2000E360BDE7194804F005FB0126B8E7184830
:103E300004F000FB0126C0E7164804F0FBFA012657
:103E4000C4E7154804F0F6FA0126CCE7F8BD00BF38
:103E5000F2080020E3BA0108C8080020FCBA0108F3
:103E60009FBB01081FBB010823BB01084ABB010817
:103E70000BE3010872BB01089CBB0108A1BB010850
:103E8000C5B90108E6BA01080CD4010803BB010852
:103E90002CBB010853BB01087DBB010870B5234B47
:103EA000C0B21B78984206D10FF088FB0FF040FAA1
:103EB0001F4B187870BD1F4D0FF080FBFFF750FFB0
:103EC00095F905000CF0B4FC0AF0EEFF28790CF02F
:103ED0007DFC0AF0DDFF68780BF0BCF8164B1A6821
:103EE0001C4612F0010213D10421144E0846326020
:103EF000716006F049FE306018B912211048FEF7D3
:103F00005BFA01230F4A10490C48236012F0EDFBC5
:103F10000E4B1A680AB9094A1A600D480BF0D6F818
:103F2000EB780BB10B4BC4E70B4BC2E7C308002087
:103F300014080020C808002098080020E00800208D
:103F400041B901080000002015330008A408002032
:103F5000C5430008C008002013080020034B93F855
:103F60003230022B0CBF022000207047D800002006
:103F700008B5FFF7F3FF30B90AF098FD18B9BDE8AE
:103F800008400AF06FBDFFF7E9FF022806D10AF0EA
:103F90008DFD18B1BDE808400AF0AABD08BD0000BB
:103FA00008B5FFF7DBFF02280CBF024B024B187865
:103FB00008BD00BFDD080020DC080020054B1B8980
:103FC00013B9054B18787047044B5B7A002BF8D176
:103FD000FFF7E6BFC808002010080020AC0800204A
:103FE000FFF7DEBF01232DE9F348324C002000210A
:103FF0006372FFF719FE10B12F4B187816E0236893
:10400000984710B92D4B1B788BB30BF065F801283E
:1040100071F1000306460F460BDBFEF72BFC324620
:104020003B46217AFFF72FF9FFF7BAFF02B0BDE850
:10403000F08823689847024670B1002364680093B3
:10404000ADF80430FFF7CFFD01466846A04768464B
:10405000FFF7C4FD1A4BD0E7184B1B783BB1194B47
:104060001B88022B23D80146FFF7A4FDF2E7164D6B
:104070006B89D3B1EB78C3B1FEF7FCFBFFF720F9F6
:1040800003681B6898476B89104A114D5A43D5E95C
:104090000067861B61EB0707D317B242BB4104DA06
:1040A00040F24A310B48FEF787F9002363720A4B4E
:1040B000A3E700BFAC080020D9080020DE080020DC
:1040C000D8080020DA080020C8080020805101002C
:1040D00040000020C5B90108100800202DE9F04F6C
:1040E0000446574D87B0C5E90023019100230A22F9
:1040F000544903A8FEF726FA03A92046FEF7CAFA98
:10410000514A8146287251492046FCF7C7FC504A63
:10411000054650492046FCF7C1FC4F49074620465A
:10412000FFF7D4FA4D498DF802002046FFF7DEF97B
:104130004B498DF803002046FFF78EFB4949824624
:104140002046FFF797FB8346474EDFF838813378E8
:1041500098F8002039462046FCF7ABFC434A3378F8
:10416000394620461278FCF7A4FC414A5B463946A2
:1041700020461278FCF79DFC3E492B460A782046E3
:104180003946FCF796FC394A2B46594620461278A8
:10419000FCF78FFC337898F8002059462046FCF74E
:1041A00088FC337898F8002029462046FCF781FCEB
:1041B0002E4A3378294620461278FCF77AFC2E4A9C
:1041C0009DF80230294620461278FCF772FC2949F6
:1041D0002B460A7820469DF80210FCF76AFC274A15
:1041E0009DF80330294620461278FCF762FC2B46E6
:1041F0004A469DF803102046FCF75BFC204A5346D4
:10420000294620461278FCF754FC2B464A46514674
:104210002046FCF74EFC337898F8002051462046A3
:10422000FCF747FC6D230393019B03A920460493ED
:104230008DF81470FEF738FB07B0BDE8F08F00BFB3
:10424000AC08002072BC0108E53F000882BC0108F0
:104250000D3D000890BC01089DBC010845BA01084D
:1042600050BA0108A9BC010811080020100800205C
:104270001308002014080020D8080020DC080020C3
:10428000DD080020D9080020F8B51D460023417143
:10429000BDF8181004460360C180174602B115B975
:1042A00023712046F8BD0749284610F001F906465B
:1042B00010B920712660F4E72A46394613F063FEF0
:1042C0002571F7E7E9F4010810B50446006808B164
:1042D00010F0F0F8204610BD70B5304E86B0326850
:1042E000044622B94FF4E6712D48FEF765F8002C1C
:1042F00051D000222B4B1A80D4E91C23134316D033
:10430000294B1D6807F02CFB01462848A847D4E933
:104310001C2303A803F0A6FFD4E91C23244903A807
:10432000C1E900232349C1E9002301F0A3FCFEF702
:10433000A1FAFEF7C5FF03681B6898471E4B1F4A8A
:10434000C3E90001237AC3F3C0031370637F13B37F
:10435000237F03B31A49082010F0A0F8054630B1B6
:104360006289237F617F0092A26EFFF78DFF039524
:104370008DB1002330681A4603A9006806F028FCB6
:10438000012808D0039C34B12046FFF79DFF082187
:10439000204610F091F806B070BD00BFA4080020C0
:1043A000C5B90108DA080020D80000202EBA01089B
:1043B000480000205000002040000020DE080020BF
:1043C000E9F4010810B50446FFF786FF24B1204642
:1043D000BDE810400CF096BD10BD000038B542F2AB
:1043E00010700AF0A1FB0446D0B10578022D13D15C
:1043F00040680021FFF714FBD4F89800FFF76CFF2A
:10440000237A13B10022084B1A7020460BF0DAFA17
:10441000032D06D1284638BD032DEDD10020E8E755
:104420000125FFF7A5FDF5E7C5080020002310B51D
:10443000134C84F836300AF039FB08B10AF058FB07
:10444000FFF7CCFF032812D8DFE800F002020705CF
:104450000C4B187810BD0C4BFBE7FFF77FFD0228D3
:1044600009BF0123094B84F83630094BF1E70948AD
:1044700040F2BB21FDF7A0FF4FF0FF30EAE700BF9D
:10448000D80000201408002013080020C4080020D1
:10449000A0080020C5B90108FF2300210D4A1370B0
:1044A0000D4A13700D4A13700D4A13700D4A1370A4
:1044B0000D4A13700D4A13700D4A13700D4A137094
:1044C0000D4A13700D4A13700D4AC2E900111372A0
:1044D000704700BFC2080020C1080020C3080020A8
:1044E000D9080020D8080020DD080020DC080020C2
:1044F000C0080020C4080020A0080020A108002057
:10450000AC08002010B101210FF0D6BF704710B5E4
:104510000446D0F8C802FFF7F5FFD4F8BC0210B18A
:1045200004210FF0C9FFD4F8B00210B104210FF03C
:10453000C3FF204610BD00007FB500240E4601A831
:104540002146CDE90144039412F086F8051E04DAF1
:1045500029460F4803F06EFF0EE001A9304611F026
:10456000E5FE08B1F36953B929460A4803F062FF32
:10457000284612F047F80024204604B070BD2846B3
:1045800012F040F804460028F6D129460248E1E737
:10459000EFBC010816BD01084CBD0108F8B5064680
:1045A0000F460024094D39463046FFF7C5FF50B984
:1045B0000134E4B20F2CF6D911F004FE3421284660
:1045C000FDF7FAFEEFE70120F8BD00BF77BD010857
:1045D0002DE9F0438046006A8DB003680C461B68E5
:1045E00098471C2206460F4605A8002113F0EFFC51
:1045F000E3886079ADF8283009F0C2FC012E8DF80F
:104600002D0077F100032079A8BF069603F0AEFFD6
:104610000546A8B32279216813F0B5FC607909F04A
:10462000B7FC41288DF82E0005D042282BD0194820
:1046300003F000FF21E02179284611F095FB0446A4
:104640000246294608F52C7010F060FF00B30DF10A
:104650000C09002322462946484611F08FFECDE979
:10466000006708F1280099E8060000F0F6FA002338
:1046700005AA2146284611F09FFE284603F060FF58
:104680000DB0BDE8F0832179284611F088FBD6E70C
:104690000148CDE7B4BC0108D2BC010882B0F7B52F
:1046A000044600250F46164600211C22099313F0EC
:1046B0008EFC04F128031846294625774FF4227210
:1046C000276213F084FC29464FF4207213F07FFC1C
:1046D0002946C4F8A85284F8AC52282204F52C705C
:1046E0000E4D13F074FC04F536730DAA07CA83E867
:1046F00007002A781AB96F210948FDF75DFE0023EB
:104700002B700C9B3046009309AB0ECB11F076FD5D
:10471000204603B0BDE8F04002B0704758000020CA
:1047200077BD010882B070B5144C86B00E460AA958
:1047300081E80C0023680546DB0716D403AB0EAAFC
:1047400007CA83E807000BAB93E807000A9B8DE8D4
:104750000700324629460A48FFF7A0FF0123094A0D
:1047600009490748236011F0C0FF0548074B18604E
:1047700006B0BDE8704002B0704700BFF4080020EA
:1047800000090020000000200F450008F808002064
:1047900010B5044C22681AB97C210348FDF70CFEC1
:1047A000206810BDF808002077BD01082DE9F04F02
:1047B00004468BB08A46FFF7EBFF237F069000F19B
:1047C00028081BB985219A48FDF7F6FD94F800B03A
:1047D000D4F80C90BBF1000F08D0638833B1A388E4
:1047E00023B1944803F026FE4FF0000B206A0368C3
:1047F0001B689847BAF1020FCDE9040113D10023D9
:1048000062888D4DCDE902236322DDE9020150EA81
:10481000010315D12946894803F00CFE0020002130
:104820000BB0BDE8F08FBAF1010F06D10023A288CA
:10483000834DCDE902237322E7E72D22814DE9E77D
:10484000D4F8D832504698477F49D1E90023134322
:104850008A4633D1404600F085FA404600F033FAEC
:104860007A4B1870002800F0CB804046079300F088
:1048700008FABBF1000F00F0C780079B1B78002BE4
:1048800040F0C280DDE9020103F06AFDDDE9026764
:10489000B6197F4139468246304603F061FD5246E3
:1048A000034629466A4803F0C5FDDDE90423921951
:1048B0007B411F461646644BC3E90067022099FB03
:1048C000F0F94A46D317CDE90223206A03681B6832
:1048D00098475D4B0646D3E9009A484571EB0A03B9
:1048E0000F4674DAB9EB06006AEB070103F038FDF6
:1048F00029460246574803F09DFDD4F8DC324FF4B8
:104900007A7098478146C0B101460698FFF760FE6D
:10491000D9F8000003F014FE484603F011FEBBF185
:10492000000F0AD0404600F047FA484B1B7823B1ED
:1049300001224948114603F07DFD09AB0093DDE9F2
:104940000223B21A67EB0303404600F0D7F9814611
:104950008A4659EA0A0316D0099BA3B13946304664
:1049600003F0E8FC01463D4803F064FD514648462B
:1049700003F0E0FCA9EB06020146394803F05AFDBA
:10498000099800F019F9BBF1000F9ED02F4B1B784E
:10499000002B9AD159EA0A0319D0DDE90223DDE997
:1049A0000201B9EB02026AEB0303801979419042DC
:1049B00071EB030389DAB9EB06006AEB0701DDE965
:1049C0000234C31A61EB04041846214628E7404626
:1049D00000F0D1F9011E05DD224803F02BFD404611
:1049E00000F04FF9D4F8E032984729461E4803F00A
:1049F00021FD002214491046C1E9002211460FE7AB
:104A0000BBF1000F7FF43EAFDDE9020103F0A8FC2B
:104A100029460246154803F00DFDDDE90467DDE98E
:104A2000022392197B4116461F46CAE9006745E7F3
:104A300077BD0108CCBD0108C3BD010815BE010842
:104A4000C9BD0108E3F70108F00B0020E80B0020C6
:104A50004FBE0108DBBE010807BF01082EBF0108D9
:104A60003DBF010859BF01088BBF01089FBE010867
:104A7000F8B504460D4607460E460FCD0FC495E81F
:104A8000070084E8070007F52C743169204610F010
:104A9000BFFF7169204611F035F8B169204611F069
:104AA000A7F801233B77F8BD37B5034668460024D5
:104AB000002580E806000021C3E90045C3E904455C
:104AC00003F11804197203C884E80500184603B0FE
:104AD00030BD00002DE9D848D0E904BC1F465BEA90
:104AE0000C03044616460DD0D0E90023134309D128
:104AF000B6EB0B0067EB0C01C4E90001014604486A
:104B000003F098FC0123C4E904672372BDE8D88848
:104B1000ADBF010810B504460EF050FD04490EF07B
:104B2000F5FB002801DDC11710BDD4E90001FBE74A
:104B3000B9AC01082DE9F843994604469046FFF7C1
:104B4000E9FF06460F4656EA070323D004F1100595
:104B5000D5E9004554EA050318D0B8EB040069EB29
:104B60000501002871F1000310DB3B46324612F0CC
:104B7000FDFE10F1010808FB07F341F1000906FBF7
:104B80000933A8FB0601194424184D412046294643
:104B9000BDE8F88304460D46F8E708B5D0E90423DC
:104BA000134307D0FFF7B6FF50EA010314BF0120FB
:104BB000002008BD0020FCE773B50446856900F1BC
:104BC0001001D1E9000103F0B5FB06462046FFF7CE
:104BD000A1FF237A3246009329460346024803F098
:104BE00029FC02B070BD00BFC4BF0108F0B58BB096
:104BF0006C460646034684E806009DF8042000F54E
:104C00002075AB42184607D01F7F974202D19F699B
:104C10008F4209D02033F4E7D6F88032132B05D920
:104C20000123002086F884320BB0F0BD94E8060022
:104C300002A8FFF739FFD6F880C202AC06EB4C178A
:104C40003D460FCC0FC594E80F0085E80F000CF12E
:104C50000103C6F880323846E6E737B5DDE9064598
:104C60006B4683E8060093E80600FFF7BFFF30B10C
:104C700022462B4603B0BDE83040FFF72BBF03B000
:104C800030BD2DE9F043074606464FF0000889B0D5
:104C900000F52079B14510D034466D461822002128
:104CA000684613F094F90FCD0FC4CDE9068820367D
:104CB00095E80F0084E80F00ECE7002387F88432C2
:104CC00009B0BDE8F08338B5D0F8803293B104461E
:104CD00000F52075A5420FD0A3690BB92034F9E780
:104CE000D4E90423134305D02046FFF713FF50EA0D
:104CF0000103F3D1012038BD0020FCE72DE9F04786
:104D000098460023089D91462B6090F8843203BB9F
:104D100004460026002700F5207A54451BD0A369DD
:104D2000ABB1237A9BB943464A462046FFF702FFC0
:104D300050EA010313D056EA070303D0B04271EBE7
:104D4000070304DA2B6803B12C6006460F462034B3
:104D5000E3E71646474630463946BDE8F087064643
:104D60000F46F8E7002300F52072824202D003725A
:104D70002030FAE7704700F52072034600209A427F
:104D800006D0996911B1197A01B901302033F6E7DB
:104D9000704770B50446002500F52076B44208D06F
:104DA000A36923B12046FFF7F8FE00B10135203496
:104DB000F4E7284670BD000073B50446144803F0BC
:104DC00039FB144803F036FB2046FFF77CFF06460C
:104DD0002046FFF7D0FFD4F88022151A2046FFF7AF
:104DE000D8FFD4F880322A460093314603460A4859
:104DF00003F020FB04F52075AC4206D0A36913B183
:104E00002046FFF7D9FE2034F6E702B070BD00BFA0
:104E1000F3BF0108D6B3010804C00108002103E074
:104E20000A4B5B584350043109480A4B42189A42D6
:104E3000F6D3094A02E0002342F8043B074B9A42AA
:104E4000F9D300F00DF8FCF7FFF8704744FA0108B9
:104E5000000000207804002078040020485600203C
:104E6000314B82B01A6842F480721A6099682F4AF6
:104E70000A409A601A6822F0885222F001121A60E1
:104E80001A6822F480221A609A6822F47D029A60DD
:104E90000022DA6001921B6813F4007318BF01232B
:104EA0000193019B012B37D14FF48051204B1A689D
:104EB000A3F5806322F00102C3F80024D3F8002494
:104EC00022F00202C3F80024D3F8002422F00402E6
:104ED000C3F800245A6A42F080525A62154A11609F
:104EE0005168C906FCD49A689A609A689A609A6870
:104EF0009A605A6822F460425A605A6842F440420A
:104F00005A609A6822F003029A609A689A60064A88
:104F1000936813F00C0FFBD14FF00062064B9A60C0
:104F2000064ADA6002B07047003802400CC0FF88C1
:104F3000003C02400070004000ED00E00003FA0574
:104F400070B5064688B02E4801F046FB2D4B1A6816
:104F50000092009A91073CD501214FF4007001F0B6
:104F600095FD012001F088FB274A536843F4003384
:104F70005360A2F5374253681B07FCD50024012576
:104F800002A801F063FB02A91D488DF80D400694AC
:104F90008DF81C508DF80C4001F032FB2A46062398
:104FA0003146174801F074FB2946154801F05AFBB9
:104FB0000221134801F0FEFB114801F0EDFB134DF7
:104FC00001940F4C0221204601F0EEFB58B108B0CD
:104FD00070BD1A6842F001021A60009A9207BBD4B1
:104FE0001A680092F9E7019B01330193019BB3F525
:104FF000805FE7DB38212846FDF7DEF9E2E700BFF6
:1050000000240140003802400027014038C0010858
:1050100008B5002001F030FB0021074801F022FB19
:1050200000214FF4007001F031FD044A136823F0B1
:105030000103136008BD00BF002401400038024096
:1050400013B5072301220146114801F021FB02217B
:105050000F4801F0AFFB0E4801F09EFB00230D4C02
:10506000019302210A4801F09FFB28B1084802B0D1
:10507000BDE8104001F095BB019B01330193019BFA
:10508000B3F5805FEDDB4C212046FDF795F9E8E7AD
:105090000024014038C0010870B506460825FFF716
:1050A0004FFF00243046FFF7CBFF013D0444F9D108
:1050B000FFF7AEFFC4F3CF0070BD0000000000009A
:1050C00008B51120FFF7E8FF12F0ECF90146084897
:1050D00012F0F4FA11F0CEFD03A3D3E9002311F08E
:1050E00021FE12F0D9F808BD2FDD24068195F33F8B
:1050F00000F07F450F4A536A43F0805353620E4BD2
:105100001A465968C906FCD41B68022823F4C05308
:1051100006D143F4C05313605368DB06FCD47047D8
:10512000012802D143F48053F5E70028F3D143F47A
:105130000063F0E7003802400070004010B50C4BEF
:105140005A68D206FCD41C6814F4C05F0BD114F466
:1051500080500AD114F4006404D106482A21FDF7D6
:105160002BF9204610BD0220FCE70120FAE700BF22
:105170000070004086C0010838B50546012001F0E6
:1051800029FB022D01BF144A136843F00103136089
:10519000124B1A6842F480721A601A689205FCD5A4
:1051A0005A6822F4604242F440425A6000229A60F7
:1051B0000A4B9C6814F00C04FBD14FF480721A6007
:1051C000074B084A28461A60FFF794FF2046BDE8BF
:1051D000384001F0F3BA00BF003C02400038024002
:1051E0005C000020D0FE3F000C4B5A6B900513D49E
:1051F0005A6A42F080525A62094A116841F4807139
:105200001160596B41F480715963596B8905FCD564
:10521000136823F480731360704700BF00380240A6
:1052200000700040054B5A6B910706D45A6B42F050
:1052300001025A635A6B9207FCD57047003802404E
:10524000094B5A6A42F020025A629A6942F02002DF
:105250009A619A6922F020029A610022A3F509332B
:105260001A801A855A6270470038024015210238A8
:10527000002248430121064B1A85D86299825A625E
:105280001A8219801A8AD207FCD500221A80704728
:1052900000140040002349F6FE7282B00193019B86
:1052A000934201DD02B07047019B01330193F6E7A1
:1052B000002340F6FE7282B00193019B934201DD10
:1052C00002B07047019B01330193F6E7002382B0DF
:1052D0000193019BB3F5CC7F01DD02B07047019BC8
:1052E0000133F5E7D0B1012801D1FFF7EFBF0C4B37
:1052F00000211A684FF47A73B2FBF3F2094B013ABA
:1053000092B21A8501220138D8629A8259621982B2
:105310001A801A8AD207FCD500221A80704700BF73
:105320005C0000200014004000F1774303F578038F
:10533000B3F5804F2DE9F04106460C4617462DD2B5
:1053400002F1F73303F608030344B3F5804F25D287
:10535000FFF7F4FE804610B10020FFF7CBFE01F00E
:1053600051FA01252744361BA7420AD101F05AFA07
:10537000B8F1000F02D04046FFF7BCFE2846BDE85A
:10538000F08141F6027001F055FA301914F8011B52
:1053900001F0ACFA042818BF0025E5E70025EDE789
:1053A00010B50C4600F1774101F57801B1F5804F59
:1053B0000DD202F1F73303F608030344B3F5804F2F
:1053C00005D20146204612F0DEFD012010BD00206E
:1053D000FCE7000008B5114B984215D003F5806337
:1053E000984213D003F58063984211D003F580638F
:1053F00098420FD003F5006398420DD0084B094A3C
:105400001421094812F06CFC002008BD0120FCE7C3
:105410000220FAE70320F8E70520F6E70000024043
:105420001DC10108D7C0010836C101080F2808B501
:1054300005D9094B094A3B21094812F051FC0123C7
:1054400003FA00F0C043074A5168014051601368F5
:105450001840106008BD00BF87C10108E1C0010805
:1054600036C10108000401400F292DE9F84F82469A
:105470000D4693461F4605D95A4B5B4A54215B485B
:1054800012F02EFC4FF0010909FA05F900F0B8F806
:105490006FEA0903564E032D7268564C02EA030266
:1054A0007260326803EA0203534A3360136A43F0BE
:1054B000010313622ED80F22A3684FEA850802FA6F
:1054C00008F223EA0203A3605046FFF783FFA368B4
:1054D00000FA08F01843A0601BF0020F18BFB36871
:1054E000464A1CBF43EA0903B3601BF0040F1EBF0A
:1054F000F36843EA0903F360336843EA090333605E
:105500003B01DBB2002D45D182F806334023136006
:10551000BDE8F88F072D13D80F22A5F10408E36822
:105520004FEA880802FA08F223EA0203E3605046D1
:10553000FFF750FFE36800FA08F01843E060CBE79C
:105540000B2D13D80F22A5F1080823694FEA88080C
:1055500002FA08F223EA020323615046FFF73AFFFA
:10556000236900FA08F018432061B5E70F22A5F17E
:105570000C0863694FEA880802FA08F223EA02037A
:1055800063615046FFF726FF636900FA08F018438D
:105590006061A1E7012D03D182F807338023B6E7CC
:1055A000022D04D182F808334FF48073AFE7032D46
:1055B00004D182F809334FF40073A8E7042D04D115
:1055C00082F80A334FF48063A1E7092D04D882F8EA
:1055D00017334FF400039AE782F828334FF48073AF
:1055E000536095E793C10108FCC0010836C101086A
:1055F00000040140000001400038024000E100E0EA
:10560000144B984205D1144AD36943F00103D36186
:105610007047124B984204D10F4AD36943F00203FA
:10562000F5E70F4B984204D10B4AD36943F00403CA
:10563000EDE70C4B984204D1074AD36943F00803C5
:10564000E5E7094B9842E3D1034AD36943F02003CD
:10565000DDE700BF000002400038024000040240C5
:1056600000080240000C02400014024003234900DD
:1056700010B584688B4024EA030484600124022A64
:1056800004FA01F407D0032A0DD0012A07D1836858
:105690002343836003E083688A401A4382608368FF
:1056A0001C43846010BD82681343F2E70F29F8B5EC
:1056B00004460F4615461E4603D940211948FCF7FB
:1056C0007BFE2046FFF79CFF03237A009340DB43D9
:1056D0002168194021600121D4F800C001FA02F0CC
:1056E0004CEA000CB940C4F800C009B266B1A68803
:1056F000314389B2A180E168012D03EA0103E3602F
:1057000006D0022D08D0F8BDA68826EA0101F1E7EF
:10571000E3680343E360F6E7E36805FA02F21A433D
:10572000E260F0E7E3C101080F2970B505460C46B9
:10573000164603D960210E48FCF73EFE2846FFF7C7
:105740005FFF032361008B40DB43EA68012E02EA1E
:105750000302EA6005D0022E03D02A6813402B60B2
:1057600070BDEA6806FA01F11143E960F5E700BF90
:10577000E3C101080F2910B505D9074B074A762167
:10578000074812F0ADFAFFF73BFF4B000321026818
:1057900099401143016010BD87C101089FC10108F4
:1057A000E3C101080F2938B50446154605D97C2107
:1057B0001B4B1C4A1C4812F093FA0F2A03D91B4BAF
:1057C000184A7D21F6E7FFF71BFF07294FF00F036B
:1057D00018D8006A8A00934020EA03032362236AF0
:1057E00005FA02F21A4322620322236849008A4022
:1057F00023EA020323600223226803FA01F1114322
:10580000216038BDA1F10802406A9200934020EA6D
:1058100003036362636A95401D436562E4E700BF6A
:1058200087C10108B2C10108E3C10108D0C1010864
:10583000012303FA01F189B201837047012303FABE
:1058400001F189B241837047012303FA01F189B262
:105850000AB10183704741837047008A084100F014
:10586000010070470F2938B505460C4603D9A92118
:105870000548FCF7A1FD28686400E04000F0030043
:10588000431E5842584138BDE3C10108808A08418F
:10589000C04300F00100704710B5084C23681BB9E5
:1058A000012005F039FA206023682BB9BDE81040CB
:1058B00036210348FCF780BD10BD00BFF80B002067
:1058C00032C2010810B50B4C22681AB93C210A48B3
:1058D000FCF772FD206842F2107105F065FB0128AB
:1058E0000CBF0124002403D040210348FCF764FDD1
:1058F000204610BDF80B002032C2010810B5074C3D
:1059000022681AB951210648FCF756FD0023206889
:105910001A46BDE81040194605F05AB9F80B0020A8
:1059200032C2010810B50446FFF7B6FFFFF7CAFF01
:1059300021461022034801F04BFD0446FFF7DEFF2D
:10594000204610BD0054004010B5FFF7A5FFFFF73B
:10595000B9FF01F0F5FC0446FFF7D0FF204610BD6B
:1059600008B513460A460146034801F067F90030BE
:1059700018BF012008BD00BF0054004008B5134601
:105980000A460146034801F05FFA003018BF0120C3
:1059900008BD00BF0054004008B513460A46014642
:1059A000034801F0E3FA003018BF012008BD00BF32
:1059B0000054004008B513460A460146034801F06A
:1059C00065FB003018BF012008BD00BF0054004037
:1059D00008B513460A460146034801F0AFFB003004
:1059E00018BF012008BD00BF005400400123064A33
:1059F00083405169194205D05361044B53F820305C
:105A000003B11847704700BF00040140FC0B0020A1
:105A10000F2838B504460D4603D926210348FCF764
:105A2000CBFC034B43F8245038BD00BF80C20108B3
:105A3000FC0B00200020FFF7D9BF0120FFF7D6BFE5
:105A40000220FFF7D3BF0320FFF7D0BF0420FFF7EA
:105A5000CDBF08B50920FFF7C9FF0820FFF7C6FF33
:105A60000720FFF7C3FF0620FFF7C0FFBDE808408F
:105A70000520FFF7BBBF08B50F20FFF7B7FF0E20CB
:105A8000FFF7B4FF0D20FFF7B1FF0C20FFF7AEFFCB
:105A90000B20FFF7ABFFBDE808400A20FFF7A6BFC9
:105AA000FEE7FEE7FEE7FEE7FEE7FEE7FEE7FEE7CE
:105AB000FEE7FEE7FEE7FEE7FEE7FEE7FEE7FEE7BE
:105AC000FEE7FEE7FEE7FEE7FEE7FEE7FEE7FEE7AE
:105AD000FEE7FEE7FEE7FEE7FEE7FEE7FEE7FEE79E
:105AE000FEE7FEE7FEE7FEE7FEE7FEE7FEE7FEE78E
:105AF0000A23B0FBF3F203FB120040EA0210C0B22B
:105B000070470000CA22024B5A6253225A62704701
:105B100000280040014B1860704700BF3C0C00207B
:105B20004FF400320F4B10B50F4C5A61E368DB05A0
:105B300003D430210D48FCF73FFCFFF7E3FF4FF49F
:105B40000072A36823F48853A360094BC3F8842030
:105B5000FF236362074B1B6813B1BDE81040184771
:105B600010BD00BF0004014000280040CEC2010863
:105B700000E100E03C0C00202DE9F04F9846374B47
:105B800085B01B78824691469DF838709DF83C6040
:105B90002BB9334B334A8C21334812F0A1F8431E02
:105BA0001E2B59D80C2957D8A2F5FA63632B53D86A
:105BB000B8F1170F50D83B2F4ED83B2E4CD802F1DE
:105BC0003000C0B2FFF794FF83460846FFF790FF0E
:105BD00004465046FFF78CFF40F400554046FFF75F
:105BE00087FF45EA0B4545EA042504463846FFF79A
:105BF0007FFF000240EA04443046FFF779FF20436C
:105C00001A4CFFF77FFFE36843F08003E360E3682B
:105C10005B06FCD565602060E36823F08003E360E9
:105C2000124BDA689206FCD5FF2204A85A6200F8EB
:105C30000C6D8DF807A08DF80810ADF809908DF85F
:105C400006808DF8057002F032FB094BC3E90001B4
:105C5000012005B0BDE8F08F0020FAE7400C0020DD
:105C60004FC301081CC30108CEC201080028004030
:105C7000480C002037B50578C4788378B0F8052043
:105C800001790195407800902046FFF775FF03B039
:105C900030BD000038B52B4B04461B781BB9E421FE
:105CA0002948FCF789FB294AD36823F02003D360F5
:105CB000D3689B06FCD513685268C2F307410809F4
:105CC00000EB800001F00F0101EB4001C9B201F5CA
:105CD000FA61A4F80510C2F30721C1F30010850092
:105CE000284401F00F0101EB4001D2B22171C2F34F
:105CF000011101EB810102F00F0202EB4102E2709F
:105D0000C3F30742C2F3011101EB810102F00F025C
:105D100002EB4102A270C3F30722C2F3021101EBAE
:105D2000810102F00F0202EB4102DBB26270C3F3A9
:105D3000021202EB820203F00F0303EB4203237013
:105D400038BD00BF400C0020CEC201080028004032
:105D50001FB501A8FFF79EFF01A802F0A8FA05B041
:105D60005DF804FB08B5FFF73FFA1B4A136843F4DC
:105D700080731360FFF7C6FE184A536B23F4403359
:105D800043F482035363164BDA6842F08002DA6010
:105D9000DA685106FCD5FF221A611A6942F4FE0244
:105DA0001A619A6822F040029A609A6822F44C5272
:105DB0009A60DA6822F08002DA60094BDA689206AB
:105DC000FCD5FF225A620122064B1A70FFF7C0FF72
:105DD000054BC3E9000108BD0070004000380240D7
:105DE00000280040400C0020480C002008B5094B5A
:105DF0001B7823B940F21F110748FCF7DDFAFFF7C3
:105E000081FE064B9A6822F480729A60FF225A62E1
:105E100008BD00BF400C0020CEC201080028004091
:105E200008B5144B1B7833B9134B144A40F22711B1
:105E3000134811F055FFFFF765FE124BDA6822F4A4
:105E40008072DA60104A916841F400319160116803
:105E500041F400311160F0210C4A82F829134FF40B
:105E6000007151609A6842F488529A60FF225A6227
:105E700008BD00BF400C00204FC3010828C3010823
:105E8000CEC20108002800400004014000E100E00B
:105E9000F8B51E46194B17461B7833B9184B194AEB
:105EA0004FF4A571184811F01BFF184CFFF72AFE9C
:105EB000A56825F48075A560E56825F48075E56022
:105EC000FFF716FE05460846FFF712FE000440EAFB
:105ED00005613846FFF70CFE05463046FFF708FE21
:105EE000084340EA0520E368DB07FCD5FF23E061B7
:105EF0006362BDE8F840FFF793BF00BF400C00208D
:105F00004FC301083DC30108CEC20108002800406C
:105F1000037842788178C078FFF7BABF38B50D466C
:105F2000044604F057FB194A136823F00103136079
:105F300004F070FB25B1164A536843F00603536022
:105F400072B6BFF34F8FBFF36F8F124A01201368F1
:105F500023F0030343F4007343F00103136000F0E4
:105F600045FC0D4B1A6942F004021A6130BF1A69F0
:105F7000022022F004021A61FFF7FEF8034A1368B8
:105F800043F00103136004B162B638BD10E000E0D5
:105F9000002004E00070004000ED00E062B67047B1
:105FA00000220E4B10B51A700D4A0E4C1388204675
:105FB00023F040031B041B0C13800D210222FFF76A
:105FC000B3FB204602220E21FFF7AEFB2046BDE8C0
:105FD000104002220F21FFF7A7BB00BF500C00208A
:105FE000003800400004024038B50546274A2848DA
:105FF000536A0C4643F4804353620D210522FFF798
:10600000D1FB05220E212248FFF7CCFB05220F21F0
:106010001F48FFF7C7FBC5B101220D211C48FFF740
:1060200025FB01220E211A48FFF720FB01220F2138
:106030001748FFF71BFB012C21D144F451740122B6
:10604000144B1C80144B1A7038BD2A460D21104881
:10605000FFF70CFB2A460E210D48FFF707FB2A46E7
:106060000F210B48FFF702FB012C05D0022C03D0B7
:10607000032C14BF0024032444F45974DFE7022CDA
:10608000DBD0032C0CBF03240024D6E700380240E9
:106090000004024000380040500C0020064B074A24
:1060A000988111781A461889C00701D40029FAD1BD
:1060B0009089C0B2704700BF00380040500C0020EB
:1060C000284A38B5136A054643F480531362052203
:1060D00025480C461146FFF765FB0522062122489C
:1060E000FFF760FB052207211F48FFF75BFBC5B1E7
:1060F000022205211C48FFF7B9FA022206211A489C
:10610000FFF7B4FA022207211748FFF7AFFA012C74
:1061100021D144F451740122144B1C80144B1A7089
:1061200038BD2A4605211048FFF7A0FA2A46062165
:106130000D48FFF79BFA2A4607210B48FFF796FA0E
:10614000012C05D0022C03D0032C14BF00240324FF
:1061500044F45974DFE7022CDBD0032C0CBF03247A
:106160000024D6E700380240000002400030014021
:10617000510C002000220E4B10B51A700D4A0E4C27
:106180001388204623F040031B041B0C13800521B9
:106190000222FFF7C9FA204602220621FFF7C4FABD
:1061A0002046BDE8104002220721FFF7BDBA00BF1C
:1061B000510C00200030014000000240064B074A0D
:1061C000988111781A461889C00701D40029FAD19C
:1061D0009089C0B2704700BF00300140510C0020D0
:1061E000054AD36823F4E0631B041B0C43F0BF6330
:1061F00043F40033D360704700ED00E0202200211B
:10620000114B10B5C3F88420104B114C1A6A20466C
:1062100042F480421A625A6942F480425A615A69D1
:1062200022F480425A610B4A91811A6A092122F4B0
:1062300080421A620222FFF777FA2046BDE810403A
:1062400002220A21FFF770BA00E100E000380240A4
:10625000000002400038014010B50B4C40F22551BF
:10626000204600F0C4FC48B1204600F09EFC074BDD
:10627000C0B21B6833B1BDE810401847A388044A78
:10628000DBB2137010BD00BF00380140540C002079
:106290007055002010B504468021084800F0A1FC8C
:1062A0000028F9D02146054800F07BFC034C402132
:1062B000204600F096FC0028F9D010BD00380140BF
:1062C00010B5441E14F8010F00B910BDFFF7E2FF2E
:1062D000F8E7000008B5024800F067FCC0B208BD4E
:1062E000003801402DE9F0438846012189B08146FC
:1062F000084614461D4600F0BDFB01214FF48040C6
:1063000000F0C4FB4FF4C06702230122002602A95B
:106310003F488DF80C308DF80D308DF80F20029726
:106320008DF80E6000F008FB07220921384800F0C4
:1063300045FB07220A21364800F040FBB8F1450F23
:10634000CDF810903CD14FF48063ADF81830072C95
:1063500042D10023ADF81430052D4ED14FF48053B7
:10636000ADF816300023ADF81C300C2304A92948E1
:10637000ADF81A3000F0BAFB274B1A6802B10122BF
:1063800040F22551234800F014FC0121214800F07F
:10639000FDFBFFF79FFF25238DF804309DF840306B
:1063A0008DF8053000238DF8063001238DF8073075
:1063B000FFF716FF01A800F0F3F809B0BDE8F0837D
:1063C000B8F14F0F02D1ADF81870C0E7072CADF847
:1063D00018600DD1592107E0082C02D14FF48053E9
:1063E000B8E7092CB8D154210C48FBF7E5FFB3E717
:1063F000082CAED0092CAFD1F0E70F2D02D14FF40D
:106400004053ADE7022D0CBF4FF400530023A7E724
:106410000000024000380140540C002058C301081D
:106420000E2307B5082200934E210123FFF75AFFE0
:1064300003B05DF804FB000070B5134C40F2255129
:10644000204600F0D4FBC0B1104B1D6825B120469A
:1064500000F0ABFBC0B2A84740F226610A4800F04A
:10646000C6FB78B140F22661074800F0DFFB084B1D
:106470001B683BB1BDE870401847A388054ADBB2F2
:106480001370E9E770BD00BF00440040580C0020C5
:106490005C0C002070550020BFF34F8F0449054B62
:1064A000CA6802F4E0621343CB60BFF34F8FFEE78C
:1064B00000ED00E00400FA0510B5441EE3B2052B20
:1064C00003D90E211148FBF777FFFEF7ABFE45F22B
:1064D00055520F4B1A60DA68D207FCD4052C06D847
:1064E000DFE804F003090B0D0F1101225A604CF68E
:1064F000CC421A6010BD0222F8E70322F6E704221C
:10650000F4E70522F2E70622F0E700BF31C40108F4
:106510000030004010B5194C23683BB95F2000F0F3
:10652000CDFA28B1164B236000F0D8FA206810BDD0
:106530005E2000F0C3FA08B1124BF4E75D2000F0D2
:10654000BDFA08B1104BEEE75C2000F0B7FA08B1D5
:106550000E4BE8E75B2000F0B1FA08B10C4BE2E724
:106560005A2000F0ABFA08B10A4BDCE7592000F0E2
:10657000A5FA08B1084BD6E7084BD4E7600C002019
:10658000A7C30108B7C30108CDC30108E8C30108C8
:10659000F7C3010806C401081FC4010829C4010883
:1065A00030B5012403780A4D03F01F029440C278ED
:1065B000590952B1074A2B44D26842781201D2B22B
:1065C00083F8002345F8214030BD2031FAE700BFB1
:1065D00000E100E000ED00E008B5084B98420BD167
:1065E00001214FF4007000F05DFABDE80840002181
:1065F0004FF4007000F056BA08BD00BF00240140FF
:1066000043680A7923F0407323F4807343EA02233A
:106610000A6810B513434360D1E9032313438A6822
:1066200084681343084A224013434A7943EA4203E9
:1066300083600A7D036B013A23F0F873D2B243EA18
:106640000253036310BD00BFFDF7FFC000234FF0EE
:1066500040720360037143718360C0E90323012327
:1066600003757047836819B143F001038360704775
:1066700023F00103FAE70000044B5A6818B142F412
:1066800000025A60704722F40002FAE70027014036
:106690001D2970B51BD90725A1F11E06C46D06EB97
:1066A0004606B54024EA050403FA06F62643C66505
:1066B000062A38D81F24013A036C02EB8202944068
:1066C00023EA040301FA02F21A43026470BD13299B
:1066D0000DD90726A1F11405C46805EB4505AE40A8
:1066E00024EA060403FA05F52543C560E0E7092915
:1066F0000DD90726A1F10A04056904EB4404A6405C
:1067000025EA060503FA04F42C430461D0E70726C2
:10671000446901EB4105AE4024EA060403FA05F69C
:1067200026434661C4E70C2A0CD81F24073AC36BE2
:1067300002EB8202944023EA040301FA02F21A43B4
:10674000C263C3E7122A0CD81F240D3A836B02EBF5
:106750008202944023EA040301FA02F21A4382639C
:10676000B4E7182A0CD81F24133A436B02EB8202B9
:10677000944023EA040301FA02F21A434263A5E7B4
:106780001F24193A036B02EB8202944023EA0403AC
:1067900091401943016399E7836843F08043836024
:1067A0007047806D80B270470368194214BF0120A2
:1067B00000207047C943016070470000044B1A680D
:1067C00018B142F002021A60704722F00202FAE7A2
:1067D000003C0240044B1A6818B142F004021A60EF
:1067E000704722F00402FAE7003C0240044B1A68AA
:1067F00018B142F008021A60704722F00802FAE766
:10680000003C0240044B5A68D20741BF034ADA6099
:10681000034ADA60704700BF003C0240EFCDAB890D
:1068200005040302024A536843F0010353607047B2
:10683000003C0240014B9861704700BF003C0240A1
:10684000084B9A69D10709D49A69D20508D49B6983
:1068500013F4F05F14BF0320042070470120704739
:1068600002207047003C0240042313B504468DF813
:106870000730FFF7E5FF8DF807009DF80730012B83
:106880000AD11CB905238DF8073007E0FFF7D8FFC0
:10689000013C8DF80700F0E7002CF3D09DF80700CD
:1068A00002B010BD10B504464FF40040FFF7DCFF06
:1068B000042804BF0023236010BD000038B504463F
:1068C0004FF400400D46FFF7CFFF04280BD1064AD6
:1068D0004FF40040536823F4807353602560BDE893
:1068E0003840FFF7C1BF38BD003C024038B5044610
:1068F0004FF400400D46FFF7B7FF04281BD135B118
:1069000025704FF40040BDE83840FFF7ADBFFF23CE
:1069100024F0030504F003042968E40003FA04F4F6
:1069200021EA04042846FFF7BDFF21462846BDE8BA
:106930003840FFF7C3BF38BD2DE9F04300220127DF
:1069400003250E6807FA02F333EA060431D14FEA51
:10695000420C05FA0CF4E44391F804E0D0F80090FE
:106960000EFA0CF804EA09090EF1FF3E48EA09089C
:10697000BEF1010FC0F8008011D8D0F808E004EA99
:106980000E0E4C7904FA0CF444EA0E0484608488F8
:1069900024EA03048B7993409BB223438380C3682A
:1069A00005FA0CF423EA0404CB7903FA0CF323432D
:1069B000C3600132102AC5D1BDE8F08310B50F24A1
:1069C00001F00703C90800EB8100016A9B009C40AD
:1069D00021EA04010162016A9A400A43026210BD81
:1069E000204B10B59A6802F00C020C2A30D8DFE870
:1069F00002F02F2F2F2F072F2F2F072F2F2F2000A1
:106A0000194B184A036093681849C3F30313CC5C0D
:106A10000368E34043609468C4F302240C5D23FAE6
:106A200004F484609268C2F3C2228A5CD340C360DB
:106A300010BD99680E4CC1F383419A68615C9B68F4
:106A4000094BC2F381524B430132B3FBF2F3D8E757
:106A50004FF400425B68C3F34233013302FA03F39D
:106A6000CFE700BF003802400024F400600000209F
:106A700070000020044BDA6911B11043D8617047EF
:106A800022EA0000FAE700BF00380240044B1A6A0D
:106A900011B110431862704722EA0000FAE700BF04
:106AA00000380240044B5A6911B1104358617047D5
:106AB00022EA0000FAE700BF003802404309012B38
:106AC000054B00F01F000CBF1B685B6B23FA00F046
:106AD00000F00100704700BF00380240024A536BCB
:106AE00043F08073536370470038024030B50D4661
:106AF0000446028AEB8892B222F440521A438989F2
:106B000002828389288923F4B052AB8822F00C02D8
:106B10000343688985B003431343A381A38A68466E
:106B20009BB223F440730B43A382FFF759FFDDE9C7
:106B30000231154A944218BF19461923A2894B43C2
:106B4000296810044CBF49008900B3FBF1F16425AA
:106B5000B1FBF5F3A2891801120405FB13130BD541
:106B6000DA003232B2FBF5F202F0070242EA000329
:106B70009BB2238105B030BD1B013233B3FBF5F36B
:106B800003F00F030343F3E700380140838919B191
:106B900043F400538381704723F400531B041B0C00
:106BA000F8E7C1F30801818070478088C0F30800CE
:106BB000704701F01F0310B5C1F342140121012CED
:106BC00001FA03F105D10C3003683AB119430160B1
:106BD00010BD022C0CBF10301430F5E723EA010180
:106BE000F5E70388194214BF0120002070470123F4
:106BF000C1F3421210B5012A01F01F0403FA04F395
:106C00000DD182891340028892B26BB10123090A27
:106C100003FA01F10A4214BF1846002010BD022AEF
:106C20000CBF028A828AEDE71846F7E70B0A0121BA
:106C30009940C94389B20180704700002DE9F341B2
:106C40001F46002304460D46019316461AB901203B
:106C500002B0BDE8F08140F6FF7301934FF40031BC
:106C6000204600F00EFD002852D10121204600F000
:106C7000D8FC4FF2FF71204600F0ECFC01212046C9
:106C800000F0B9FC40F6FF73DFF8B881019341468C
:106C9000204600F0EBFC002841D039460122204676
:106CA00000F0CAFC40F6FF73614F0193394620465D
:106CB00000F0E7FC002838D0012E42D10021204608
:106CC00000F0AFFC03F086FC31462046238B00F039
:106CD0009DFC03F09FFC40F6FF73564E0193314636
:106CE000204600F0CEFC30B3204600F0B0FC287007
:106CF00040F6FF73504D01932946204600F0C1FC39
:106D00000028A4D0019B5A1E0192002BF4D104E06C
:106D1000019B5A1E0192002BA0D1002098E7019BF5
:106D20005A1E0192002BB2D1F7E7019B5A1E019225
:106D3000002BBBD1F1E7019B5A1E0192002BCED153
:106D4000EBE7022E25D103F045FC4FF4006120460D
:106D500000F080FC0021204600F063FC238B03F050
:106D600059FC40F6FF73354E01933146204600F042
:106D700088FC40B10121204600F048FC238A2B709A
:106D8000238A6B70B4E7019B5A1E0192002BECD151
:106D9000C3E740F6FF77033E238BDFF8A0802E4445
:106DA000B54201972CD1254E3146204600F069FCB2
:106DB00090B30021204600F034FC03F00BFC204689
:106DC00000F045FC01212870204600F01FFC03F074
:106DD00021FC204600F03BFC40F6FF73184E687023
:106DE00001933146204600F041FCD8B1204600F026
:106DF0002EFCA8707CE7019B5A1E0192002B8CD0C0
:106E00004146204600F03DFC0028F4D0204600F02A
:106E10001EFC05F8010BC3E7019B5A1E0192002BD3
:106E2000C2D17AE7019B5A1E0192002BD9D174E797
:106E300002000010400000101000001004000010BC
:106E400040000300010003002DE9F3411E4600232A
:106E500004460D46019317461AB9012002B0BDE859
:106E6000F08140F6FF7301934FF40031204600F0AB
:106E700008FC002846D10121204600F0BCFB40F66A
:106E8000FF73DFF8E48001934146204600F0EEFBFB
:106E900000283ED031460022204600F0CDFB40F6CF
:106EA000FF732D4E01933146204600F0DFFB002892
:106EB00035D0297820466E1C00F0C7FB3D4440F6D3
:106EC000FF77DFF89880AE42019733D1234D2946F2
:106ED000204600F0D6FB002838D02046012100F0E3
:106EE00095FB40F6FF731E4D1E4C0193294620462C
:106EF00000F0C7FB0028B0D0019B5A1E0192002B66
:106F0000F4D104E0019B5A1E0192002BACD1002069
:106F1000A4E7019B5A1E0192002BB5D1F7E7019B14
:106F20005A1E0192002BBED1F1E7019B5A1E01921D
:106F3000002BECD04146204600F0A3FB0028F4D003
:106F400016F8011B204600F080FBBCE7019B5A1E8F
:106F50000192002BBBD1DAE7820007000400001089
:106F60001000001000540040010003002DE9F3411F
:106F70001E46002304460D46019317461AB9012008
:106F800002B0BDE8F08140F6FF7301934FF4003189
:106F9000204600F076FB002837D10121204600F082
:106FA0002AFB40F6FF73DFF8E0800193414620465C
:106FB00000F05CFB002842D031460022204600F061
:106FC0003BFB40F6FF732C4E01933146204600F008
:106FD0004DFB002839D0297820466E1C00F035FB87
:106FE0003D4440F6FF77DFF89480AE42019737D1F9
:106FF000224D2946204600F044FB0028BFD1019BCA
:107000005A1E0192002BF4D104E0019B5A1E0192FA
:10701000002BBBD12046012100F0F8FA40F6FF73A7
:10702000174D184C01932946204600F02AFB20B149
:10703000019B5A1E0192002BF5D10020A0E7019B75
:107040005A1E0192002BB1D1E4E7019B5A1E019216
:10705000002BBAD1DEE7019B5A1E0192002BD9D03A
:107060004146204600F00DFB0028F4D016F8011B25
:10707000204600F0EAFAB8E782000700040000109A
:1070800010000010005400400100030000232DE90F
:10709000F3410D464FF4003104461746019300F0CA
:1070A000F0FA18B9002002B0BDE8F0810FB9012054
:1070B000F9E7297820466E1C00F0C7FA3D4440F6F7
:1070C000FF77DFF86C80AE4201971FD1184D29463B
:1070D000204600F0D6FA28B32046012100F096FAA7
:1070E00040F6FF73134D144C01932946204600F0DF
:1070F000C8FA0028DBD0019B5A1E0192002BF4D164
:10710000D0E7019B5A1E0192002BCBD0414620466E
:1071100000F0B7FA0028F4D016F8011B204600F062
:1071200094FAD0E7019B5A1E0192002BCFD1B9E708
:107130000400001010000010005400402DE9F3413D
:107140001F46002304460D46019316461AB9012036
:1071500002B0BDE8F0814FF4003100F092FA08B9B6
:107160000020F5E70121204600F05BFA4FF2FF71A5
:10717000204600F06FFA0121204600F03CFA40F66C
:10718000FF73DFF8B88101934146204600F06EFAA4
:1071900000283AD039460122204600F04DFA40F648
:1071A000FF73614F01933946204600F06AFA0028C8
:1071B00031D0012E3BD10021204600F032FA03F0FD
:1071C00009FA31462046238B00F020FA03F022FA18
:1071D00040F6FF73554E01933146204600F051FAB8
:1071E000F8B1204600F033FA287040F6FF73504D96
:1071F00001932946204600F044FA0028A7D0019BBD
:107200005A1E0192002BF4D1AAE7019B5A1E01924B
:10721000002BB9D1A4E7019B5A1E0192002BC2D1C9
:107220009EE7019B5A1E0192002BD5D198E7022EB2
:1072300029D14FF40061204600F00CFA03F0CAF99E
:1072400000212046238B00F0ECF903F0E3F940F62F
:10725000FF73384E01933146204600F012FA60B1B8
:1072600003F0B8F90121204600F0D0F9238A2B70F1
:10727000238A6B7003F0CEF9B7E7019B5A1E019287
:10728000002BE8D16CE740F6FF77033E238BDFF855
:10729000A4802E44B54201972DD1264E314620467A
:1072A00000F0EFF998B30021204600F0BAF903F09E
:1072B00091F9204600F0CBF901212870204600F01A
:1072C000A5F903F0A7F9204600F0C1F940F6FF73D5
:1072D000194E687001933146204600F0C7F9E0B1BD
:1072E000204600F0B4F9A8707FE7019B5A1E019276
:1072F000002B3FF435AF4146204600F0C2F900288C
:10730000F3D0204600F0A3F905F8010BC2E7019B7A
:107310005A1E0192002BC1D122E7019B5A1E0192F5
:10732000002BD8D11CE700BF020000104000001065
:1073300010000010040000104000030001000300D2
:1073400038B5204B08219A691F4842F400129A610F
:107350009A6922F400129A615A6A22F400125A625F
:10736000FEF766FA012308211A461748FEF79EF930
:10737000092115480122FEF7D7F909211248FEF725
:107380006CFAD8B1012038BD08212846FEF750FA22
:10739000FDF79CFF08212846FEF750FAFDF796FFFF
:1073A000013CF1D109210848FEF757FA20B94FF402
:1073B000B6710648FBF700F82046E4E73324024D97
:1073C000EEE700BF003802400004024084C4010818
:1073D0002DE9FF41444B054698420E4617467CD1A5
:1073E00003F5F2335A6A082142F400125A629A698C
:1073F0003E4842F400129A619A6922F400129A619E
:10740000FEF716FA012308211A463848FEF74EF90E
:10741000092136480122FEF787F909213348FEF792
:107420001CFA002855D0012308211A462F48FEF7E0
:107430003DF9042208212D48FEF7B4F90123092162
:107440001A462A48FEF732F9042209212748FEF796
:10745000A9F9274B9A6942F400129A619A6922F4B9
:1074600000129A61684600F0ADF8224B694601931C
:107470004FF48063ADF80A304FF480432846ADF8EE
:107480000C30ADF80870009600F038F8284601215D
:1074900000F0A6F8012019E008214046FEF7C8F9DF
:1074A000FDF714FF08214046FEF7C8F9FDF70EFF6F
:1074B000013CF1D109210D48FEF7CFF90028B2D1E6
:1074C0000D484FF4CA71FAF777FF204604B0BDE8C3
:1074D000F0813324DFF81480EAE740F2A311064874
:1074E000FAF76AFFBEE700BF005400400004024004
:1074F000003802400000FFBF84C401087FB5044685
:10750000868868460D46FFF76BFA029A2B4926F0EB
:107510003F06B2FBF1F13604360C88B20643A68072
:107520002388274E23F001031B041B0C23802B68A8
:10753000B3421ED85B00B2FBF3F39BB2042B38BFFF
:107540000423013080B22084A3832388AA8843F0D7
:10755000010323802388698923F481630A4323F08C
:107560000203134323802A89AB891343238104B088
:1075700070BD4BF6FF70EE8886421BBF1920434357
:1075800003EB4303B2FBF3F30BBFB2FBF3F39BB28A
:107590009BB243F48043C3F30B020AB943F00103E7
:1075A0004FF496724A434FF47A7192FBF1F2013232
:1075B00092B243F400432284C6E700BF40420F006A
:1075C000A086010041F28832044BC0E90023002369
:1075D00083604FF480438381704700BF0000FFBF8A
:1075E000038819B143F001030380704723F00103BE
:1075F0001B041B0CF8E7038819B143F48073038064
:10760000704723F480731B041B0CF8E7038819B13F
:1076100043F400730380704723F400731B041B0CB6
:10762000F8E7038819B143F480630380704723F4BB
:1076300080631B041B0CF8E722B141F0010189B201
:107640000182704701F0FE01F9E701827047008A6C
:10765000C0B270470388B1F5006F1BBF23F400630D
:107660001B0443F400631B0C03807047838A008B68
:1076700043EA004321F07F401840431A58425841E2
:107680007047002382B0009301930B0F0190009389
:10769000009B21F07F4153B1019B14330193019B67
:1076A0001B680B4214BF0120002002B07047019BF1
:1076B000090C1833F2E7F8B50E46054680B14F1CA9
:1076C000384600F053FF044640B13A46002110F01E
:1076D0007EFC32462946204610F055FC2046F8BD77
:1076E0000446FBE738B50D46044628B111F044FBCB
:1076F00023462044834201D1002038BD13F8012BDA
:10770000AA42F7D10120F8E737B504460D4610F03C
:1077100013FB002201A90260204611F05BFC044625
:1077200010F00AFB0368222B08D0019B1B782BB9B1
:10773000002C03DB20462B6003B030BD012300206A
:107740002B60F9E72DE9F04F05464FF0010B0026BD
:1077500087B0CDE9031206F10903122B8CBF032079
:10776000022000F003FF0090E8B13246364911F0E4
:10777000D1FA039B53F82690EDB90024009800F04D
:10778000DFFEBBF1000F02D1284600F0D9FE84B124
:10779000049B0136B34225464FF0000BDBD1204657
:1077A00007B0BDE8F08FBBF1000F02D1284600F012
:1077B000C7FE0024F3E7254B4FF00008B9F1000F96
:1077C00008BF9946484611F0D7FA0190009811F089
:1077D000D3FA02902846494611F0FDFAB8B9284676
:1077E00011F0CAFADDE9012301309B1A08FB0300FE
:1077F00000F0BCFE04460028BFD003462F4618F117
:10780000FF3809D23946184611F0AEFAB6E7019BA7
:1078100008F101081844DEE749463846059311F09F
:10782000DAFA059BA0EB070A52463946184611F0D2
:10783000BDFA0099504411F097FA019A029B9244C4
:10784000C3185744DBE700BF7BE101080BE40108E4
:1078500030B580B10346021F00F1180452F8045FEE
:107860008D4208D0A242F9D11C301A461468043364
:10787000013401D1116030BD8342F6D1FBE770B510
:10788000044680B1064600EB8105AE4204D1204695
:10789000BDE8704000F054BE56F8040B0028F4D048
:1078A00000F04EFEF1E770BD2DE9F74F89460092DA
:1078B000002838D00027C45D8CBB05468346264689
:1078C00000EB070AD34538D104B10136002E6FD042
:1078D0000137384600F04AFE8346002866D03A4613
:1078E000002110F074FBB00000F040FE04460028B8
:1078F00060D04FF000084146AA4532D131B1584618
:10790000FFF7D9FE002855D044F82800584600F06B
:1079100017FE009B1E60204603B0BDE8F08F0137C4
:10792000B7F5807FC7D10024264620460024314683
:10793000FFF7A5FF009B1C60EDE79BF800304B456F
:1079400005D10CB1002401360BF1010BBAE710F0A0
:10795000CDFA9BF80030184443781B0758BF013418
:10796000F2E72B784B4513D181B15846FFF7A3FEC0
:1079700000B308F1010344F8280000213A465846B4
:10798000019310F024FB019B002198460135B3E7D9
:10799000019110F0ABFA2B7801991844407810F05F
:1079A000080F04BF0BF801300131EFE70446BCE7D4
:1079B0003446B0E7584600F0C3FDB6E72DE9F7437B
:1079C000002506460820884691461F46009500F08F
:1079D000CDFD0446002868D0C0E90055304611F0BE
:1079E000CBF901280FD133782A2B0CD109F1FF33C1
:1079F000C4F80080636022684A4502D263684B4540
:107A000043D32B4B0EE02D213046FFF76BFE05468E
:107A1000C0B902A941F8040D3046FFF775FE019B7D
:107A200063B1244B3B6000992846FFF728FF002CE8
:107A300037D0204600F084FD002432E0C4E9000085
:107A40001D46D8E76A462D213046FFF72DFF009BE3
:107A50000546013B012B01D9174BE3E7002302AE9A
:107A600046F8043D31460068FFF74EFE2060019B5A
:107A70000BB1124BD6E731466868FFF745FE6060F0
:107A8000019B002BB7D00E4BCCE7424501D34345B9
:107A900001D20C4BC6E700992846FFF7F0FE002301
:107AA0003B60204603B0BDE8F0830546BBE700BF5E
:107AB000AFC5010829C5010848C5010871C50108FD
:107AC00090C50108CFC5010838B590B1451E15F81D
:107AD000014F0CB9204638BD10F008FA2346204467
:107AE000427802F00302022A08BFA4F120032B709F
:107AF000EDE70120EFE708B520B34A1C22D00629A4
:107B000020D8DFE801F0040D101316191C00002323
:107B1000036010F03FFB0840431C5842584108BD29
:107B200000234360F5E700238360F2E700238361CD
:107B3000EFE70123C360ECE700230361E9E70023DB
:107B40004361E6E70120EAE770B506460D1F01F143
:107B5000180455F8041F4B1C03D1A542F9D100208D
:107B600070BD3046FFF7C7FF0028F6D0F8E70823BE
:107B70004A4291FBF3F302F0070201F0070158BFFC
:107B800051420122DBB2C9B202FA01F1C25C1143D7
:107B9000C154704708234A4291FBF3F302F00702F5
:107BA00001F0070158BF51420122DBB2C9B28A403D
:107BB000C15C21EA0201C1547047082391FBF3F331
:107BC000DBB2C05C4B4203F0070301F0070158BF72
:107BD0005942C9B2084100F0010070472DE9F04751
:107BE000089E8A4690461D46DDF82890074610B14B
:107BF0001446A24507D875B9012200240B9B1A60D0
:107C00002046BDE8F08721463846FFF7D6FF00281A
:107C100061D10134EDE7099B023B042B04D8DFE876
:107C200003F0282C2C3034006B6801336B6028463D
:107C300010F0B0FA013108BFB0F1FF3FDCD031469F
:107C40002846FFF758FF0028D6D12FB30446214617
:107C50003846FFF7B2FF002841D10134A245F6D1E2
:107C60000446013E042E19D8DFE806F02B2D2F31F3
:107C70003300AB680133AB60D9E7EB680133EB60ED
:107C8000D5E72B6901332B61D1E76B6901336B6158
:107C9000CDE7002DE5D1AFE73C46E2E72C60284672
:107CA00010F078FA013108BFB0F1FF3FA4D0B9F16C
:107CB000000FA1D049462846FFF746FF00289FD075
:107CC0009AE76C60EBE7AC60E9E7AC61E7E7EC6092
:107CD000E5E72C61E3E7A045DBD1444690E7A0450A
:107CE000BFD1FAE700232DE9F04F06468BB01C20E8
:107CF0000C469046099300F039FC0546002800F038
:107D0000E4801C2000F032FC0746002800F0DD80F3
:107D10004FF0FF31021F2B1F05F1180043F8041F1D
:107D2000984242F8041FF9D100230121D4F800A0A1
:107D30000DF12409CDE90031CDE902793C2123463A
:107D400052463046FFF74AFF099900296ED1824515
:107D500002D12846FFF77CFD02234FF0010AD4F838
:107D600004B0CDE900A3CDE9025923465A463C218F
:107D700006F10800FFF732FF099B002B56D183451F
:107D80004CD151462846FFF763FD03234FF0020A0A
:107D9000D4F808B0CDE900A3CDE9025923465A46EC
:107DA000182106F11000FFF719FF099B002B3DD1A8
:107DB000834546D151462846FFF74AFD40F26F1BE6
:107DC000A3690593E368049306F114030693DDF8B1
:107DD00010A006F11303079351460698FFF7EDFE36
:107DE00028B105990798FFF7E8FE002836D1BBF1C6
:107DF000010B33D0E36820460133E36010F0CAF989
:107E0000013108BFB0F1FF3F24D0A36929462046C5
:107E1000D4F80CA00593FFF797FEDDE74246214614
:107E20003046FFF75FFF09900028AED0284600F0EB
:107E300087FB17B1384600F083FB09980BB0BDE80B
:107E4000F08F424621463046FFF74CFF099000284C
:107E5000ECD1B3E701234FF0000A0993099B002BF3
:107E6000E4D1049B534520D104212846FFF7F0FCC0
:107E700005230622D4F810A0CDE90032CDE902593D
:107E8000234652460C2106F11800FFF7A7FE099B76
:107E9000002BCBD18245C9D06369A3EB0803042B27
:107EA0000CD94FF0FF330993C0E7424621463046D4
:107EB000FFF718FF09900028B8D1D9E742462146BC
:107EC0003046FFF70FFF0990B0E74FF0FF330993FB
:107ED000002DB2D00027A9E72DE9F04F002487B08C
:107EE000924606AA894642F80C4D2C219846109DD0
:107EF000FFF7DAFC074688B93E4B2B6003993846FA
:107F0000FFF7BDFC07B0BDE8F08FD0F800B0726895
:107F10005A451CD2304600F013FB0134039BA342A8
:107F2000ECD957F824602F213046FFF7DBFBA8B9C6
:107F30002B46304642465146FFF740FD2B68064629
:107F4000002BE2D00028D9D000F0FAFAD6E7594643
:107F50004846FFF70CFE0BF1010BD8E700232F2159
:107F6000304604AA0493FFF79FFC049906464B1E73
:107F7000012B04D9204B2B60FFF781FCBEE7424662
:107F80002B4651460068FFF719FD2A6883462AB13F
:107F900008B100F0D5FA04993046EDE72D2130689C
:107FA000FFF7A0FB18B908F1FF32CBF8042000233B
:107FB00006A941F8043D7068FFF7A6FB059A0090FA
:107FC0001AB10E4A58462A60E3E7DBF80020DBF8D6
:107FD0000410914205D230460499FFF750FC5846F0
:107FE00099E7114648460192FFF7C1FDDDE90032ED
:107FF0001A44ECE7F4C5010806C601082BC60108BF
:108000002DE9FF4100230E460393144602B902AC4A
:10801000236048B90546564B236003992846FFF76D
:108020002EFC04B0BDE8F08103AA2021FFF73CFC40
:10803000039B0546062B02D04E4B2360EDE71A2228
:10804000002130460FF0C3FF009400223C2331464C
:108050002868FFF741FF2268002ADED100943C2304
:1080600006F108016868FFF737FF2268002AD4D1BB
:108070000094182306F11001A868FFF72DFF23686C
:10808000002BCAD16869FFF71FFD07223A496869CA
:10809000FFF758FB804610F06FFE012806F113072A
:1080A00006D198F800303F2B04BF2A2388F800300F
:1080B00000220823394640460094FFF70DFF404652
:1080C00000F03EFA2268002AA7D107213846FFF7C0
:1080D00074FD30B111463846FFF749FD0721FFF71F
:1080E00059FDEF6806F11408384610F045FE0128E6
:1080F00004D13B783F2B04BF2A233B70202300226E
:10810000414638460094FFF7E7FE00214046FFF75E
:1081100041FD2368002B80D12F693846FFF7D4FC3E
:1081200000287FF47AAF38460D221449FFF70AFB86
:10813000074600283FF471AF183600940D23012242
:108140003146FFF7C9FE384600F0FAF9012421460E
:108150003046FFF732FD30B1611E3046FFF707FDB4
:108160002146FFF717FD01340D2CF0D155E700BF74
:10817000D3C40108EBC401087C0000209800002053
:10818000F0B58DB0CDE90023054628B94FF0FF309A
:108190004FF0FF310DB0F0BD2422002103A80FF0F5
:1081A00016FF03A968460FF0F1FD04460028EDD044
:1081B0000FF0F0FF4A1C08BFB0F1FF3F06460F4624
:1081C000E4D0626921462846FFF78CFD0028DDD106
:1081D00020460FF0DFFF4B1C08BFB0F1FF3FD5D0AA
:1081E0008F4208BF864203D020460FF0D3FFD1E76D
:1081F00023682046013323600FF0CCFF013108BF14
:10820000B0F1FF3FC2D0626921462846FFF76AFD00
:108210000028E9D0BAE770B53C258AB0DDE90E64E4
:10822000019496FBF5F405FB14640294182493FB67
:10823000F4F505FB1433CDE90330481E0C2190FB07
:10824000F1F301FB13010023CDE907339DF8403022
:10825000A2F26C7201A80591069209930FF09AFFA1
:108260000AB070BDF7B5044602A860E902230FF01A
:108270007BFD0269037A551C426990F804C0077BB4
:1082800002F26C71067EC2690068A3700033207030
:1082900018BF01232046013284F801C0E770257120
:1082A000A4F80510E6712272637203B0F0BD30B518
:1082B000457A85B0C4788378B0F8052001790295B5
:1082C00005780195407800902046FFF7A4FF05B09F
:1082D00030BD904271EB0303B4BF01200020704712
:1082E000032210B5104986B00B78013393FBF2F2EC
:1082F00002EB42029B1A0D4A0B7052F8234002789F
:10830000B0F80530049242781A21039282780292E2
:10831000C2780192027920460092054A10F0C6FC0C
:10832000204606B010BD00BFB20C0020D4C6010824
:108330009AC60108B1F1004F08BF00281FB50246D8
:108340000B4608D001A8FFF78DFF01A8FFF7C8FF73
:1083500005B05DF804FB0148FAE700BFCCC6010890
:108360002DE9FF4703220D462B4900280B780446D0
:1083700003F1010393FBF2F202EB4202A3EB0203CF
:10838000264A0B7052F8236075F100033EDA4FF075
:10839000010A444265EB4505214A0023204629464F
:1083A0000FF0E4FA1E4A07460023204629460FF044
:1083B000DDFA104619464FF4616200230FF0D6FA39
:1083C0004FF4616280460023204629460FF0CEFA22
:1083D000104619463C2200230FF0C8FA3C22814681
:1083E0000023204629460FF0C1FACDF80080CDE9E0
:1083F00001923B46BAF1000F0BD00A4A1A213046CF
:1084000010F054FC304604B0BDE8F0874FF0000A8D
:10841000C2E7054AF2E700BFB20C0020D4C601084B
:1084200080510100B8C60108B9C601080FB404B0F4
:10843000704700000FB437B51B4C256855B90322AF
:108440002946012002F0A0FB2B462A46294620603F
:1084500002F0BEFB154D2A68013A03321ED8642192
:10846000206802F0A1FD8022002111480FF0AFFD2D
:1084700007AB069A80210E48019311F01BF87F2864
:1084800003DD0C490C4810F06FFC2B680848984736
:10849000002320681A46194602F09AFB03B0BDE893
:1084A000304004B0704700BF3C0D0020B40C0020E9
:1084B000BC0C002058CD0108370D00200FB410B5BA
:1084C0000D4CA2B02268013A033210D825AB249A91
:1084D000802102A8019310F0EDFF7F2804DD0749F9
:1084E0000DF1830010F040FC236802A8984722B0E9
:1084F000BDE8104004B07047B80C002058CD01080A
:1085000070B50446054E4518AC4200D170BD14F854
:10851000011B3046FFF78EFFF6E700BFE0C60108FB
:1085200038B50C461546FFF785FF20462946FFF76C
:10853000E7FFBDE838400148FFF77CBF0AE40108C7
:1085400010B5044670B102F06DF9204602F00EFA43
:1085500002F040F8BDE81040034A9388013393804D
:1085600002F058B810BD00BF7255002070B5214C04
:108570008AB0226806460132632A22601E4D0BDD56
:1085800003F0A0FD0523002201A903F0DDFC03F0A8
:10859000E7F900232860236003F0E2F92B6803F574
:1085A0007A73984204D903F0DBF900232860236032
:1085B000124A134C13781BB92360636001231370B4
:1085C00002F030F9304602F03FF9054668B1324614
:1085D00000210FF0FCFC01F0FDFF23880133238014
:1085E00002F018F828460AB070BD63880133638032
:1085F000F8E700BF440D0020480D0020400D00208A
:1086000072550020006800BA7047008840BA80B2F6
:10861000704700687047837842781B04007843EA0B
:1086200002231843704700887047FFF7F2BFB0F984
:10863000000070470370130E4370130C8370130A0D
:10864000C3700271052070470B0E03700B0C437052
:108650000B0A8370C170042070470B0A03704170CD
:10866000022070470B0A017043700B0C090E8370D7
:10867000C17004207047A0F14103052B02D83738A0
:10868000C0B27047A0F16103052B01D85738F7E756
:108690003038C0B20A2828BFFF20704700220139B5
:1086A00010B50144441E8C4204D014F8010F08B1E7
:1086B000002A01DA104610BDFFF7DDFF0F2802D8AF
:1086C00040EA0212EFE74FF0FF32F3E738B5054614
:1086D0000C4610F0A7FA611B013190FBF1F303FB8C
:1086E0001100284438BD0078013070470FB404B041
:1086F000704700002DE9FF470F46002104AC254ECE
:1087000044F8041D8046924630682246994602F09D
:108710008DFD0128039B31D13BB14FF080521E4BA0
:108720001A60BFF34F8FBFF36F8FB7F5C87F88BF55
:108730004FF4C87741463A4618480FF024FC184DCC
:10874000164B21463068AF802B60A5F806A085F84F
:10875000089002F04DFB039B3BB14FF080520E4B53
:108760001A60BFF34F8FBFF36F8F0E480094002342
:1087700001220421006803F067FE039B3BB14FF028
:108780008052054B1A60BFF34F8FBFF36F8F04B059
:10879000BDE8F087500F002004ED00E0B40D00208C
:1087A000A80D0020580F00200348002301220221B9
:1087B000006803F0DFBD00BF580F00201FB5002385
:1087C0000C4904AA42F8043D08700B48009240216D
:1087D0000122006803F038FE039B3BB14FF080524A
:1087E000064B1A60BFF34F8FBFF36F8F05B05DF874
:1087F00004FB00BF980D0020580F002004ED00E09E
:108800001FB5002304AA42F8043D0A4800928021C3
:108810000122006803F018FE039B3BB14FF0805229
:10882000054B1A60BFF34F8FBFF36F8F05B05DF834
:1088300004FB00BF580F002004ED00E01FB5104BF3
:108840001C680346A8B1002304AA42F8043D009224
:1088500008210122204603F0F7FD039B3BB14FF0B6
:108860008052084B1A60BFF34F8FBFF36F8F04B075
:1088700010BD01220821204603F07CFDF7E700BF70
:10888000580F002004ED00E01FB5002304AA42F8B1
:10889000043D0092012209481146006803F0D4FD0E
:1088A000039B3BB14FF08052054B1A60BFF34F8FD3
:1088B000BFF36F8F05B05DF804FB00BF580F0020B9
:1088C00004ED00E01FB5002304AA42F8043D0A4865
:1088D000009210210122006803F0B6FD039B3BB11A
:1088E0004FF08052054B1A60BFF34F8FBFF36F8F6D
:1088F00005B05DF804FB00BF580F002004ED00E058
:1089000000487047900D0020114810B50023032245
:108910004FF48071006803F02DFD4FF080520D4B35
:108920001A60BFF34F8FBFF36F8F0B4C206802F0BC
:10893000C9FC40B1BDE81040002308481A4619465A
:10894000006802F045B9012003F05AF9EEE700BFD4
:10895000580F002004ED00E0540F00204C0F0020C1
:10896000F8B5104B0146186802F01EFB0446B8B17A
:108970004FF080560C4F0D4D002303224FF4007131
:10898000386803F0F7FC2E60BFF34F8FBFF36F8F93
:10899000386802F05BFF2E60BFF34F8FBFF36F8F1D
:1089A0002046F8BD4C0F0020580F002004ED00E0D9
:1089B000014B1860704700BF440F002070B504469B
:1089C00078B10378032B0CD1436853B10025054ED1
:1089D0001868F26990476068F369056098476560B8
:1089E000257070BD6C0D00200A4810B500230522CB
:1089F0000949006802F0ECF8012805D1074B1B6813
:108A00003BB1BDE8104018470348BDE81040FFF7F0
:108A1000D5BF10BD480F00209C0D0020440F002042
:108A20001FB5064C002201A9206802F02BFA08B9F4
:108A300004B010BD01A8FFF7C1FFF3E7480F002005
:108A4000014B1868704700BF480F002010B504465E
:108A5000064B010AA3F84A00202000F045FBE1B2D2
:108A60002120BDE8104000F03FBB00BF7C55002036
:108A700008B5FFF7EBFF0122014B83F8522008BD38
:108A80007C550020002238B50B4B05461D2083F88D
:108A90004E100C4683F84C2000F07EFB20F00600C0
:108AA00040EA4401C9B21D2000F01EFB2946BDE882
:108AB0003840232000F018BB7C55002013B5164C1D
:108AC0000120A3689847002341F6FE720093009BA3
:108AD000934218DDA36802209847002341F6FE72F6
:108AE0000193019B934212DD0C4BB5211C6C40207D
:108AF000A047A0214120A04700210120234602B029
:108B0000BDE810401847009B01330093DFE7019B4D
:108B100001330193E5E700BF6C0D00203CC701085D
:108B2000094B07B51B6CC2213B209847002341F637
:108B3000FE720193019B934202DD03B05DF804FBDA
:108B4000019B01330193F5E73CC701082DE9F74F7D
:108B5000814B8248824E0360824B834C8360834BFF
:108B6000DFF830924360824BDFF82CB2C360814B58
:108B70000361814B8361814BC36133689847002354
:108B800020681A46194602F023F87D4B1879F0B98F
:108B90004FF0FF33194601AA03F0A8FB0028F4D0D8
:108BA000019BD8051AD500F05DFA002000F0AEFD5B
:108BB000F36A9847FFF734FF0023D9F800001A46FC
:108BC000194602F005F8002003F092F8DDE741F2C3
:108BD000883301AA4FF0FF310020DDE799050DD55C
:108BE00000F040FAFFF79CFFF36A9847FFF718FF81
:108BF0006421D9F8000002F0D7F9C6E7D9F80000DF
:108C000002F060FB0128C0D0DBF8003023B940F24D
:108C10003B115C48F9F7D0FB019B1A0604D50722EB
:108C2000594B1A70FFF7E0FE019B5B074DD5002101
:108C3000206802F0B9F9012847D1DFF860A10C20C3
:108C4000DAF818309847054668B9034602460146E7
:108C5000206801F0BDFF002897D14FF4A871494862
:108C6000F9F7AAFB91E7DFF83881DAF81830B8F89D
:108C700004009847074678B9DAF81C302846984728
:108C80003B463A463946206801F0A2FF00287FF4AF
:108C90007CAF4FF4AC71E2E708F1040303CB2F6023
:108CA0006860A9603846D8F80010B8F804200FF0C2
:108CB0006AF90322344B1A705D60FFF795FE0023BA
:108CC00020681A46194601F083FF019BDF0709D58A
:108CD00001232D4D2B7000236B6002F041FEA86034
:108CE000FFF782FE019BDD0606D50522264B1A7092
:108CF00000225A60FFF778FE019B180706D5042270
:108D0000214B1A7000225A60FFF76EFE019B9907F3
:108D100006D502221C4B1A7000225A60FFF764FE2F
:108D2000019B9A0606D50622174B1A70174A5A60FD
:108D3000FFF75AFE019B5B067FF527AF144B1A78AD
:108D4000114B32B108221A7000225A60FFF74CFE14
:108D50001BE70922F7E700BF898800084C0D0020B7
:108D60003CC70108F5860008500F0020A9870008BD
:108D70003D880008C5880008BD87000801880008F4
:108D8000900D0020EEC601089C0D0020990D0020DA
:108D9000980D0020540F0020480F00206C0D00207B
:108DA000A80D0020044B10B55B6998470446FFF7F7
:108DB00085FE204610BD00BF3CC70108F0B55D4CE4
:108DC000064625460F460FCE0FC596E80F0085E8EC
:108DD0000F0097E803006369574D013B033388BFD9
:108DE000564B85B088BF6361636885E80300013B2B
:108DF000033304D94FF423715148F9F7DDFA23689E
:108E0000013B033304D94FF424714D48F9F7D4FAE8
:108E1000A368013B033304D94FF425714848F9F79F
:108E2000CBFAE368013B033304D94FF4267144487D
:108E3000F9F7C2FA2369013B033304D94FF42771D0
:108E40003F48F9F7B9FAE369013B033304D94FF41A
:108E500028713B48F9F7B0FAA369013B033304D901
:108E60004FF429713648F9F7A7FA364B0FCB8DE846
:108E70000F0094E80F0000F0CBF823689847FFF745
:108E80001DFE314B42205B6C9847222807D040F2F0
:108E9000B6212B48F9F790FA002005B0F0BD032267
:108EA0000021012001F070FE284B1860012001F024
:108EB00033FF274B186020B940F2BF212048F9F753
:108EC0007BFA012001F028FF224C206020B940F2FB
:108ED000C3211B48F9F770FA4FF0FF31206802F008
:108EE00063F800220C21032001F04EFE1A4B18609B
:108EF00010B940F2C921CCE7184B194A1A602B6807
:108F00000BB904232B60174B1C680CB10120C4E77C
:108F100001932B68FA22009313490123134802F0AE
:108F2000FDFA0128F2D0064840F2DB21F9F744FAB5
:108F30002046B2E76C0D0020900D0020ED86000861
:108F4000EEC601087C0D00203CC70108500F002030
:108F50004C0F0020540F0020480F00208C0D0020E3
:108F6000E7860008580F0020E6C601084D8B000870
:108F7000014B83F8280070477C550020014B186096
:108F8000704700BF8C0D002070B5084C0546226864
:108F90000E4622B940F2EB210548F9F70DFA236895
:108FA00031462846BDE87040184700BF8C0D0020B0
:108FB000EEC6010800F046B8034B03440348834261
:108FC0008CBF0020012070470071BDCCFF6789096C
:108FD0000120704708B5FFF793FC4379002B0CBFC5
:108FE0008020002008BD0000002310B5074951F87B
:108FF0003340DA00844203D80A449468844203D898
:109000000133152BF3D1FEE7107910BDA8C7010875
:1090100084B030B503AC84E80F00064C03AD0FCD2F
:109020000FC495E80F0084E80F00BDE8304004B09D
:10903000704700BF88120020014B1878704700BFAE
:109040007C550020C82307B50093002304481A4626
:109050000321006803F024FB03B05DF804FB00BFAC
:10906000600F002013B5104C0120A368984700231F
:109070000093009BB3F5CC7F0FDDA36800209847D9
:10908000002342F6FE720193019B934208DD022009
:10909000A36802B0BDE810401847009B0133E7E722
:1090A000019B01330193EFE7881200202DE9F04185
:1090B00007460C4C0D46E368002016469847236986
:1090C00047F080009847013D2E44B54204D1E36843
:1090D0000120BDE8F0411847236915F8010F9847B2
:1090E000F3E700BF8812002007B502AB03F8011DAB
:1090F00001221946FFF7DAFF03B05DF804FB000018
:10910000134A10B55060134A904219D00DF090FDEB
:109110000DA3D3E900230DF02FFF0EF09DF80446B8
:10912000C4F307410620FFF7DFFFC4F30721072040
:10913000FFF7DAFFE1B20820BDE81040FFF7D4BF27
:10914000054CEDE7AFF300800000000080844E4046
:109150007C550020F01FCB33CD3CD9002DE9F041E8
:1091600007460C4C0D46E3680020164698472369D5
:1091700007F07F009847013D2E44B54204D1E368D3
:109180000120BDE8F041184723690020984705F801
:10919000010FF2E78812002007B501220DF1070147
:1091A000FFF7DCFF9DF8070003B05DF804FB00004B
:1091B00001282DE9F84F0D4603D0022854D0002095
:1091C0004BE06D4E2720B48BFFF7E6FFA4B220F0F2
:1091D000F800013420440DF02BFDB37F0022002B5A
:1091E0003DD1664B0DF0E8FB804630208946FFF705
:1091F000D3FF30F0F9030CBF0023604B0022404640
:1092000049460DF0D9FB8046284689460DF020FDE1
:1092100002460B46404649460DF0CEFB96F82030FC
:109220000022F3B900230DF0C7FB0022544B0DF0D0
:1092300079FDB669044630460D460DF0F9FC02464C
:109240000B46204629460DF097FE00224D4B0DF0AF
:1092500069FD0DF05DFB0DF0FFFFBDE8F88F002309
:10926000C0E74FF08043DEE7434C226C022A79D8F6
:10927000454B03EBC203D3E900670120636C9840C0
:109280000DF0E6FC02460B46304639460DF074FE02
:1092900002460B46002039490DF06EFE06460F4689
:1092A000B4F84A000DF0D4FC0022384B0DF084FBDA
:1092B00032463B460DF036FD8B46616C824694F893
:1092C0004E0094F84C308900002BC1F11C0101EBD9
:1092D000001114BF1420002001EBC501081A0DF085
:1092E000A7FC8046606C94F848308946002B14BF78
:1092F00002230023C3EB80000DF09AFC02460B46CC
:10930000404649460DF038FE0DF0F6F98046894694
:1093100094F8490004300DF09BFC42464B460DF09A
:1093200001FD0022002304460D460DF08BFFE0B145
:109330000022134B204629460DF03EFB32463B46A9
:109340000DF0F0FC52465B460DF036FB00220D4B53
:109350000DF0E8FC06A3D3E900230DF02DFB0DF082
:1093600053FA78E70026002787E700200449E5E75D
:109370002B8716D9CEF7EF3F7C5500200000F03F39
:109380000000204000408F4090C7010800001140BD
:10939000012808B504D002280AD04FF0FF3006E0BB
:1093A0001120FFF7F9FEC0F34700404200B208BDAC
:1093B0001B20FFF7F1FE8B38F8E700000B4B10B5D0
:1093C0005B68044660B9022098470120FFF7E4FE7D
:1093D00000F0F80121430120BDE81040FFF784BEF2
:1093E00003280CBF01200020EEE700BF88120020F8
:1093F00013B5C82400230B4800941A4603210068C3
:1094000003F04EF90023084800941A46032100682F
:1094100003F046F90020FFF7D1FF0022034B1A703A
:1094200002B010BD600F0020841200207C55002087
:1094300013B5C82400230B4800941A460321006882
:1094400003F02EF90023084800941A46032100680F
:1094500003F026F90120FFF7B1FF0022034B1A7039
:1094600002B010BD600F0020841200207C55002047
:1094700073B55D4C06466378DBB2012B03D0022B3B
:1094800065D0002538E0402094F82250FFF784FE94
:109490000C214020FFF728FE4120FFF77DFE60F001
:1094A0000E01C9B24120FFF71FFE3520FFF774FE01
:1094B00000F0C00141F012013520FFF715FE352004
:1094C000FFF76AFE00F03F00112184F83A003F20C8
:1094D000FFF70AFE00230D2084F82C3084F82D308D
:1094E0002387E386FFF758FE00F04001EDB241F01C
:1094F0002E010D20FFF7F8FD4FF4C87200213B4804
:109500000EF065FD01232370394B18684FF0FF33CF
:10951000002E5BD04FF47A7101FB06F20093B2FB90
:10952000F1F20023042103F0BBF86378012B52D140
:109530000520FFF743FF0D20FFF72EFE40F020012E
:109540000D20C9B202B0BDE87040FFF7CDBD94F860
:10955000513033201BB3FFF71FFE40F04101C9B269
:109560003320FFF7C1FD19213B20FFF7BDFD94F823
:10957000525094F84F30EDB2E3B11D211120FFF7A6
:10958000B3FD4020FFF708FE00F033014020FFF755
:10959000ABFD00210F20FFF7A7FD0021A9E7FFF792
:1095A000FBFD00F0BE0141F001013320FFF79CFDFF
:1095B0001D21D9E70F211120FFF796FD4020FFF76D
:1095C000EBFD00F03C0141F00101DFE70093324682
:1095D00033460321A7E72DB1052002B0BDE8704056
:1095E000FFF7ECBE0620F8E77C550020640F002052
:1095F000600F002037B54FF47A72642350432B4D2F
:10960000B0FBF2F2009304210023286803F048F82D
:109610000022274B274C1A706378DBB2012B14D041
:10962000022B26D0022323702C6802F099F905231F
:109630000246009301210023204603F031F8032065
:1096400003B0BDE83040FFF7B9BE14214020FFF75A
:109650004BFDB0214120FFF747FD8F213520FFF75B
:1096600043FD3520FFF798FD00F03F0084F83A00F5
:10967000D8E794F84F3073B1F5211120FFF734FD8E
:109680004020FFF789FD00F0330141F04001402008
:10969000FFF72AFDC6E7F7211120FFF725FD40203F
:1096A000FFF77AFD00F03F01EFE700BF84120020D2
:1096B000A81200207C55002010B5124C6378DBB254
:1096C000012B04D0022B09D040F2114101E040F2FD
:1096D000FA31BDE810400C48F8F76EBEFA211120AF
:1096E000FFF702FD4020FFF757FD00F0FC0140208E
:1096F000FFF7FAFC032307202370BDE81040FFF7B3
:109700005DBE00BF7C5500206CC8010808B51A4B2F
:109710005A7882422ED058705B780020022B13D0EA
:10972000FFF74CFE0120FFF737FD00F07F0101201D
:10973000FFF7DAFC00214020FFF7D6FC3021412062
:10974000BDE80840FFF7D0BCFFF738FE0120FFF767
:1097500023FD60F07F01C9B20120FFF7C5FC0021A5
:109760004020FFF7C1FC00214120FFF7BDFC432151
:109770003120E5E708BD00BF7C5500201D4B13B527
:10978000186000231C4C1A4600944FF47A711B4851
:1097900002F064FF1A4B186020B94FF48671194823
:1097A000F8F70AFE002300941A464FF47A7116481F
:1097B00002F054FF154B186020B94FF4877111481F
:1097C000F8F7FAFDFFF74EFC0020FFF79FFF00209F
:1097D000FFF7F4FD4FF4C87200210D480EF0F7FBBF
:1097E000002201210B4B83F8282083F829101A70DE
:1097F00002B010BD5C0F0020BD9D000858C80108D4
:10980000841200206CC801085BC80108600F0020AA
:10981000640F00207C55002073B50E4614460546A3
:10982000FFF774FF3046FFF76BFC0520FFF7C6FD1E
:1098300000230193019BB3F5CC7F0BDD2846FFF796
:10984000A7FD0546FFF7D4FDA542CCBF00200120AF
:1098500002B070BD019B0133EBE773B50024022019
:10986000FFF754FFFF211120FFF73EFC0520FFF713
:10987000A5FD254626460196019BB3F5CC7F0DDD5F
:109880002C20FFF789FC00F00100A0400134202CBF
:1098900045EA0005EFD1284602B070BD019B0133B7
:1098A0000193E9E7000000002DE9F04F824687B000
:1098B0000093109B0D4601939DF85C309DF8581065
:1098C000029393469DF864309DF8602003930492C0
:1098D000BDF84460BDF848409DF84C709DF850803C
:1098E0009DF854900591FFF711FFDDE90332BAF1BD
:1098F000010F06D0BAF1020F059968D007B0BDE894
:10990000F08F7F4C019925615846C4F818B0616109
:10991000A77784F81F8084F8209084F8212084F8A9
:109920002230A6830DF084F902460B4672A1D1E9DC
:1099300000010DF021FB0DF08FFC1FFA80FB4FEAB8
:109940001B210220FFF7D0FB5FFA8BF10320FFF70A
:10995000CBFB2846FFF748FB01461220FFF7C4FB6C
:109960000198FFF741FB01461320FFF7BDFB310AC9
:109970002520FFF7B9FBF1B22620FFF7B5FBE27F08
:109980002346DAB9A27FCAB184F829A04146322021
:10999000FFF7AAFB3020FFF7FFFB002F14BF0021C9
:1099A000802100F06F0040EA0919302041EA0901E6
:1099B000C9B207B0BDE8F04FFFF796BB00224FF4E5
:1099C000D271504883F82920F8F7F6FCDEE74C48BE
:1099D0009DF800C00564C0F844B080F849C0A0F804
:1099E0004A6080F84C7080F84D8080F84E9080F886
:1099F0004F109DF80810BBF10C0F80F850108246F4
:109A000080F8512080F8523072D8BBF1050F60D930
:109A100025B9ABF10B03012B5DD804E0012D5AD120
:109A2000BBF10C0F57D101238AF848301D20FFF7F6
:109A3000B3FB9AF84810009B41EA490141EA8701CB
:109A400041EAC30141EA8511C9B21D20FFF74CFB71
:109A50001E20FFF7A1FBC4F3012100F00C0001431D
:109A600041EA0B11C9B21E20FFF73EFBE1B21F20F5
:109A7000FFF73AFB310A2020FFF736FBF1B2212035
:109A8000FFF732FB1FB141462220FFF72DFB9AF86A
:109A90004F306BB14B20FFF77FFB60F07F01C9B205
:109AA0004B20FFF721FB9AF850102420FFF71CFBF6
:109AB000BBF1060F4FF031000FD1FFF76DFB00F047
:109AC000F80141F005013120FFF70EFB0C21372092
:109AD0006FE74FF0060B0023A6E7FFF75DFB00F0F2
:109AE000F80141F003013120FFF7FEFA0A21EEE709
:109AF0004FF00C0B012D8FE70000000080847E41A9
:109B00007C5500206CC801082DE9F04F89B01E4635
:109B10009DF84C300C4602939DF85C300192059301
:109B20009DF86030009006939DF86430129D039379
:109B30001A9BBDF8507004939DF854809DF858907E
:109B4000FFF7E4FD0920FFF727FB82465A20FFF7C5
:109B500023FB0AF07F01DFF860A28346DAF80400F5
:109B60000791FFF737FA07990843C0B2030600F0E0
:109B7000F00C2ED5112CCBBF4BF007020BF0F802E6
:109B80005FFA82FB42F0040B0BF00701072918D1A2
:109B9000142CA8BF1424052CB8BF0524611F4CEA5F
:109BA0000101C9B20920FFF79FFA59465A20FFF771
:109BB0009BFA009B012B13D0022B6CD009B0BDE89F
:109BC000F08F112CA8BF1124022CB8BF0224A11EB3
:109BD000E5E70E2CA8BF0E2444EAE474611CDEE71E
:109BE000019B8AF80840CAF80C309DF80C30CAF87E
:109BF0001060CAF81850AAF81C708AF81E808AF8FB
:109C000020908AF82130049B0198CAF824300DF086
:109C10000FF865A3D3E900230DF0AEF90DF01CFB9E
:109C200084B2210A0420FFF75FFAE1B20520FFF7B2
:109C30005BFA28460CF0FCFF02460B465CA1D1E91A
:109C400000010DF099F90DF007FB84B2210A022002
:109C5000FFF74AFAE1B20320FFF746FA390A252056
:109C6000FFF742FAF9B22620FFF73EFA3020FFF75D
:109C700093FAB8F1000F0CBF8021002100F06F00B3
:109C800040EA0919302041EA0901C9B209B0BDE82A
:109C9000F04FFFF729BA484A9DF8083082F83C4057
:109CA0001664556482F849309DF81430A2F84A7061
:109CB00082F84C8082F84F309DF818300C2D82F8D5
:109CC00050309DF80C3082F84E9082F85130049B51
:109CD0001446536562D8052D52D926B9A5F10B0259
:109CE000012A4ED803E0012E4BD10C2D49D101227F
:109CF00084F8482094F84F206AB14B20FFF74CFAC3
:109D000060F07F01C9B24B20FFF7EEF994F85010D4
:109D10002420FFF7E9F91D20FFF73EFA9AF84810D2
:109D2000029B41EA490141EA880141EAC30141EA53
:109D30008611C9B21D20FFF7D7F91E20FFF72CFAB4
:109D400000F00F0141EA0511C9B21E20FFF7CCF95E
:109D5000390A2020FFF7C8F92120F9B2FFF7C4F92A
:109D6000062D4FF031000ED1FFF716FA00F0F80182
:109D700041F005013120FFF7B7F90C21372085E7C5
:109D800006250022B4E7FFF707FA00F0F80141F0DA
:109D900003013120FFF7A8F90A21EFE70C25012E76
:109DA0009FE700BFAFF300800000000080844E40BA
:109DB0000000000080847E417C55002010B5254CB9
:109DC0002378DBB2012B02D0022B34D010BD637894
:109DD000012B29D100230B213E2084F82C3084F85C
:109DE0002D302387E386FFF77FF910213F20FFF70F
:109DF0007BF994F8223003F0FF029BB10D20FFF7AE
:109E0000CBF940F02001C9B20D20FFF76DF9124BDC
:109E10001B68002BDAD0DB68002BD7D0BDE81040E0
:109E2000002018472270F2E794F85230002BEED051
:109E3000FFF7FEFAEBE7002301222370074B1A70AD
:109E4000054B1B68002BC1D05B68002BBED0BDE862
:109E5000104018477C5500205C0F0020A8120020FD
:109E600007B50022154B8DF8072083F82C2083F8C6
:109E70002D201A87DA8683F82E2093F8223023B912
:109E800003B05DF804EBFFF7B3BA3F20FFF784F9A6
:109E90008DF807009DF80730DB0603D510213F2021
:109EA000FFF722F90D20FFF777F940F040010D2070
:109EB000C9B203B05DF804EBFFF716B97C5500207A
:109EC0002DE9F04107460D4C0D46E368002016468B
:109ED0009847236907F07F009847013D2E44B5421B
:109EE00004D1E3680120BDE8F04118472369002050
:109EF0009847C04305F8010FF1E700BF8812002022
:109F00000A4601460020FFF7D1B80000F7B5554CCE
:109F1000064663780D46DBB2012B04D0022B34D009
:109F2000002528461AE0002323878BB2E386A37F0F
:109F300013B13220FFF7D8F86B1E3F2B1BD884F8E3
:109F40003B500025304694F83B10FFF7D9FF94F8BA
:109F50003B30228F13449BB22387606AFFF74AFB92
:109F60006378012B7BD1002D79D03F4E3F4D337864
:109F7000002B4DD073E02A4631463C480EF003F8E2
:109F80003C23012584F83B30DCE794F85130332042
:109F90002BB3FFF701F900F0BE013320FFF7A4F85F
:109FA00019213B20FFF7A0F82946222084F85C50B5
:109FB000FFF79AF800210E20FFF796F800210D20F8
:109FC000FFF792F80120FFF7E7F830F0F80711D01B
:109FD00029463046FFF794FF0025606DBEE7FFF786
:109FE000DBF800F0BE0141F001013320FFF77CF8FF
:109FF0001D21D6E7FFF71CFA0197019BB3F5CC7F33
:10A00000E6DC019B01330193F7E7012001F0F8FD45
:10A010003F20FFF7C1F88306F7D4E38E218F94F831
:10A020003B205B1A9342208F0BDD94F83B102844B1
:10A03000FFF766FF94F83B30228F13449BB22387CF
:10A0400095E7E18E238F2844C91AC9B2FFF758FF5C
:10A05000E18E228F238F0B449B1A9BB2238703B080
:10A06000F0BD00BF7C550020A8120020640F002026
:10A070000A4601460020FFF771B80A460146002053
:10A08000FFF71EBF38B505460C46FFF73FFB012D15
:10A0900002D0022D0AD038BD064B9B7F002BFAD18F
:10A0A00021463220BDE83840FFF71EB82146232064
:10A0B000F8E700BF7C5500207FB50022654D8DF884
:10A0C0000B202B780392DBB2012B2C4604D0022B01
:10A0D00000F09E8004B070BD6B78DBB2012B34D0F1
:10A0E000022BF7D140211220FEF7FEFF1220FFF7CE
:10A0F00053F88DF80B009DF80B30574E13F0200FDE
:10A1000029D020211220FEF7EFFF95F8523003F0FE
:10A11000FF0203B92A7000225048009203AB0821C5
:10A12000006802F0BDFA039B3BB14FF080524C4BEC
:10A130001A60BFF34F8FBFF36F8F3368002BC9D006
:10A140001B69002BC6D09847C4E740F21C51454814
:10A15000F8F732F9BEE71920FFF71EF840B285F88C
:10A16000580095F8583095F858501B0642BF6DB20C
:10A170006D42C5F385054FF01A004CBF6D42AD0826
:10A18000FFF70AF8002D40F30B13B8BF40198B38C6
:10A190009BB203441BB2A4F85A301320FEF7FCFF15
:10A1A00084F85C001020FEF7F7FF01460D20FEF753
:10A1B0009BFF94F85C102C48FFF75AFF94F852303C
:10A1C00003F0FF028BB925482270009203AB0821EF
:10A1D000006802F065FA039B3BB14FF08052204BC0
:10A1E0001A60BFF34F8FBFF36F8F3368002B3FF4BC
:10A1F00071AF9D68002D3FF46DAF94F85C10B4F81A
:10A200005A2094F8583012B25BB21748A84761E759
:10A210001648009203AB0821006802F041FA039B44
:10A220003BB14FF080520E4B1A60BFF34F8FBFF31C
:10A230006F8F6378022B03D108211220FEF754FFA1
:10A2400000232370044B1B68002B3FF443AF1B68B3
:10A2500077E700BF7C5500205C0F0020600F0020D6
:10A2600004ED00E06CC80108640F00208412002097
:10A270002DE9FF41002259498DF80B200B780392FC
:10A28000DBB2012B0C4605D0022B00F0A58004B0F8
:10A29000BDE8F0814B78DBB2012B22D0022BF6D146
:10A2A0004F48009203AB0821006802F0F9F9039BC4
:10A2B0003BB14FF080524B4B1A60BFF34F8FBFF34F
:10A2C0006F8F80211220FEF70FFF00232370464B73
:10A2D0001B68002BDBD0DB68002BD8D0012098470F
:10A2E000D5E73F20FEF758FF8DF80B009DF80B30A7
:10A2F0009A06CCD59DF80B30DB0605D53B48FEF71A
:10A30000DDF8FFF7ADFDC2E794F8293023B940F23C
:10A31000C1513748F8F750F894F82830022B2DD166
:10A32000238F344894F83A101844FFF7A6FE238F81
:10A330009BB2002B3DD094F83A30228F13449BB24D
:10A340002387238FE28E9A42A1D8E28E29492A4898
:10A350000DF019FE94F82E50E48EFFF781FD224B8C
:10A360006DB21B68A4B2002B91D09E68002E8ED0D7
:10A3700000232A4621462048B04788E71F4D002089
:10A38000EB6898472B69002098470027DFF8648026
:10A3900094F83A30BB4203DCEB6801209847C6E7EB
:10A3A0002B690020268F9847B6B24644F0550137F6
:10A3B000EEE794F82D30002BA3D094F83A100D4816
:10A3C000FEF7E2FDE086E38EB3F5C87F99D2E38E17
:10A3D0009BB2002B95D0AEE74B7858E77C55002018
:10A3E000600F002004ED00E05C0F00205EC8010853
:10A3F0006CC80108640F0020F410002088120020AF
:10A4000010B51A4C2378DBB2012B02D0022B2AD0D4
:10A4100010BD6178C9B2012918D00229F8D194F889
:10A420004F30002BF4D01220FEF75EFE104B1B685D
:10A43000002BEDD05C69002CEAD01C20FEF7ACFEAE
:10A440002346BDE8104000F03F00184700231120CC
:10A45000238784F82D10FEF79FFE4008404240B24B
:10A4600084F82E00D4E76178C9B2D6E77C55002085
:10A470005C0F00201F4B70B55A78022A05D11B785B
:10A48000DBB2012B02D0032B13D070BD1220FEF7DC
:10A4900083FEC306F9D510211220FEF725FE164BC8
:10A4A0001B68002BF1D0DB69002BEED0BDE87040BB
:10A4B00018471220FEF770FE10F001050E4C0DD06B
:10A4C00005211220FEF710FE2368002BDDD09B69CA
:10A4D000002BDAD00120BDE870401847042112207B
:10A4E000FEF702FE2368002BCFD09B69002BCCD057
:10A4F0002846F0E77C5500205C0F0020074A53787F
:10A50000012B09D11378DBB2012B05D102213E20AA
:10A5100082F82C30FEF7E8BD704700BF7C55002064
:10A52000014B5B78704700BF7C55002006480068EF
:10A53000006880F3088862B661B6BFF34F8FBFF33F
:10A540006F8F00DF00BF000008ED00E0002307B5BB
:10A5500001930B4B1B68013303D0CA210948F7F75D
:10A560002BFF4FF0500383F31188BFF36F8FBFF3BE
:10A570004F8F019B002BFCD003B05DF804FB00BFA4
:10A58000CC000020C1C801084FF0807340F8043CA3
:10A59000054B21F0010140F8081C40F80C3C40F844
:10A5A000202C4038704700BF4DA500080000000077
:10A5B000074B19680868B0E8F00F80F30988BFF30B
:10A5C0006F8F4FF0000080F311884EF00D0E704732
:10A5D000C84E00204FF0500383F31188BFF36F8FF4
:10A5E000BFF34F8F084A13680133012B136009D161
:10A5F000064B1B6813F0FF0F04D040F2751104489E
:10A60000F7F7DABE704700BFCC00002004ED00E091
:10A61000C1C8010810B5074C236823B94FF4BE71B7
:10A620000548F7F7C9FE2368013B23600BB983F3A4
:10A63000118810BDCC000020C1C801080000000036
:10A64000EFF30980BFF36F8F0D4B1A6820E9F00F0D
:10A6500010602DE908404FF0500080F3118801F0A0
:10A66000F5FA4FF0000080F31188BDE80840196842
:10A670000868B0E8F00F80F30988BFF36F8F704768
:10A68000C84E002008B54FF0500383F31188BFF384
:10A690006F8FBFF34F8F01F06FF918B14FF08052F9
:10A6A000024B1A60002383F3118808BD04ED00E01B
:10A6B0000022054B05491A600A6041F26701044A0D
:10A6C000116007221A60704710E000E018E000E017
:10A6D00014E000E013B5264B264C1A78D2B2019252
:10A6E000FF221A701B78244ADBB28DF803309DF8E4
:10A6F000033003F0500313700723002223609DF8FA
:10A700000310581E090629D402B123602368032BC5
:10A7100004D04FF49B711948F7F74EFE2368144A92
:10A720001B0203F4E06323600024019BDBB213707F
:10A73000134B1A6842F470021A601A6842F07042B1
:10A740001A60FFF7B5FF0F4B1C60FFF7EFFE01F03B
:10A750007DFAFFF7FBFE204602B010BD9DF80330E6
:10A7600001225B00DBB28DF803300346C7E700BF70
:10A7700000E400E0AC120020A9120020C1C80108CA
:10A7800020ED00E0CC00002008B5EFF305830F2B8F
:10A790000AD90D4A9B5C0D4A12789A4204D940F2BC
:10A7A000A5210B48F7F708FE0A4B0B4A1B681268F5
:10A7B00003F4E063934206D9BDE8084040F2B521B6
:10A7C0000348F7F7F9BD08BDF0E300E0A912002047
:10A7D000C1C801080CED00E0AC12002010B50F4B11
:10A7E0001A68824218D35C681919884201BF41680F
:10A7F000184609195960446801198A4207D1084965
:10A8000009688A421FBF516812680919416098425D
:10A81000026018BF186010BD1346E1E7C04E00206B
:10A82000B012002038B5064B064D1C68246804B9E8
:10A8300038BD6307FAD079212846F7F7BDFDF5E763
:10A84000C04E002021C901082DE9F843074601F058
:10A850007FF83F493F4D0B680BBB3F4A3F4E5007C7
:10A860001DBFD01D20F0070002F570534FF4705348
:10A870001CBF02461B1A00201344083B23F00703A9
:10A8800070603260C3E90000981A0B60C2E90030C2
:10A89000334B1860334B18604FF000432B602B682C
:10A8A0001F4252D1002F41D007F1080462071CBF9C
:10A8B00024F007040834002C47D02A4B1A68984625
:10A8C000A24242D3254B1E687268A24202D230686F
:10A8D000002837D10968B14237D01F683168121B90
:10A8E000102A07F10807196010D906EB040919F0BE
:10A8F000070F03D0D7211C48F7F75EFD7368484661
:10A900001B1BC9F804307460FFF768FF14497268B4
:10A91000D8F8003008689B1A8342C8F8003038BF66
:10A920000B602B68134373600023336001F0B4F8AD
:10A930007B0704D040F217110B48F7F73DFD38466E
:10A94000BDE8F88333460646BEE70027EEE700BFC2
:10A95000B0120020B44E0020B4120020C04E0020DF
:10A96000BC4E0020B84E002021C9010838B504466D
:10A9700070B3184D50F8041C2A68114204D140F2FB
:10A980002B111548F7F718FD54F8083C23B14FF484
:10A9900096711148F7F710FD54F8043C2A681342E9
:10A9A00016D054F8081C99B923EA020344F8043C71
:10A9B00000F0CEFF094A54F8043C1168A4F10800E5
:10A9C0000B441360FFF70AFFBDE8384001F064B89C
:10A9D00038BD00BFB44E002021C90108B84E002088
:10A9E000014B1868704700BFB84E0020014B186833
:10A9F000704700BFBC4E002010B50446FFF7EAFDCB
:10AA0000A46BFFF707FEB4FA84F0400910BD70B5DF
:10AA10001546026C0446866B42B905689DB980688C
:10AA200001F0B8FBA5600136A66370BD6DB9406842
:10AA30000DF0A9FA6368226C1344A2686360934224
:10AA400001D3236863600020EDE7C0680DF09BFA36
:10AA5000236CE2685B4221681A448A42E2603EBF8E
:10AA6000A2689B18E360022DEDD10EB1013EEAE72A
:10AA70003046D8E703461A6C10B4084662B1D9686C
:10AA80009C681144A142D96028BF196810BC28BF36
:10AA9000D960D9680DF077BA10BC704770B504461C
:10AAA000FFF798FD94F8455004F124066DB2002D8F
:10AAB00014DCFF2384F84530FFF7ACFDFFF78AFD77
:10AAC00094F8445004F110066DB2002D12DCFF23FF
:10AAD00084F84430BDE87040FFF79CBD636A002BEA
:10AAE000E7D0304601F0A8F908B101F027FA013D9E
:10AAF0006DB2DCE72369002BE9D0304601F09CF908
:10AB000008B101F01BFA013D6DB2DEE738B50D4624
:10AB1000044620B940F203111948F7F74DFCFFF73E
:10AB200059FDD4E90F314B432268D0185B1A134406
:10AB3000A060E3600020FF23A063626084F84430DB
:10AB400084F8453095B9236963B104F1100001F030
:10AB500073F938B14FF080520A4B1A60BFF34F8F30
:10AB6000BFF36F8FFFF756FD012038BD04F11000D1
:10AB700001F0D6FE04F1240001F0D2FEF2E700BF9E
:10AB80007FC9010804ED00E0F8B50D4617460646FA
:10AB900020B94FF4BB710D48F7F70EFC05FB06F02A
:10ABA0005030FFF751FE044648B155B92060C4E962
:10ABB0000F6501212046FFF7A9FF84F84C7020465D
:10ABC000F8BD00F150030360F1E700BF7FC9010841
:10ABD0002DE9FF47884601921E46044620B940F2FF
:10ABE000F1214B48F7F7E8FBB8F1000F06D1236CD1
:10ABF00023B140F2F2214648F7F7DEFB022E07D1DF
:10AC0000E36B012B04D040F2F3214148F7F7D4FB6A
:10AC100001F05EFA30B9019B23B140F2F6213C48C5
:10AC2000F7F7CAFB0027B946DFF8E8A0FFF7D2FC28
:10AC3000A26BE36B9A4201D3022E19D132464146F0
:10AC40002046FFF7E4FE636A1BB104F1240001F023
:10AC5000F3F838B14FF080522E4B1A60BFF34F8F8C
:10AC6000BFF36F8FFFF7D6FC012004B0BDE8F0877B
:10AC7000019D1DB9FFF7CEFC0020F6E717B902A829
:10AC800001F01AF9FFF7C6FC00F062FEFFF7A2FC24
:10AC900094F84430FF2B08BF84F8449094F8453072
:10ACA000FF2B08BF84F84590FFF7B4FC01A902A868
:10ACB00001F00EF928BBFFF78DFCA26BE36B9A4203
:10ACC0000ED1FFF7A7FC019904F1100001F07AF80A
:10ACD0002046FFF7E3FE00F0DFFE48B10127A5E7BD
:10ACE000FFF798FC2046FFF7D9FE00F0D5FEF5E708
:10ACF0004FF08053CAF80030BFF34F8FBFF36F8F10
:10AD0000ECE72046FFF7CAFE00F0C6FEB4E700BF3E
:10AD10007FC9010804ED00E010B5024600210120C2
:10AD2000FFF732FF044638B1002383600360C3603D
:10AD30001A461946FFF74CFF204610BD2DE9F8438F
:10AD4000894690461F46044620B940F2C331274841
:10AD5000F7F732FBB9F1000F06D1236C23B14FF4A2
:10AD600071712248F7F728FB022F07D1E36B012B03
:10AD700004D040F2C5311D48F7F71EFBFFF704FD74
:10AD8000EFF311864FF0500383F31188BFF36F8FF9
:10AD9000BFF34F8FA26BE36B9A4201D3022F22D1F4
:10ADA00094F845503A466DB249462046FFF72FFECB
:10ADB0006B1C13D1636A0BB901200BE004F1240072
:10ADC00001F03AF80028F7D0B8F1000FF4D00120D4
:10ADD000C8F8000086F31188BDE8F88301356DB22C
:10ADE00084F84550E8E70020F4E700BF7FC9010878
:10ADF00070B50D46044620B94FF48C612048F7F732
:10AE0000DBFA236C23B140F264411D48F7F7D4FA12
:10AE1000236833B9A36823B140F269411848F7F7B2
:10AE2000CBFAFFF7B1FCEFF311864FF0500383F339
:10AE30001188BFF36F8FBFF34F8FA26BE36B934209
:10AE40001CD994F8453001325BB2A2635A1C10D170
:10AE5000636A0BB9012009E004F1240000F0ECFF63
:10AE60000028F7D0002DF5D00120286086F3118846
:10AE700070BD01335BB284F84530EBE70020F5E7A5
:10AE80007FC901082DE9F04385B00F4601920446C1
:10AE900020B94FF4A0614248F7F78EFA37B9236C16
:10AEA00023B140F204513E48F7F786FA01F010F959
:10AEB00030B9019B23B140F209513948F7F77CFAC8
:10AEC0000026B046DFF8DC90FFF784FBA56BD5B118
:10AED00039462046013DFFF7CDFDA563236963B1E7
:10AEE00004F1100000F0A8FF38B14FF080522D4B54
:10AEF0001A60BFF34F8FBFF36F8FFFF78BFB0120FB
:10AF000005B0BDE8F083019D1DB9FFF783FB00206C
:10AF1000F6E716B902A800F0CFFFFFF77BFB00F0C1
:10AF200017FDFFF757FB94F84430FF2B08BF84F858
:10AF3000448094F84530FF2B08BF84F84580FFF724
:10AF400069FB01A902A800F0C3FFF0B92046FFF792
:10AF500053FDA0B1019904F1240000F033FF204615
:10AF6000FFF79CFD00F098FD38B94FF08053C9F809
:10AF70000030BFF34F8FBFF36F8F0126A4E7204649
:10AF8000FFF78CFD00F088FDF7E72046FFF786FD10
:10AF900000F082FD2046FFF72FFD0028EDD0B6E738
:10AFA0007FC9010804ED00E02DE9FF41044601914D
:10AFB00020B940F291515248F7F7FEF9236C23B1C2
:10AFC00040F295514E48F7F7F7F901F081F830B9A2
:10AFD000019B23B140F29A514948F7F7EDF900255A
:10AFE0002F462E46DFF81C81FFF7F4FAA36BE3B17E
:10AFF000013BA363236813B901F06CF9A0602369D6
:10B0000063B104F1100000F017FF38B14FF0805227
:10B010003C4B1A60BFF34F8FBFF36F8FFFF7FAFA05
:10B020000125284604B0BDE8F081019B4BB925B14C
:10B0300040F2E1513248F7F7BFF9FFF7EBFA00258C
:10B04000EFE717B902A800F037FFFFF7E3FA00F0C7
:10B050007FFCFFF7BFFA94F84430FF2B08BF84F859
:10B06000446094F84530FF2B08BF84F84560FFF733
:10B07000D1FA01A902A800F02BFF40BB2046FFF740
:10B08000BBFCF0B123683BB9FFF7A4FAA06801F05C
:10B090002FF80546FFF7BEFA019904F1240000F0ED
:10B0A00091FE2046FFF7FAFC00F0F6FC38B94FF0AD
:10B0B0008053C8F80030BFF34F8FBFF36F8F012765
:10B0C00092E72046FFF7EAFC00F0E6FCF7E72046AF
:10B0D000FFF7E4FC00F0E0FC2046FFF78DFC0028C1
:10B0E000EDD0002D9DD0FFF775FA616A19B1236B81
:10B0F0001968C1F10501A06801F098F89DE700BF4B
:10B100007FC9010804ED00E02DE9F04385B00F464A
:10B110000192044620B94FF4CD614248F7F74CF94B
:10B1200037B9236C23B140F26C613E48F7F744F91C
:10B1300000F0CEFF30B9019B23B140F27161394874
:10B14000F7F73AF90026B046DFF8DC90FFF742FA4D
:10B15000A36BD3B139462046E568FFF78BFC636AE1
:10B16000E56063B104F1240000F066FE38B14FF0F1
:10B1700080522D4B1A60BFF34F8FBFF36F8FFFF7D5
:10B1800049FA012005B0BDE8F083019D1DB9FFF724
:10B1900041FA0020F6E716B902A800F08DFEFFF78D
:10B1A00039FA00F0D5FBFFF715FA94F84430FF2B7D
:10B1B00008BF84F8448094F84530FF2B08BF84F81A
:10B1C0004580FFF727FA01A902A800F081FEF0B937
:10B1D0002046FFF711FCA0B1019904F1240000F012
:10B1E000F1FD2046FFF75AFC00F056FC38B94FF04D
:10B1F0008053C9F80030BFF34F8FBFF36F8F012624
:10B20000A4E72046FFF74AFC00F046FCF7E720469B
:10B21000FFF744FC00F040FC2046FFF7EDFB002860
:10B22000EDD0B6E77FC9010804ED00E02DE9F84351
:10B2300089469046054620B940F2FB612048F7F761
:10B24000BBF8B9F1000F06D12B6C23B140F2FC61C1
:10B250001B48F7F7B1F8FFF797FAEFF311874FF0B4
:10B26000500383F31188BFF36F8FBFF34F8FAC6B25
:10B270001CB395F84460494676B22846FFF7FAFBBE
:10B28000013C731CAC6313D12B690BB901200BE09B
:10B2900005F1100000F0D0FD0028F7D0B8F1000F44
:10B2A000F4D00120C8F8000087F31188BDE8F883C6
:10B2B000013676B285F84460E8E72046F4E700BF3F
:10B2C0007FC9010810B5044620B940F28A710548CB
:10B2D000F7F772F8FFF77EF9A46BFFF79BF92046AA
:10B2E00010BD00BF7FC9010838B5054620B940F23E
:10B2F000A4710648F7F760F8FFF76CF9A86BEC6BE0
:10B30000241AFFF787F9204638BD00BF7FC901081E
:10B31000002330B5064A52F8335002EBC3041DB97E
:10B3200042F83310606030BD0133052BF3D1FAE7EA
:10B33000DC550020002310B5074A02EBC3014C681E
:10B34000844204D1002042F83300486010BD01332C
:10B35000052BF2D1FAE700BFDC55002010B50446FA
:10B3600020B94FF4F8610548F7F726F82046FFF7B3
:10B37000E1FF2046BDE81040FFF7F8BA7FC9010899
:10B3800070B504460D461646FFF724F994F844308C
:10B39000FF2B04BF002384F8443094F84530FF2B82
:10B3A00004BF002384F84530FFF734F9A36B2BB9B1
:10B3B0003246294604F1240000F01EFD2046BDE877
:10B3C0007040FFF76BBB0000064A13681968064B14
:10B3D00019B94FF0FF321A6070471268D268D2680C
:10B3E0005268F8E7CC4E00207C4F002010B5044690
:10B3F00020B940F2F2610848F6F7DEFF6269074BB8
:10B400009A4207D1A06A064B984203D0B0FA80F066
:10B41000400910BD0020FCE7CBC901089C4F00206B
:10B42000844F0020F8B51B4B1B4E1C680546306846
:10B430000F46043001F0A5FA334640B901203168C7
:10B44000164EC96A3268884022EA000232606A1CDD
:10B4500007D137B1196812480431BDE8F84001F04E
:10B460006DBA1A686419546007D30E4A10681968D7
:10B47000BDE8F840043101F06DBA0B4A1068196854
:10B48000043101F067FA094B1A68A24288BF1C60B8
:10B49000F8BD00BFC44F0020C84E00204C4F002014
:10B4A0009C4F0020D04E0020CC4E00207C4F00202E
:10B4B00080B5DFF86480144F144C154E236863B9CF
:10B4C000144B1B68012BF8D94FF08053C8F800309B
:10B4D000BFF34F8FBFF36F8FEEE7FFF77BF8FB688B
:10B4E000DD68281D01F04DFA3368013B33602368A5
:10B4F000013B2360FFF78EF8286BFFF737FA2846E9
:10B50000FFF734FADAE700BFB04F00203C4F0020CD
:10B51000384F0020D44E002004ED00E02DE9F84F14
:10B520004FEA820A804650460D4699460B9EFFF729
:10B530008BF90746002800F0AB805C20FFF784F908
:10B540000446002800F0A180076325B94FF4587124
:10B550005648F6F731FF5246A521206B0CF037FD17
:10B56000236BAAF1040A9A442AF0070A6B1E04F11D
:10B5700034020F3513F8011F02F8011B197809B1C5
:10B58000AB42F7D10A9D4FF0000B042D28BF0425D4
:10B59000271DE562C4E9135B384684F843B001F027
:10B5A000CAF9C5F1050504F1180001F0C4F9C4F8A1
:10B5B00054B02461A561646284F858B04A4641469B
:10B5C0005046FEF7E1FF206006B13460FFF702F855
:10B5D000374B384E1A68DFF8188101321A6032682A
:10B5E000002A58D134601B68012B25D1324801F064
:10B5F00097F9324801F094F9314801F091F9DFF8F8
:10B60000F490304801F08CF92F4D304801F088F962
:10B61000484601F085F9284601F082F92C4801F0EE
:10B620007FF92C4801F07CF92B4801F079F92B4B7C
:10B63000C3F800902A4B1D6001252A4A2A49136845
:10B64000086801331360E26A636405FA02F3034396
:10B6500014200B60184B394600FB023001F06EF9E4
:10B66000FEF7D8FFD8F8003063B13368DA6AE36ACE
:10B670009A4207D24FF080521C4B1A60BFF34F8F93
:10B68000BFF36F8F2846BDE8F88F3846FFF76EF995
:10B690004FF0FF35F6E7D8F80030002BCCD13368F7
:10B6A000DA6AE36A9A4298BF3460C5E7CBC90108F9
:10B6B000384F0020C84E0020D44E0020E84E002015
:10B6C000FC4E0020104F0020644F0020244F00202B
:10B6D000844F0020B04F00209C4F0020CC4E002013
:10B6E000D04E0020484F00204C4F002004ED00E0D9
:10B6F000984F0020504F002070B50446284DFEF7AB
:10B7000069FF04B92C68261D304601F03AF960B98A
:10B710001421E06A234B41435B5833B9012222498B
:10B7200082400B6823EA02030B60A36A1BB104F199
:10B73000180001F026F91D4A1368013313602B68C5
:10B74000A34220D131461A4801F0F8F8194A13688B
:10B7500001331360FEF75EFF174B1B6893B12B6834
:10B76000A3420FD1154B1B6823B140F2B6411448D8
:10B77000F6F722FE4FF08052124B1A60BFF34F8F44
:10B78000BFF36F8F70BD104A206B1368013B1360CD
:10B79000FFF7ECF82046FFF7E9F8FFF715FED9E7C9
:10B7A000C84E0020D44E00204C4F0020484F0020AF
:10B7B000B04F00203C4F0020984F0020444F002005
:10B7C000CBC9010804ED00E0384F0020F8B505466C
:10B7D00020B940F24C511748F6F7EEFD164B1B68A6
:10B7E000AB4220D0FEF7F6FE144B6C691F68144B79
:10B7F0001E68FEF70FFFBC4217D0B44215D0114BA4
:10B800009C4208D1AB6A83B995F85830012B0CBF24
:10B8100002200320F8BD0C4B9C4208D0002C0CBF2A
:10B8200004200120F6E70020F4E70220F2E70420DC
:10B83000F0E700BFCBC90108C84E0020CC4E002065
:10B84000D04E00209C4F0020B04F002070B5044621
:10B8500020B940F21C711948F6F7AEFD184D2B685F
:10B86000A34229D044B3FEF7B5FE2046FFF7BEFD44
:10B87000F0B1261D304601F084F801231149E26A37
:10B8800008689340034314200B600F4B314600FBC4
:10B89000023001F053F82B68E26ADB6A9A4207D360
:10B8A0004FF08052094B1A60BFF34F8FBFF36F8F79
:10B8B000BDE87040FEF7AEBE70BD00BFCBC9010849
:10B8C000C84E00204C4F0020D44E002004ED00E074
:10B8D00013B50024174B00940193502223461649B8
:10B8E0001648FFF71BFE012818D100F091FE012831
:10B8F00014D14FF0500383F31188BFF36F8FBFF360
:10B900004F8F4FF0FF320E4B1A600E4B18600E4BEC
:10B910001C6002B0BDE81040FEF7DCBE013007D16C
:10B9200040F60401094802B0BDE81040F6F744BDF6
:10B9300002B010BD784F002017CA0108B1B400084A
:10B940007C4F0020984F0020C44F0020CBC9010835
:10B95000024A136801331360704700BF444F002050
:10B96000014B1868704700BFC44F0020014B186896
:10B97000704700BF384F00202DE9F84F3A4B1B6845
:10B98000002B6AD1394B1C6801341C609CB9384DBE
:10B990002B681B6823B140F662213648F6F70CFD90
:10B9A000354B2A68196829601A60344A13680133D4
:10B9B0001360FFF709FD324D4FF0000B2B68314F3C
:10B9C000A34211D93A68304BD16A14224A439A589B
:10B9D000022A28BF4FF0010B2C4A1268002A0CBF24
:10B9E00058460120BDE8F88FDFF884A0DFF8A49066
:10B9F000DAF8002012681AB94FF0FF322A60E1E746
:10BA0000DAF80020D268D66871688C4201D22960C9
:10BA1000D8E706F10408404600F0B3FFB16A19B157
:10BA200006F1180000F0ADFF01224FF0140CF06A8F
:10BA3000D9F8003002FA00F11943134BC9F800108D
:10BA40000CFB0030414600F079FF3868F16AC26AA9
:10BA5000914228BF4FF0010BCAE70D4A4FF0000B8F
:10BA6000136801331360B7E7444F0020C44F002030
:10BA7000CC4E0020CBC90108D04E0020804F0020C2
:10BA80007C4F0020C84E0020D44E0020C84F00201C
:10BA9000404F00204C4F00202DE9F8432E4C2368E6
:10BAA00023B940F668012D48F6F786FCFEF792FDB3
:10BAB0002368013B236024682CB10024FEF7AAFD13
:10BAC0002046BDE8F883264B1B68002BF5D0254D9A
:10BAD000254EDFF8A8801FE0EB680127DC6804F141
:10BAE000040904F1180000F04CFF484600F049FF3B
:10BAF0001420E26A316807FA02F30B4300FB02806C
:10BB00004946336000F01AFF184BE26A1B68DB6A93
:10BB10009A4201D3164B1F602B68002BDCD10CB16D
:10BB2000FFF752FC134D2C6844B10127104EFFF76C
:10BB300023FF00B13760013CF9D12C600C4B1B682E
:10BB4000002BBAD04FF080520B4B1A60BFF34F8FCF
:10BB5000BFF36F8F0124B1E7444F0020CBC9010828
:10BB6000384F0020844F00204C4F0020C84E00204A
:10BB7000C84F0020404F002004ED00E0D44E0020CC
:10BB800038B50C46054620B940F2CA411848F6F7C8
:10BB900013FC24B940F2CB411548F6F70DFC154BC8
:10BBA0001B6823B140F2CC411148F6F705FCFFF7C2
:10BBB000CFFE114B2A68186814192CBF01210021EF
:10BBC00082422C600CD961B9FFF766FF38B94FF09B
:10BBD00080520A4B1A60BFF34F8FBFF36F8F38BD8F
:10BBE00009B9A042F0D20021201AFFF71BFCEBE7B5
:10BBF000CBC90108444F0020C44F002004ED00E0F1
:10BC000010B5044640B94FF080520D4B1A60BFF397
:10BC10004F8FBFF36F8F10BD0A4B1B6823B14FF4DA
:10BC2000A4610948F6F7C8FBFFF792FE0021204601
:10BC3000FFF7F8FBFFF730FF0028E4D0EBE700BF89
:10BC400004ED00E0444F0020CBC90108224B70B541
:10BC50001A68224B12B101221A6070BD204E1A6080
:10BC600033681B6B1A68B2F1A53F0BD15A68B2F169
:10BC7000A53F07D19A68B2F1A53F03D1DB68B3F1C4
:10BC8000A53F04D0306831683431F6F765FB154BB9
:10BC90001C68B4FA84F41423E4B2C4F11F046343AF
:10BCA000114DEB5823B940F688311048F6F784FB64
:10BCB000142202FB04F3E9184868083340682B4457
:10BCC000984202FB045408BF4368486008BF4B60B9
:10BCD0006368DB683360C0E7444F0020C84F002032
:10BCE000C84E00204C4F0020D44E0020CBC9010884
:10BCF00070B504462A4EFEF76DFC04B93468251D64
:10BD0000284600F03EFE60B91421E06A254B41430D
:10BD10005B5833B90122244982400B6823EA0203AD
:10BD20000B60A36A1BB104F1180000F02AFE29463B
:10BD30001E4800F003FE94F858301D4D012B04BF3F
:10BD4000002384F85830FEF765FC2A682AB1FEF714
:10BD500041FCFFF739FBFEF75DFC3368A34211D1CC
:10BD60002B6883B1134B1B6823B14FF4D961124880
:10BD7000F6F722FB4FF08052104B1A60BFF34F8F43
:10BD8000BFF36F8F70BD094A11680D4A1268914266
:10BD900001D13360F6E7BDE87040FFF757BF00BF41
:10BDA000C84E0020D44E00204C4F00209C4F002055
:10BDB000984F0020444F0020CBC9010804ED00E05B
:10BDC000384F002038B50D46044620B940F69F3163
:10BDD0000748F6F7F1FA074B20461968183100F0CA
:10BDE000B9FD2846BDE838400121FFF71BBB00BF65
:10BDF000CBC90108C84E002070B50E461446054652
:10BE000020B940F6CA310A48F6F7D6FA094B284657
:10BE10001968183100F092FD002C214608BF304609
:10BE2000BDE8704018BF4FF0FF30FFF7FBBA00BF0E
:10BE3000CBC90108C84E002038B5C368DC6824B9F6
:10BE400040F6FA311548F6F7B7FA04F11805284616
:10BE500000F097FD124B1B68E3B9251D284600F042
:10BE600090FD01230F49E26A0868934003431420C0
:10BE70000B6029460C4B00FB023000F05FFD0B4BC2
:10BE8000E26A1B68DB6A9A4285BF0120084B0020EA
:10BE9000186038BD29460748EFE700BFCBC9010845
:10BEA000444F00204C4F0020D44E0020C84E0020AC
:10BEB000C84F0020844F0020034B1B680360034BD6
:10BEC0001B684360704700BF804F0020C44F0020B4
:10BED00070B50C46054620B940F665411448F6F7A2
:10BEE0006BFA24B940F666411148F6F765FAFEF799
:10BEF00071FB104B1A682368591C0FD00E482E682E
:10BF000000686968864201D091420ED9521A934264
:10BF100009D99B1A23602846FFF7CEFF0024FEF7BD
:10BF200079FB204670BD002323600124F7E700BFA2
:10BF3000CBC90108C44F0020804F00200122014BD3
:10BF40001A607047C84F002070B50C46164605466B
:10BF500008B91B4A156805F134026260EA6A052BCC
:10BF600022612A6B2560E2616A6CA260EA6C626100
:10BF70004FF00002A2611BD011490968A9420BD100
:10BF80002273D6B1296B0A46531A12F8010BA52861
:10BF9000FAD09B08238470BD032B2373F1D1FFF7E4
:10BFA000D7FCAB6A0BB102232373FFF775FDE8E7FB
:10BFB0002846FFF70BFC2073E3E72684EBE700BF7E
:10BFC000C84E00202DE9F84F0D6881460C46924678
:10BFD0001DB300254FF0240B4B6801F108075B6887
:10BFE000BB424B6004BFCB684B604B68D3F80C80FE
:10BFF00063680BFB05915B6801229F42636008BF89
:10C00000E36805F1010508BF63606368DE685346B5
:10C010003046FFF799FFB045EAD12846BDE8F88FD2
:10C020002DE9F84305461746FFF792FC1F4B1B68A6
:10C030008B4238D84FF0000824264446DFF8809021
:10C0400009EB080106FB04500122FFF7BBFFA8F132
:10C05000140818F1640F0444F2D1154B0222196838
:10C0600006FB0450FFF7AEFF124B0444196802228E
:10C0700006FB0450FFF7A6FF044404220E4906FB0A
:10C080000450FFF79FFF044406FB045003220B49B2
:10C09000FFF798FF04440FB100233B60FFF7FCFC5F
:10C0A0002046BDE8F8830024F8E700BF384F0020A1
:10C0B000CC4E0020D04E0020B04F00209C4F0020DE
:10C0C000244F0020014B1868704700BFC84E002065
:10C0D000054B1B6833B1054B1B68002B0CBF0220BE
:10C0E0000020704701207047984F0020444F0020E7
:10C0F0002DE9F0410446002836D0234AC36A11686E
:10C100001746C96A8B4237D2142682691F4D002A0E
:10C11000A8BF3A6806FB0353A2BFD26AC2F1050268
:10C12000826142699A4221D100F10408404600F040
:10C1300028FC174B48B9E06A4643AA592AB901219D
:10C140001A68814022EA01021A603A681968D26AC4
:10C15000E262012404FA02F0084318601420414608
:10C1600000FB025000F0EAFB204603E03B68DB6A7C
:10C17000C3620120BDE8F0811368C06CDC6AA04294
:10C180002CBF00200120F5E7C84E0020D44E00202F
:10C190004C4F0020F8B5044608B90020F8BD1F4BED
:10C1A0001B68834204D040F67A711D48F6F704F903
:10C1B000236D23B940F67B711948F6F7FDF8236D1E
:10C1C000E16AE26C013B91422365E6D0002BE4D1A9
:10C1D000251D284600F0D5FB124E134A50B91421F4
:10C1E000E76A794373582BB901201368B84023EAF2
:10C1F00000031360E36CC3F10501A161E362012454
:10C20000116804FA03F0084310601420294600FB6B
:10C21000036000F093FB2046C0E700BFC84E00203B
:10C22000CBC90108D44E00204C4F0020F8B50D4674
:10C230000446002845D0036D23B940F6C971214852
:10C24000F6F7BAF8E36C9D4238BF1D46E36AAB428D
:10C2500037D0236D012B34D11B4B1B68A34204D173
:10C2600040F6E4711748F6F7A7F81426A269E36AC6
:10C27000002AE562A4BFC5F10505A561134D6269F9
:10C2800006FB03539A421CD1271D384600F079FB68
:10C29000E26A0F4C40B95643AB592BB901212368D0
:10C2A000914023EA01032360012314202168934075
:10C2B0000B432360394600FB0250BDE8F84000F014
:10C2C0003DBBF8BDCBC90108C84E0020D44E0020AC
:10C2D0004C4F0020044B1A681AB119680A6D0132DC
:10C2E0000A651868704700BFC84E00202DE9F0416C
:10C2F0001E4C1E4680460F461546FEF76BF9236816
:10C3000093F85830022B14D0012123685A6D22EA89
:10C3100008025A65236883F8581056B13046FFF773
:10C3200081F84FF08052124B1A60BFF34F8FBFF36A
:10C330006F8FFEF76FF9FEF74DF915B123685B6D4E
:10C340002B602368002293F85830022B09BF012587
:10C3500000252368596D04BFB9435965236883F8E4
:10C360005820FEF757F92846BDE8F081C84E002056
:10C3700004ED00E0F8B50E4617461D46044620B908
:10C3800041F219212B48F6F717F8FEF723F90DB102
:10C39000636D2B60022394F8585084F85830EDB246
:10C3A000042F16D8DFE807F00A0307051100636DB4
:10C3B0001E43666502E0636D01336365012D11D094
:10C3C0000124FEF727F92046F8BD022DF1D1002403
:10C3D000F7E7636D0133F1D041F24A211548F5F7D3
:10C3E000EBFFEBE7261D304600F0CBFA1420124A93
:10C3F000E36A11689D400D431560104A314600FB09
:10C40000032000F09BFAA36A23B141F259210948A5
:10C41000F5F7D2FF0A4BE26A1B68DB6A9A42CFD972
:10C420004FF08052074B1A60BFF34F8FBFF36F8FEF
:10C43000C6E700BFCBC901084C4F0020D44E0020F6
:10C44000C84E002004ED00E02DE9F843DDF820801F
:10C450000E4691461D46044620B941F28C213548CE
:10C46000F5F7AAFFFEF790F9EFF311874FF05003AD
:10C4700083F31188BFF36F8FBFF34F8F0DB1636DDF
:10C480002B60022394F8585084F85830EDB2B9F17B
:10C49000040F16D8DFE809F00A0307051100636DE1
:10C4A0001E43666502E0636D01336365012D11D0A3
:10C4B000012087F31188BDE8F883022DF1D1002017
:10C4C000F7E7636D0133F1D041F2CF211948F5F759
:10C4D00073FFEBE7A36A23B141F2DA211548F5F7C0
:10C4E0006BFF154B1B6803BB251D284600F049FA5E
:10C4F00001231249E26A08689340034314200B6049
:10C5000029460F4B00FB023000F018FA0D4BE26A8F
:10C510001B68DB6A9A42CBD90123B8F1000F01D026
:10C52000C8F80030084A1360C2E704F11801074850
:10C53000EAE700BFCBC90108444F00204C4F002060
:10C54000D44E0020C84E0020C84F0020844F002049
:10C5500038B5054608B9084B1D680024FEF73AF8BF
:10C5600095F85830022B04BF85F858400124FEF797
:10C5700051F8204638BD00BFC84E0020F8B50F4C1A
:10C58000FEF728F82568ADB90D4F0E4E384600F07D
:10C59000C7F9304600F0C4F90B4B2A461F600B4B1D
:10C5A0000C210A201E60FEF7EFFA206010B1084946
:10C5B000FEF7AEFEBDE8F840FEF72CB800500020B4
:10C5C000D44F0020E84F0020CC4F0020D04F002057
:10C5D0001CCA0108914208B5416000610AD8D21A0C
:10C5E00083699A420DD2084B011D186800F0B2F918
:10C5F000002008BD9A4201D2994202D2011D034B8C
:10C60000F3E70120F5E700BFD04F0020CC4F00201A
:10C6100007B5FFF7B3FF0C4B1B6843B90B484FF44A
:10C620008971F5F7C9FE002003B05DF804FB084BE3
:10C63000C822019301230749009307480023FEF70E
:10C640006DFF0028EAD0EFE70050002021CA010862
:10C65000045000206ECA010875C700082DE9F0419A
:10C6600080462C200D4617461E46FEF7EDF8044680
:10C6700088B125B94FF4B6710848F5F79DFEFFF76C
:10C680007DFF069BC4F80080C4E9065726626362FA
:10C69000201D00F050F92046BDE8F08121CA0108B4
:10C6A0002DE9FF410D4690461F46064620B94FF43E
:10C6B000C3710F48F5F780FE0E4C206878B1052D48
:10C6C000CDE9015803960DDCFFF702FD0023022897
:10C6D0000CBF0A9A1A4601A92068FEF779FA04B03D
:10C6E000BDE8F08100233A4601A9FEF727FBF6E7F3
:10C6F00021CA0108005000202DE9F74300271A4DF8
:10C70000DFF86C802B681A6832B9184A1168136018
:10C71000296003B0BDE8F083DB68DC681E6804F1C3
:10C720000409484600F02DF9636A20469847E369FA
:10C73000012BE7D1A36933449E4206D26360246192
:10C740004946286800F006F9DCE7002300973246E6
:10C7500019462046FFF7A4FF0028D3D140F27231DA
:10C760004046F5F729FECDE7CC4F0020D04F002002
:10C7700021CA01082DE9F04F4FF00108624D89B040
:10C78000DFF898B1DBF80020136843B30024D368C6
:10C79000D3F80090FFF7DCF8FFF7E2F85B4B824636
:10C7A0001A681F4690425A4E1CD31860002C4CD079
:10C7B000584B1B681A68B2FA82F25209A9EB0A01B7
:10C7C0003068FEF7DDFDFFF767F998B94FF080524A
:10C7D000514B1A60BFF34F8FBFF36F8F0AE00124F4
:10C7E0009946D7E70393FFF787FF039BC3F800A0A1
:10C7F000FFF752F9002205A93068FEF743FB002835
:10C80000BED0059B002BF5DB079C636913B1201D8F
:10C8100000F0B7F8FFF7A4F83B688146984201D2D0
:10C82000FFF76AFF059BC7F80090092BE2D808FACA
:10C8300003F313F4047A57D113F0C70F33D19B06D7
:10C84000D8D52046FEF792F8D4E7814529D8FFF7DE
:10C8500023F9DBF80030DB68D3F80CB00BF10400EF
:10C8600000F08FF8DBF81C30012B15D1DBF8181025
:10C870004B46524649445846FFF7ACFE60B100941F
:10C8800023464A4621465846FFF70AFF20B94FF48F
:10C89000F4712846F5F790FDDBF8243058469847A8
:10C8A000A8E722468AE7A169069B4A461944204622
:10C8B000FFF790FE00289DD0636A20469847E36901
:10C8C000012B97D1A2690699CDF800A00A445346DE
:10C8D00051462046FFF7E4FE00288BD140F201319B
:10C8E0002846F5F769FD85E7069BA36123B94FF458
:10C8F00046712846F5F760FDA1694B464A46494412
:10C900002046FFF767FE75E721CA0108FC4F0020AB
:10C9100000500020D04F002004ED00E0CC4F00205C
:10C920004FF0FF3200F108034360C0E902230361C6
:10C9300000230360704700230361704743689A68CF
:10C940004B608A609A68516099600368086101339E
:10C95000036070470A6830B5531C0AD103695A68EE
:10C960004A6091608B60596003680861013303601D
:10C9700030BD00F108035C6825689542EFD8234676
:10C98000F9E70369D0E901128A6082685160596849
:10C99000814208BF5A60002202611A68013A1A6097
:10C9A00018687047021C18BF012200210148F8F7DF
:10C9B0004BBF00BF00040240F9F700BC38B5054684
:10C9C0000C460020FFF7EEFF45F08000FFF7F4FF74
:10C9D0002046FFF7F1FFBDE838400120FFF7E2BF36
:10C9E00008B50120F8F722FD0A20F8F71FFD0B20FB
:10C9F000F8F71CFD0720F8F719FD0520F8F716FDDC
:10CA0000BDE808400420F8F711BD0000204B70B5C8
:10CA10009D780446EDB958B902211E48F8F70EFF7B
:10CA200023461A460221BDE870401A48F8F73EBE78
:10CA3000012805D102211748F8F7FAFE2B46F0E746
:10CA4000022823D102460146BDE870401148F8F79C
:10CA50006BBE012D14D138B904210E48F8F7EEFE53
:10CA6000002304211A46DEE7012804D104210948E5
:10CA7000F8F7DEFEF4E7022808D102460421E3E7D6
:10CA80006A21BDE870400448F5F796BC70BD00BF50
:10CA9000085000200000024076CA010808B50020B6
:10CAA000FFF7B4FFF8F704FC0120FFF7AFFFF8F73A
:10CAB000FFFB0220FFF7AAFFBDE80840F8F7F8BB2C
:10CAC00008B500210120F9F7FBFA0120FFF76AFF02
:10CAD0000023094819461A46F8F7E8FDB521402019
:10CAE000FFF76CFFA0214120FFF768FFBDE8084079
:10CAF00000210120FFF762BF0004024010B5FFF7DC
:10CB00006FFF0120FFF74EFF00233A481A461946EF
:10CB1000394CF8F7CBFD00210120F9F7D1FA227842
:10CB20007AB1002306211A463248F8F7BFFD0621E4
:10CB30003048F8F77DFEF8F7BBFB19215820FFF7C6
:10CB40003DFFFFF7ABFFFFF7BBFF63785BB100234F
:10CB500004211A462948F8F7A9FD00230D211A4699
:10CB60002748F8F7A3FD002201212248F8F7DCFD51
:10CB700000220A211F48F8F7D7FD00220B211D488B
:10CB8000F8F7D2FD002207211A48F8F7CDFD002260
:10CB900005211848F8F7C8FD002204211548F8F7C8
:10CBA000C3FD0523022201211248F8F75DFC05238D
:10CBB00002220A210F48F8F757FC052302220B2115
:10CBC0000C48F8F751FC0523022207210948F8F721
:10CBD0004BFC0523022219460648F8F745FC094B91
:10CBE0001B782BB9BDE81040BE210748F5F7E4BB20
:10CBF00010BD00BF000402400850002000000240A9
:10CC0000000802400B50002076CA010882B0019053
:10CC100002AB33F8041D054A9B7811809370012202
:10CC2000034B1A7002B0FFF769BF00BF0850002025
:10CC30000B5000201A4B10B55B78D3B10128194C6A
:10CC400018D104211848F8F7F3FD0D211748F8F71B
:10CC5000F5FD23786BB1002304211A461248F8F73A
:10CC600025FD00230D211A461048F8F71FFD00236B
:10CC7000237010BD40B904210B48F8F7DFFD0D21EA
:10CC80000A48F8F7D5FDE4E7022204210648F8F740
:10CC90004BFD02220D210548F8F746FD0123E7E789
:10CCA00008500020D0000020000002400008024090
:10CCB00008B5FFF795FEFFF7F1FEFFF701FFF9F763
:10CCC00059FA012200211F48F8F72EFD0220FFF734
:10CCD000B1FF0220FFF79AFE022201211948F8F75E
:10CCE00023FD02220A211748F8F71EFD02220B211C
:10CCF0001448F8F719FD022207211248F8F714FD2D
:10CD0000022205210F48F8F70FFD022204210D48E9
:10CD1000F8F70AFD0C4B1B781BB9E2210B48F5F71D
:10CD20004BFB0B4B1B785BB1002306211A460548D1
:10CD3000F8F7BCFCBDE8084006210248F8F77EBDC4
:10CD400008BD00BF000402400B50002076CA010855
:10CD50000850002010B5064C022220460021F8F7AA
:10CD6000E3FC2046BDE8104002220121F8F7DCBCBC
:10CD700000140240014BDB68184700BF0C50002034
:10CD80000120704701B1096818B1806A431A5842FE
:10CD90005841704738B50C4B0546186800F031FB18
:10CDA00010B90023184638BD4FF47A7403686C43F9
:10CDB0001A68A242F6D000F01BFB0028F1D00368ED
:10CDC0001A689442F6E700BF0C50002010B50446E4
:10CDD00018B9D2210748F5F7EFFA074B5B68984777
:10CDE000D4E90623904271EB0304B4BF101A00206B
:10CDF00010BD00BFFCCA01080C5000202DE9F84905
:10CE00008846044610B10369012B03D1E721174876
:10CE1000F5F7D2FAD4E906BC5BEA0C0323D0D4E9D7
:10CE20000867BBEB06006CEB07010AF055FB0546F3
:10CE3000206901380AF036FB014628460AF03EFC1C
:10CE4000054640460AF02EFB29460AF083FB294698
:10CE50000AF076FA0AF06AFD321847F1000310462C
:10CE60001946C4E90601BDE8F88900BFFCCA0108FB
:10CE700041F65832A0F55223A3F61833934224D832
:10CE8000A0F55423A3F1F902622A1ED96FF454725B
:10CE90009A18C62A19D9A3F21353302B15D9104B5F
:10CEA000984214D903F6B833984212D903F5167391
:10CEB000984210D903F5167398420ED903F5E17321
:10CEC000984294BF0520062070470020704701203B
:10CED000704702207047032070470420704700BF4E
:10CEE000E8320D00F8B5054618B9F3212248F5F7E8
:10CEF00063FA224E306800F084FA00283BD0002DFF
:10CF000039D003681A79AA4231D11F7B00F070FA38
:10CF100020BB87B3062D03D940211748F5F74CFAFB
:10CF2000174B53F8354024BBFE211348F5F744FA5C
:10CF3000306800F066FA0646E8B17C4337683B7912
:10CF4000AB4204D121463846FFF758FF3C613046DA
:10CF500000F04EFA06460028F0D10CE003681A797A
:10CF6000AA42D3D11B7B002BD0D00137CEE70027BC
:10CF7000CCE7012CDCD1F8BDFCCA01080C50002024
:10CF8000C4CA010810B5074C206848B100F042FA45
:10CF900030B1206800F035FA00F02AFA0028FBD101
:10CFA00010BD00BF0C500020F8B5114C0646227E83
:10CFB0000F4622B94FF4B1710E48F5F7FDF920681C
:10CFC00010B900252846F8BD0B4B002E08BF1E46A1
:10CFD00000F017FA04460028F3D0256839462846A1
:10CFE000B0470028EED1204600F002FAF2E700BF79
:10CFF0000C500020FCCA010881CD00082DE9F04F3B
:10D00000394C9246227E91B08346894622B94FF42C
:10D01000C9713648F5F7D0F9206820B900242046B8
:10D0200011B0BDE8F08F324BB9F1000F08BF99463F
:10D0300000F0E7F980460028F0D00468237BDBB9D4
:10D040004FF0FF3600240027404600F0D1F980461B
:10D05000F8B9BAF1000F01D0CAF80060002EDED195
:10D06000012FDCD9791E3046FBF730FB10AB03EB08
:10D07000800050F8404CD2E7A3685B45E0DB00211C
:10D080002046C8470028DBD02046FFF79FFE064613
:10D09000D9E7D8F800502B7B002BD5D0AB685B4587
:10D0A000D2DB00212846C8470028CDD02846FFF70C
:10D0B0008DFE38B90F2F9FBF10AB03EB870343F8EA
:10D0C000405C01376CB186420AD8BDD1D4E908234F
:10D0D000D5E90801FBF7FDF8002818BF2C46B3E797
:10D0E00006462C46B0E700BF0C500020FCCA0108E1
:10D0F00081CD000800000000F8B50D46044620B9B7
:10D1000040F2E1111A48F5F757F9236923B94FF4B2
:10D11000F1711748F5F750F9164B5B6898470F46C1
:10D1200006462069C4E908670AF0BCF929460AF0F6
:10D1300011FA29460AF004F909F09CFD0AA3D3E983
:10D14000002309F019FF09F0D7FA0AF085F8321820
:10D1500047F1000319461046C4E90601BDE8F8404E
:10D16000FFF710BFAFF300800000000080842E4165
:10D17000FCCA01080C50002008B5FFF779FE00300A
:10D1800018BF012008BD00000A4B10B51B7E0446E5
:10D1900023B94FF407710848F5F70EF944B1237B22
:10D1A00033B1002320792373BDE81040FFF79ABE06
:10D1B00010BD00BF0C500020FCCA01080A4B10B57E
:10D1C0001B7E044623B94FF40A710848F5F7F4F8BA
:10D1D00044B1237B33B9012320792373BDE8104088
:10D1E000FFF780BE10BD00BF0C500020FCCA010834
:10D1F000F8B5144E0546337E23B94FF40D7112482D
:10D20000F5F7DAF8306808B90020F8BD002DFBD03A
:10D2100000F0F7F804460028F6D023689D420CD1B0
:10D220002F792846FFF7A6FD2146306800F000F967
:10D230003846FFF757FE0120E7E7204600F0D8F810
:10D24000E8E700BF0C500020FCCA01082DE9F843B4
:10D250002A4D07462B7E8846914623B940F2F911A4
:10D260002748F5F7A9F83846FFF786FF18B90024D4
:10D270002046BDE8F8833846FFF78CFD08B1FFF77C
:10D28000B7FF2B7E1BB976211D48F5F795F8AB68E3
:10D290003020984704460028E9D0302200210AF0C7
:10D2A00096FE3846FFF7E4FD0646207118B9EB6894
:10D2B00020469847DBE7062803D940211048F5F7B8
:10D2C0007BF8104B214603EBC60253F83630526808
:10D2D00023614FF47A73A2605F4300220023C4E904
:10D2E000062301232760C4E90A892373286800F014
:10D2F00069F82079FFF7F6FDBAE700BF0C5000206F
:10D30000FCCA0108C4CA010838B50A4C0546227E89
:10D3100022B94FF41C710848F5F74EF823682BB179
:10D32000064C29462046FFF73FFE00B938BDFFF7FF
:10D3300021FDF6E70C500020FCCA010885CD00084D
:10D34000014B187E704700BF0C50002084B070B5B0
:10D3500004AC84E80F00104C237ECBB9251D04AE2D
:10D360000FCE0FC533682B600BB90C4B636123697B
:10D370000BB90A4B2361E3680BB1A3681BB9084BD7
:10D38000E360084BA36000F00FF8012320602376D0
:10D39000BDE8704004B070470C5000202D84000898
:10D3A000197F0108097F010810B50820FBF7DEF896
:10D3B0000446FEF7CDFA0023C4E90034FEF76CFB07
:10D3C000204610BD70B505460C200E46FBF7CEF882
:10D3D000044660B10660FEF7BBFA002363606B6829
:10D3E000A3601C6004346C60FEF756FB012070BD26
:10D3F00010B50446FEF7ACFA6468FEF74DFB204614
:10D4000010BD10B50446FEF7A3FA2468FEF744FBEE
:10D41000204610BD10B50446FEF79AFA2368002492
:10D420001BB9FEF739FB204610BD01345B68F7E7F6
:10D4300038B50C460546FEF78BFAD4E901324BB1FC
:10D440009A60A2681360FEF727FB2046BDE83840CB
:10D45000FBF776B86A60F4E700BF70472DE9F04744
:10D46000344D354EEB6A8AB09847D5E91047337989
:10D47000A8460C20002B54D0B84740F00301C9B295
:10D480000C20A047B3682D4898474FF0040A4CF28F
:10D49000503300254FF00109CDE9003AD8F8183093
:10D4A000274A1E4648462B46CDE90859CDE9065580
:10D4B000CDE90455CDE902592249B0473321052071
:10D4C000A04750460321A04749461220A047514695
:10D4D0002120A0470C20B84720210C20A047AA21DA
:10D4E0001F20A0471848FBF749FDD8F80C30174813
:10D4F00098472846FBF73CFD3020B84700F09F01D5
:10D500003020A0472720B84731212720A0475421A9
:10D510002820A0473D21292023460AB0BDE8F04736
:10D520001847B84700F0FC010C20A047B368084832
:10D53000AAE700BF3CC701083C50002025CC0108E9
:10D54000A086010090D0030019D90008F01FCB334A
:10D5500051CC010810B50478A4F1090009F0A6FF28
:10D5600009F088FB0022064B09F0DCFB09F0C4F847
:10D5700009F072FE0134013004EB400080B210BDAE
:10D580000000B03F08B5FEF79DFD002303221946B9
:10D59000FEF7F0FEBDE808400020FEF7D9BF00000E
:10D5A0002DE9F0430126324FDFF8D8908BB0FB6AAB
:10D5B00089F83460984700254FF2244324222D49EE
:10D5C000CDE90032BC694FF400422B463046099643
:10D5D000CDE90755CDE90555CDE903650295A0478D
:10D5E0002548FBF7CBFCFB68244898473C6C33216B
:10D5F0000520A04703210420A04731461220A04760
:10D60000D7F844800C20C04700F0FC010C20A04754
:10D61000AA211F20A0473046C04700F0E70130464E
:10D62000A0470220FBF7A4FC3020C04700F09F0178
:10D6300041F020013020A0472720C04700F008011A
:10D6400041F032012720A04754212820A04776210D
:10D650002920A04796212A20A047D9F80830084859
:10D66000984728467B6B0BB0BDE8F043184700BFD6
:10D670003CC701082C8B020055D50008E034C133AB
:10D680000DCD01083C50002070B5104C05462378A4
:10D69000264648B9CBB1FBF737F90D4B0D489B68CF
:10D6A0002570BDE8704018477BB941F28830FBF720
:10D6B00057F920B940F266310748F4F77DFE01239F
:10D6C0003370034B05489B68EBE770BD3450002076
:10D6D0003C50002095CC0108ADCC0108F5CC0108E8
:10D6E0002DE9F0410546D0B918211248F4F764FE3F
:10D6F000DFF844800820D8F80C309847044680B101
:10D700000026466006600571D8F80C302846984718
:10D71000206050B9D8F810302046984701E0FF2823
:10D72000E6D100242046BDE8F0812A4631460AF0C1
:10D730004EFCF7E7ADCC01083C50002070B5094C19
:10D74000054623691BB92E210748F4F735FE2868E2
:10D75000236910B1984700232B6023692846BDE850
:10D76000704018473C500020ADCC01082DE9F04135
:10D77000474D8AB0EB6A0027804698474FF47A738A
:10D780000126CDE907730823CDE90236414B4CF25F
:10D7900050320E21EC69009330463F4BCDE90577BE
:10D7A00004970197A0473D48FBF7E8FBEB683C482E
:10D7B00098472C6CE8210520A04703210420A047AE
:10D7C0006D6C0C20A84700F0FC010C20A0473046EF
:10D7D000A84700F0E7013046A0473846FBF7C8FBF2
:10D7E0003020A84700F09F013020A047B8F1020F79
:10D7F00005D3B8F1030F08D9B8F1040F38D04FF4AE
:10D8000022712848F4F7D8FD0CE03046A84700F014
:10D81000E70141F010013046A0472720A8473721F3
:10D820002720A0471A20A84740F00101C9B21A20BA
:10D83000A04755212820A04755212920A047552140
:10D840002A20A04755212B20A04754212C20A04757
:10D850003D212D20A047B8F1020F0DD0B8F1030FE4
:10D8600011D0114B11489B680AB0BDE8F041184730
:10D870002720A8473521D3E754212E20A047CD21CA
:10D880002F20A047EDE754212E20A0473D21F7E7A8
:10D890003CC70108A086010090D0030019D90008F8
:10D8A000F01FCB33ADCC01083C50002076CC0108F2
:10D8B0002DE9F04100240E46074621464FF012089C
:10D8C000A64201DA012016E00C2C09D006DDA4F1F5
:10D8D0000C0292FBF8F308FB13230BB1A64218D1FC
:10D8E0003B1913F8022C13F8015C631E994245EAB8
:10D8F000022502DB0020BDE8F081A21E521A92B27E
:10D90000394400200CF0F0FFC04380B28542F1D1D1
:10D9100021460134D4E700001129F8B504464ED958
:10D920000378542B30D00C25264E77190022791B12
:10D9300020460DF00BF8002841D1023D04F103040C
:10D94000F4D10C211F48FFF7B3FF002837D03478FB
:10D95000A4F1090009F0AAFD09F08CF900221A4B84
:10D9600009F0E0F908F0C8FE09F076FC0134013056
:10D9700004EB40040C20A4B244436207C4F3CF007C
:10D9800001D5013080B2F8BD4378CD2B12D10C21E6
:10D990000230FFF78DFF0028F5D01022A378581D24
:10D9A0000A3B93FBF2F21B0700EB420080B2EAD085
:10D9B0000230E7E73D2B02D180780330E3E7002017
:10D9C000E1E700BF285000200000B03F2DE9F04102
:10D9D00000240E46074621464FF07608A64201DA9B
:10D9E000012015E00A2C06DDA4F10A0292FBF8F3EF
:10D9F00008FB13230BB1A64218D13B1913F8022CD4
:10DA000013F8015C631E994245EA022502DB0020FF
:10DA1000BDE8F081A21E521A92B2394400200CF0E7
:10DA200063FFC04380B28542F1D121460134D5E77E
:10DA30002DE9F04F8BB0642303AA4FF0FF31002093
:10DA4000FEF754FC012856D1039BDD0723D50024A3
:10DA5000994D0020FFF718FEFCF7BCFDAB68974816
:10DA60009847FCF7D7FD214623462246E86A85F809
:10DA70003440FDF7ADF82046FEF73AF94FF47A71DD
:10DA8000E86AFDF791FA0028D5D140F283318C483D
:10DA9000F4F792FCCFE79C0709D5FFF7F5FDFFF7F8
:10DAA00071FDFFF77DFD844B86489B689847039B7B
:10DAB000590711D50120FFF7E7FDFFF763FD0223AA
:10DAC0007D4C84F83430FFF7C9FC7F4B00205B6B42
:10DAD0009847A3687D489847039B1A070BD50120F8
:10DAE000FFF7D2FDFFF74EFD0022734B784883F815
:10DAF00034209B689847774B1F7827B96E4B764840
:10DB00009B68984797E7754B002204A91868FDF7B2
:10DB1000B9F9012840F00081049D674C6879FFF74E
:10DB200025FEFAF77DFF6B79042B40F09180287970
:10DB3000013809F08DF80022694B09F0F3F8002252
:10DB40004FF0804308F038FF09F086FBFF2882463B
:10DB500019D90146A3686348984700272846FFF76C
:10DB6000EDFD94F83410022940F09380FFF776FC25
:10DB7000554B00205B6B9847636A002B3FF45BAF0B
:10DB80003846984757E7E3689847064630B9A36890
:10DB900055489847236930469847DEE7804695F810
:10DBA00004902A6802EB090BB9F1000FABEB0900F6
:10DBB0003ADC2A7929684D48FAF7B2FC52463146D8
:10DBC0004B48FAF7ADFCA3684A4898474FF0000964
:10DBD000DFF840B12A79A368914531DB4648984780
:10DBE000394B30469B6A5FFA8AF198472369304681
:10DBF0009847FAF725FF4FF47A7207A9FDF742F923
:10DC000038B93E48A368984740F203312C48F4F7EE
:10DC1000D3FB9DF81C10A368012931D138489847DF
:10DC200007A8FAF7CBFE99E709F1FF335A424146BC
:10DC30005A410CF06BFEA9F1020908F10308B3E7A1
:10DC40002A68584612F80910984709F10109C1E7F6
:10DC5000A3682C4898470026DFF8B8902A79A36873
:10DC6000964207DB24489847174B297928689B6A16
:10DC70009847BEE72A684846915D98470136EDE728
:10DC8000022903D1204898470027C9E71F48984731
:10DC9000FAE7012902D1FFF783FC6DE719B90A4BB6
:10DCA000DB6A984768E7A3681948984740F2B521AE
:10DCB0000348F4F781FB5FE73C50002026CD0108C4
:10DCC000ADCC01083DCD01083CC701085DCD010880
:10DCD00080CD010834500020A7CD01083850002025
:10DCE0000000F83FBFCD0108F3CD010819CE0108AF
:10DCF0001FCE010825CE01080AE4010853CE010811
:10DD000078CE01083FCE010889CE01089DCE0108DA
:10DD1000BFCE010839CE0108FAF792FE002207A90A
:10DD2000FDF7B0F800283FF486AE864D9DF81C1034
:10DD300095F83430AA4613B9AB68834898479DF8E4
:10DD40001C60032E40F0F08095F83490089FB9F1E4
:10DD5000010F56D1B888A0F10C03F32B00F2A88074
:10DD6000C0B2FFF7BDFCBA8880F805900446396858
:10DD700000680AF008F9AB6874489847B7F90600DC
:10DD8000BB88E080227961790090AE687048B04726
:10DD900063795A1E012A00F2AE8021792068FFF7CC
:10DDA00087FD0646AB68002800F0B38069489847B5
:10DDB0000027DFF8C8912279DAF808309742C0F2DC
:10DDC000AD8065489847002E6FD0286B0594FDF70D
:10DDD0008BFA024638B906A9286BFDF753F810B143
:10DDE0000698FFF7ABFC002305A91A46286BFCF741
:10DDF000EFFE00285CD140F226315848F4F7DCFAF7
:10DE000056E0B9F1020F53D13868B9880278542A24
:10DE100030D14278CD2A16D1A1F10E02F32A47D88B
:10DE2000881EC0B2FFF75CFC0446002840D0BA88C8
:10DE3000396880F80590023A023100680AF0A3F8C8
:10DE4000AB68474899E73D2A14D1A1F10E02F32AA5
:10DE50002ED8881EC0B2FFF743FC044640B3BA88F0
:10DE600039684671023A023100680AF08CF8AB68F2
:10DE70003C4882E7C9B2FFF74FFDC6000C2096FB75
:10DE8000F0F6F6B20B2E13D93046FFF729FC044604
:10DE900070B104234FF00009D0F80080D7F800B02B
:10DEA00043714EB923794B4522D02046FFF746FCFB
:10DEB00007A8FAF783FDBEE5012E10D0414658466B
:10DEC00000220CF043FD023E0BF1030B08F10208A7
:10DED00009F102090028E4D04FF00009E2E73246D8
:10DEE000414658460CF032FD09F101090026F1E7E0
:10DEF000AB681D4841E7042B3FF44FAF032B04D11F
:10DF000021792068FFF762FD4BE73C211348F4F7C5
:10DF100053FAAB6815489847002649E722684846F7
:10DF2000D15D9847013746E7042EAB6802D110480F
:10DF30009847BDE7052E01D10E48F9E731460E4856
:10DF40009847B5E73C500020DECE01080DCF010810
:10DF5000FECF01089ECF010809E40108ADCC0108FD
:10DF600032CF010856CF01087ACF0108A8CF0108A7
:10DF7000B9CF0108CCCF0108DDCF0108E0C6010808
:10DF800004289ABF014B185C3F2070474ECB010814
:10DF900004289ABF014B185C3F20704753CB0108FF
:10DFA000014B1871704700BF3C50002082B0F0B5A3
:10DFB00085B002AF87E803000AA90E464A4C81E803
:10DFC0000C0004F108050FCE0FC596E80F0085E898
:10DFD0000F0097E80300002384F83430236984E8B5
:10DFE0000300013B033304D94FF48C613F48F4F73D
:10DFF000E3F9E368013B033304D940F263413B4852
:10E00000F4F7DAF9A368013B033384BF384BA3600C
:10E01000A369013B033384BF364BA3616369013BB2
:10E02000033384BF334B6361236A013B033384BFF3
:10E03000304B2362E369013B033384BF2D4BE36123
:10E04000236813B9A3682C489847FAF7F9FC20B95C
:10E05000A3682A48984700203DE0FAF7F1FC013018
:10E06000F6D0002204210120FCF78EFD244B18601D
:10E0700020B940F283411D48F4F79EF903220021A4
:10E080000120FCF781FDE06220B940F2864117488B
:10E09000F4F792F9002204210520FCF775FD2063B6
:10E0A00020B940F289411148F4F786F9154B4FF435
:10E0B0009672019323681449009314480123FDF7D5
:10E0C0002DFA012805460BD1014600230322A06A40
:10E0D000FEF750F9284605B0BDE8F04002B07047A1
:10E0E000A3680B48B6E700BF3C500020ADCC010848
:10E0F0002D84000859D40008ACCB0108D7CB010807
:10E100003850002064500020FFCB010831DA0008AD
:10E1100005CC010810B5134CA36A23B940F2A24103
:10E120001148F4F749F9012100230322A06AFEF700
:10E1300021F90E48A368984742F21071E06AFCF793
:10E1400033FF20B940F2AA410748F4F735F900231C
:10E15000E06A1A461946FCF73BFDA3680448BDE88F
:10E16000104018473C500020ADCC010858CB0108A6
:10E1700075CB010838B5154C0546A36A23B940F2A2
:10E18000C2411348F4F718F9012D0DD100230322E1
:10E190000221A06AFEF7EEF8A3680E489847A06A2D
:10E1A000FDF754FB012038BD022D03D100230322CB
:10E1B0000421EEE71DB92B4603220821E9E70448B4
:10E1C00040F2CA41F4F7F8F80020ECE73C50002098
:10E1D000ADCC010891CB0108002307B502A941F895
:10E1E000043D044B0246186BFCF74CFE019803B04B
:10E1F0005DF804FB3C50002070B50446044E451801
:10E2000014F8011B3046FAF715F9AC42F8D170BD8D
:10E2100037D0010870B515460022C0E9011502701B
:10E22000C0E90332C0E90522C0E907224262DDE904
:10E230000412044600F11C0604F05EF938B92946C0
:10E240000748FAF7F7F82B210648F4F7B5F8DDE9A7
:10E2500004233146204604F03CF9204670BD00BF3F
:10E260004FAE01087AAE010810B50446006810B13F
:10E27000012106F021F9204610BD0000F0B501266D
:10E28000044608270D468DB0694B6A4A3146009610
:10E2900002A8F2F70BF802A9204605F01BFA02A823
:10E2A000F1F7A6FF644BCDE900571A4604210DEBA8
:10E2B0000700FFF7AFFF0DEB0701204605F00AFA54
:10E2C0000DEB0700F1F794FFEB195C4A01970093FF
:10E2D00004215B4B0DEB0700FFF79CFF0DEB0701E3
:10E2E000204605F0F7F90DEB07001027F1F780FF46
:10E2F000EB190093534B04211A46019702A8FFF72C
:10E3000089FF02A9204605F0E5F9203502A8F1F7BA
:10E310006FFF4D4B4D4A00950421019702A8FFF76E
:10E3200079FF02A9204605F0D5F902A8F1F760FFB0
:10E330000C23474A00930221464B02A8F1F766FFDF
:10E3400002A9204605F0C6F902A8F1F751FF424B99
:10E35000424A3146009602A8F1F7A8FF02A92046DA
:10E3600005F0B8F902A8F1F743FF03220023039256
:10E370003B4D3C4A3C4902A88DF808300495CDE954
:10E380000523CDE90733CDE909330B9304F09CF85D
:10E3900038B929463548FAF74DF820213448F4F7C2
:10E3A0000BF80025304A09A902A804F055F802A983
:10E3B000204605F08FF902A8F1F71AFF2D4B2E4ADF
:10E3C0000095022102A8F1F721FF02A9204605F0DD
:10E3D00081F902A8F1F70CFF284B294A0095022188
:10E3E00002A8F1F713FF02A9204605F073F902A86D
:10E3F000F1F7FEFE0121234B234A009102A8F1F719
:10E4000055FF02A9204605F065F902A8F1F7F0FED4
:10E410001E4B1F4A0095022102A8F1F7F7FE02A940
:10E42000204605F057F902A8F1F7E2FE0DB0F0BD65
:10E430003CD001089CBB01084FD00108C0D30108A3
:10E44000A7D301085DD00108C8D30108F2D30108A1
:10E45000E3BA010864D00108BDD001081FBB010860
:10E46000FCBA0108F9D301089FBB01084FAE0108AF
:10E470007AAE01080ED4010823BB01084CD4010870
:10E480004ABB010887D401080BE30108A3D40108A3
:10E4900072BB010830B504468DB001467A4A684621
:10E4A00004F023FF794A214603A804F01EFF784AAE
:10E4B000214606A804F019FF7649204604F00CFF17
:10E4C00005467548F9F7B6FF0123039A02F11001DA
:10E4D000914205D011F8010D002818BF0023F7E77D
:10E4E000002B53D06D48F9F7A5FF5DB36C48F9F7E1
:10E4F000A1FF6C4A214609A804F0F7FE6A48F9F723
:10E5000099FF08210098FFF777FE6848F9F792FF16
:10E5100008210998FFF770FE6548F9F78BFF102175
:10E520000698FFF769FE6348F9F784FF0998069A91
:10E53000009900F087FE09A8FFF796FE5E48F9F7FC
:10E5400079FF61E05D48F9F775FF5D48F9F772FF03
:10E550000699009800F0D4FD5A48F9F76BFF0421A2
:10E5600000980844FFF748FE5748F9F763FF102169
:10E570005648FFF741FE5648F9F75CFF1021554811
:10E58000FFF73AFE4B48F9F755FFD7E710220698F8
:10E5900009F0EAFC5049514B002808BF1946504881
:10E5A000F9F748FF002D3DD03D48F9F743FF3D4ABC
:10E5B000214609A804F099FE4A48F9F73BFF0821D3
:10E5C0000098FFF719FE4848F9F734FF0821099829
:10E5D000FFF712FE4548F9F72DFF10210398FFF7CA
:10E5E0000BFE4348F9F726FF10210698FFF704FEBB
:10E5F0003048F9F71FFF0998039B069A009900F02D
:10E6000039FE09A8FFF730FE2A48F9F713FF06A8DC
:10E61000FFF72AFE03A8FFF727FE6846FFF724FE50
:10E620000DB030BD2548F9F705FF3248F9F702FF74
:10E63000039A0699009800F0A7FD2248F9F7FAFE20
:10E64000042100980844FFF7D7FD2B48F9F7F2FEA4
:10E6500010211E48FFF7D0FD2848F9F7EBFE1021E6
:10E660002748FFF7C9FD2748F9F7E4FE102126489F
:10E67000FFF7C2FD2548F9F7DDFE16481021FFF728
:10E68000BBFD0C485BE700BF4FD00108F2D3010887
:10E690005DD001089CBB0108EFD0010806D101083C
:10E6A00021D10108C0D3010827D1010838D10108C0
:10E6B0004AD101080AE40108F2D101086AD101082F
:10E6C0006FD10108A1D10108B3D101088001002058
:10E6D000DFD10108B00100200BE40108D8D0010807
:10E6E00011D201082ED2010840D2010853D20108EC
:10E6F00073D20108BCD20108F6D2010862D3010826
:10E700009001002079D30108A001002090D30108D6
:10E7100010B5084CD4F82C211AB964210648F3F737
:10E720004BFED4F82C010023BDE810400322202129
:10E73000FDF720BED8000020CFD50108F0B51F4658
:10E740001446C7B005460E46F122002109A809F07B
:10E750003EFC09AA1021384602F06AF920460AF068
:10E760000BFB07461022002101A809F030FC102FF6
:10E770003A46214628BF102201A809F004FC09AA44
:10E7800005A901A802F0CEF9324605A9284609F0EC
:10E79000FAFB47B0F0BD000038B50C4C0C4D94F8B6
:10E7A0003230022B0ED1082394F8FF20D4F8001148
:10E7B000012002F0F3F86B6B00209847042384F8E3
:10E7C000303038BDEB6A98470123F8E7D8000020C5
:10E7D0003CC7010810B5044601F0B4F820B9204642
:10E7E000BDE8104001F084B810BD0000054B93F85F
:10E7F000212022B993F8350080F0010070470020F5
:10E80000704700BFD8000020F0B570279DB00646C5
:10E810000D463A460021684609F0D9FB08212B46EF
:10E820000DEB010004AC0B4AFFF788FF2B46204696
:10E83000094A102108ADFFF781FF94E80F0085E831
:10E840000F003A466946304609F09DFB30461DB040
:10E85000F0BD00BFC0D50108C8D5010884B070B5AF
:10E860008AB00EAC84E80F00754C4FF49C722546BC
:10E87000002120460EAE09F0AAFB0FCE0FC596E888
:10E88000030014AE85E803000FCE04F118050FC590
:10E8900033682B600E9B0BB96A4B23600F9B0BB93F
:10E8A000684B2360109B23B94FF4A9716648F3F7B6
:10E8B00083FD129B23B94FF4AB716348F3F77CFDE2
:10E8C000119B23B94FF4AD715F48F3F775FD139BAE
:10E8D00023B94FF4AF715C48F3F76EFDA3690BB930
:10E8E0000323A361E3690BB90A23E36194F823309E
:10E8F00013B9012384F8233001F0E6FD94F82430A5
:10E9000013B9012384F8243001F0D6FDA36A0BB9B2
:10E910004E4BA36201F0C4FDFAF792F8C4F8280147
:10E920000138033004D963684948984700207FE0E4
:10E93000032200210120FCF727F9C4F8300120B997
:10E9400040F287114048F3F737FD00220421E069C7
:10E95000FCF71AF9606420B940F28B113A48F3F7DA
:10E960002BFD00220421E069FCF70EF9A06420B918
:10E970004FF4C7713448F3F71FFD00220421012032
:10E98000FCF702F9E06420B940F291112E48F3F748
:10E9900013FD082384F80931042384F80A31002385
:10E9A00084F83630012384F80D31FEF7C9FC05AD3B
:10E9B00068B9A36822690593236807920893E268FF
:10E9C00063680692009395E80F00FEF7BFFC01F024
:10E9D000A1FD23681F4E0793636806F1A002089308
:10E9E000236904960693E368DC3605930AAB43F883
:10E9F0001C2D93E803008DE8030095E80F0002F05A
:10EA000019FA0196A3694FF4CD72009312490123BC
:10EA10001248FCF783FD012805460ED1002303228E
:10EA20000421D4F82C01FDF7A5FC284684F83450C5
:10EA30000AB0BDE8704004B070476368084874E7E6
:10EA4000D80000202D840008CFD5010808E6D33374
:10EA5000F2D401082801002025D50108C1EB0008E7
:10EA60002DD5010810B50F4CD4F82C3123B94FF433
:10EA7000DF710D48F3F7A0FC002303220421D4F832
:10EA80002C01FDF777FC42F21071D4F83001FCF74D
:10EA90008BFA0023D4F830011A46BDE8104019461D
:10EAA000FCF796B8D8000020CFD5010838B50E4D38
:10EAB000D5F8303123B940F2CF110C48F3F77CFC84
:10EAC0000021D5F83001FCF76FFA0128044608D17F
:10EAD0000023D5F830011A461946FCF779F820468C
:10EAE00038BD0020FCE700BFD8000020CFD50108CA
:10EAF00010B5FFF7DBFF68B1074C0023D4F82C01F9
:10EB000003220821FDF736FCD4F82C01BDE81040A3
:10EB1000FCF79CBE10BD00BFD8000020014BD8639D
:10EB2000704700BFD8000020002307B502A941F8B4
:10EB3000043D044B0246D86CFCF7A4F9019803B0DD
:10EB40005DF804FBD800002038B5FFF7AFFF194D82
:10EB5000044620B16B6818489847002038BD686C9F
:10EB6000FCF7B0FBEB698342F7D32146204602F065
:10EB700091F905460028F0D0047000F0A7FE044685
:10EB800018B9284602F0BEF9E7E70C4A13680133CA
:10EB9000136063B91368013313606360012363700A
:10EBA000032320462370FFF715FE6068D6E713683D
:10EBB000F3E700BFD80000205DD5010874500020A5
:10EBC0002DE9F8430123604C604F614E84F83030EA
:10EBD0000A235E4A4FF0FF310020FDF787FB012832
:10EBE0006AD1386843071AD5337833B1F9F78CFE08
:10EBF0000020F9F7DDFE00233370FBF7EBFCFBF799
:10EC000009FD022384F830300023D4F830011A467D
:10EC10001946FBF7DDFF0020FDF76AF8D8E710F092
:10EC2000080521D033787BB941F28830F9F798FE96
:10EC300018B9A0214748F3F7BFFB4748F9F7B8FEDA
:10EC400001233370FFF7A8FD0020FDF781FC4FF48E
:10EC5000FA61D4F83001FCF7A7F90028B8D1A72150
:10EC60003C48F3F7A9FBB3E710F0200043D033781A
:10EC7000FBB194F83030042B1BD1DFF8E4802A4636
:10EC80004146D4F82801FCF73FFA0128814610D10B
:10EC900098F80030072B22D1284600F017FE40B12B
:10ECA0000522C0E90155056180F801900270FFF767
:10ECB00091FD0020FDF74CFC3378002B88D000F04C
:10ECC00059FE0546002883D0032384F830300378AA
:10ECD000052B35D8DFE803F01219192A2A312A4604
:10ECE0004146D4F82801FCF7CDF80128E1D140468F
:10ECF000F9F764FEDDE7FDF72BFC69E7D62115483F
:10ED0000F3F75AFBFFF748FD62E7FFF76FFD38B9ED
:10ED1000284600F0D3FA60B1284600F0E9FDF1E79B
:10ED20002846FFF757FDFFF70FFFEBE701F0F0F97B
:10ED3000F1E72846FFF74EFDE4E700F097FDEBE72B
:10ED4000636806489847E7E7D8000020885000200D
:10ED500078500020CFD5010811E70008D2D401086F
:10ED60007C500020024B93F8FC0001F08DBD00BFE9
:10ED7000D8000020F0B585B007460C461546ADF822
:10ED80000430FFF793FE3E4E28B173683D48984724
:10ED9000002005B0F0BD706CFCF794FAF369834273
:10EDA000F6D3FFF7DFFF8442F2D8002D45D1002CC7
:10EDB000EED12146384602F06DF804460028E7D02F
:10EDC0009DF80530002B3BD0042323709DF80430C0
:10EDD0003BB10D2304A901F8043D0122204600F0B7
:10EDE00005FF96F8312096F83230934203D196F819
:10EDF0003330934217D02023022A18BF00228DF807
:10EE00000C3094F8783003A90BBF43F0040343F0AF
:10EE100001038DF80D208DF80D20204684F8783000
:10EE2000022200F0E3FE6577204600F04FFD054624
:10EE300040B9204602F066F8AAE7DF2DA8D8B8E767
:10EE40000223C2E70023104A836013680133136072
:10EE500093B91368013313606B600A9B28462B61DA
:10EE600001236B702B7000F055FD38B9284600F077
:10EE70003FFD736805488AE71368EDE7686888E72F
:10EE8000D80000205DD501087450002098D50108F5
:10EE9000082808BF0120034B83F8230083F8FC00F7
:10EEA000704700BFD8000020024B83F8240083F88D
:10EEB000FD007047D800002008B5F9F7A3FB014B0F
:10EEC000586508BDD8000020034630B5054C00F158
:10EED0001005224618685968083303C2AB4214462D
:10EEE000F7D130BDA0010020034630B5054C00F13C
:10EEF0001005224618685968083303C2AB4214460D
:10EF0000F7D130BD90010020034630B5054C00F12B
:10EF10001005224618685968083303C2AB421446EC
:10EF2000F7D130BD80010020034630B5054C00F11B
:10EF30001005224618685968083303C2AB421446CC
:10EF4000F7D130BDB001002010B50446FFF7BCFF7B
:10EF50002046FFF7C9FF2046BDE81040FFF7D4BFA9
:10EF600030B51025C3B0224CF122002105A809F0CC
:10EF70002EF82A46002101A809F029F894F86730F4
:10EF800005AA8DF8053094F8663029468DF80630CC
:10EF900094F8653004F178008DF8073094F8643007
:10EFA0008DF8083094F863308DF8093094F86230A9
:10EFB0008DF80A3094F861308DF80B3094F8603099
:10EFC0008DF80C3001F034FD052305AA04F19801F9
:10EFD00001A88DF8043001F0A5FD062305AA04F16F
:10EFE000880101A88DF8043001F09CFD43B030BDCC
:10EFF000D80000200246024B0068516803C37047E6
:10F00000300100200246024B0068516803C370477C
:10F0100038010020034630B5054C00F110052246AA
:10F0200018685968083303C2AB421446F7D130BDA3
:10F0300040010020034630B5054C00F11005224682
:10F0400018685968083303C2AB421446F7D130BD83
:10F0500050010020014B83F822007047D8000020A7
:10F0600070B506460D46144608F01CFCE0B9214672
:10F07000304608F021FCC8B92946304608F060F94E
:10F0800029460646204608F05BF90146304608F05E
:10F0900015FB074908F05EFA4FF07E5108F052F96F
:10F0A00008F044FCC0B270BD0120FCE7FE20FAE786
:10F0B00000007D43014B83F80C017047D80000200D
:10F0C000014B83F831007047D8000020014B1864D1
:10F0D000704700BFD800002013B50024064B02AAD9
:10F0E00042F8044D054993F8FD00FDF787FF2146DE
:10F0F000019802B010BD00BFD8000020ADF200089A
:10F1000030B50430C7B00D46FFF7D6FE1C4B0DF1ED
:10F11000050203F10C0153F8040B8B4242F8040B77
:10F12000F9D11B880124138000238DF813300223AA
:10F1300009AA102128468DF8043001F079FC09AAAB
:10F1400005A901A801F0EEFC05A8FFF7EDFE09AA4C
:10F15000102128468DF8044001F06AFC09AA05A98F
:10F1600001A801F0DFFC05A8FFF7EEFE1022054B19
:10F1700083F8214083F8202083F8502047B030BD29
:10F1800089D50108D800002030B50430C7B00C463E
:10F190001546FFF791FE294B0DF1050203F10C0115
:10F1A00053F8040B8B4242F8040BF9D11B8820461C
:10F1B000138000238DF813300223012409AA1021A3
:10F1C0008DF8043001F034FC09AA05A901A801F06A
:10F1D000A9FC05A8FFF7A8FE09AA102128468DF86A
:10F1E000044001F025FC09AA05A901A801F09AFC38
:10F1F00005A8FFF769FE032309AA05A901A88DF850
:10F20000043001F08FFC05A8FFF76EFE042309AA65
:10F210000DEB030005A98DF8043001F083FC05A86F
:10F22000FFF772FE1122064B83F8214083F820205D
:10F2300083F8502083F8074147B030BD89D50108D5
:10F24000D800002038B50D461446FFF7D3FE2846F7
:10F25000FFF7D8FE2046FFF7DDFE2046FFF7EAFE67
:10F260000022034B83F82120102283F8202038BD90
:10F27000D800002070B50E4615461C46FFF7BAFEB2
:10F280003046FFF7BFFE2846FFF7C4FE2046FFF7D3
:10F29000D1FEBDE870400022034B83F821201122EB
:10F2A00083F82020FFF75CBED800002028B1836AD5
:10F2B000012B01D1007B7047002070472DE9F04FF2
:10F2C000054689B010B10378012B03D01C21844876
:10F2D000F3F772F86B691BB91D218148F3F76CF8DD
:10F2E0006B691B78042B05D0022B03D01E217C48B0
:10F2F000F3F762F800267B4C08AA94F8FF3094F8E4
:10F30000FD800293D4F8003142F80C6D76494046F6
:10F3100094F8FCB094F8FEA00393FDF76FFE074647
:10F3200038B9284600F08AFB0127384609B0BDE805
:10F33000F08F059B8BB1FDF725FE0599042904D9B3
:10F34000284600F0B3FB0027EFE7684841434FF43D
:10F350007A70B1FBF0F0FCF753FCAB680133012B82
:10F36000AB600FD1D4F8F03068690133C4F8F030E5
:10F3700094F80831013384F8083100F0F3FB686930
:10F3800000F054FC636D6E697360D4F8F0307381E3
:10F3900094F80431002B63D0002384F80431337ACD
:10F3A00043F00403337294F8FC30384686F87C301E
:10F3B00001F0F2F886F87D000121686900F0E8FBB1
:10F3C00094F80D214FF47A7312F00F0208BF012256
:10F3D00000265A4307AB019306AB0093394602F56A
:10F3E0007A736869069600F05DF90746002898D0A0
:10F3F000FCF7B6FAE860069860B1314600F0C8FB49
:10F40000069B1B78052B04BF012384F804310023DD
:10F4100084F80631069800F081FBDDE9060100F072
:10F4200027FE069BFBB11B7A13F004032FD0B946CD
:10F4300094F80B31AB606A691278022A02D194F811
:10F440000B21AA6000F0AEFA064610BB8A212448C0
:10F45000F2F7B2FF264B274A8B21214808F040FCE7
:10F46000A6F87A309FE79946ECE7314668689847F6
:10F470006420FCF7C5FB304600F0A4FA94F80B3189
:10F48000AA689A42BFF451AF032333705BE79946F1
:10F49000D1E780226969183008F075FD00229DF8D7
:10F4A00008300699F373039BC6F898102978727296
:10F4B000336194F83530C6F8802033752B6986F8AF
:10F4C0000CB086F80D8086F80EA03270717086F848
:10F4D0000890002BC9D1304600F08EFACEE700BF6D
:10F4E00025D60108D8000020ADF2000840420F00E8
:10F4F0006AD6010817D601082DE9F04385B0064603
:10F500000C468DF80F202BB101220DF10F010020C8
:10F51000F9F7CCFDFCF724FA1C4B1D4DDFF8788081
:10F520009DF80F1007469B6A2046984741F28832A3
:10F530002946D8F82801FBF7A5FC28B32B78012B26
:10F540001DD12846AC68F9F739FA4FF47A70A4EB6C
:10F55000070909FB000007F0A5FF01463046FDF74B
:10F56000CBFD9DF80F10CDE90049D8F800503B467F
:10F5700032680848A847204605B0BDE8F083284611
:10F58000F9F71CFA0024F6E70446F4E73CC7010843
:10F590008C50002016D70108D80000202DE9F84F24
:10F5A000394E9846736B0546894614464FF47A7A6D
:10F5B0009847DFF8DCB0354F0AFB05F202F59C32C4
:10F5C0008032B2FBFAF23249D7F82801FBF75AFC35
:10F5D00020B9336B98474FF0FF302FE09BF8003095
:10F5E000072B07D15846F9F7E9F94FF47A65F9F78F
:10F5F000E1FCE1E7032B366B22D1DBF804502879DC
:10F600002968844228BF04464846224608F0BBFCCD
:10F610003F6895F90830B5F90620A9881D48B84714
:10F62000B8F1000F05D0EB88A8F800302B7A88F8E5
:10F6300002301748F9F7C2F9B0472046BDE8F88F05
:10F64000042B0BD11248F9F7B9F9B0473C68FCF725
:10F6500087F901461048A0470020EFE7052B0AD1A3
:10F660000B48F9F7ABF9B0473C68FCF779F901466C
:10F670000A48A047AFE7D3210948F2F79DFE0448A6
:10F68000F9F79CF9B047A6E73CC70108D80000206D
:10F69000985000207BD60108A5D60108BDD60108E8
:10F6A000D3D601082DE9F04FC9B08946174608A9FD
:10F6B000FF2202901E46DDF84C8101F03DFC82469F
:10F6C00018B9002049B0BDE8F08F634CD9F800208C
:10F6D00094F8FC1094F8FE5008468D429ABF4D1BDA
:10F6E000EDB20025D4F800B00592049101F078F84D
:10F6F000039094F8FD0001F089F8DDE90412039B02
:10F7000000905648D847D9F800202846D4F800B0D1
:10F71000039201F065F8039A034629465048D847FA
:10F7200094F8FF10D4F800210846D4F800B00492F1
:10F73000039101F055F8DDE9031203464948D84723
:10F7400094F8FD3094F8FC20D9F80010002001F066
:10F7500025F90023524608A94846FFF7CDFE044686
:10F760000028AED0029B93F8783013F0050F0BD031
:10F7700013F0040F0CBF00220222374B93F8321013
:10F78000914218BF83F83220FF22002108A808F018
:10F790001EFCD9F800104FF47A792A46082301207C
:10F7A00001F0FCF809FB07F1A1F51C414039B1FB60
:10F7B000F9F106A80694FCF7E3F9FF22434608A9ED
:10F7C0004FF44D70FFF7EAFE421C05463FF479AF57
:10F7D000002821491ADD0E68FCF7C2F823460246CC
:10F7E00029462148B047B8F1000F02D0012388F81C
:10F7F00003300023529A9D42136005DDE9B208A848
:10F8000001F00CFF529B186001205BE791F8FF208C
:10F810000823D1F80011012001F0C0F809FB06F11E
:10F82000A1F51C414039B1FBF9F107A80794FCF799
:10F83000A7F94346FF2208A94FF44D70FFF7AEFE2B
:10F84000431C05463FF43DAF0028D2DDB8F1000F60
:10F85000CFD00223CBE700BFD80000208DD701080E
:10F86000C0D70108E7D701080ED8010870B5C2B0AB
:10F8700001ABFF2202A94FF47A60FFF78FFE061E4C
:10F880001EDD114DF1B26A6D02A801F097FC04462D
:10F89000B0B10378052B01D0032B0DD100212046F8
:10F8A00000F076F9204600F039F92046019900F081
:10F8B000DFFB2B6C204613B901F024FB00E09847D6
:10F8C000304642B070BD00BFD800002038B5074BAD
:10F8D0000546DB6818209847044620B11422002111
:10F8E00008F075FB6561204638BD00BFD8000020D8
:10F8F00010B5044650B1406901F004FB0023636178
:10F90000034B2046BDE810401B69184710BD00BFDF
:10F91000D8000020037807B5052B4FF0000302A99B
:10F9200041F8040D06481A460CBF806C406CFBF78A
:10F930004FF9431E5842584103B05DF804FB00BF25
:10F94000D800002007B5037802A941F8040D084843
:10F95000052B4FF000024FF001030CBF806C406C90
:10F96000FBF736F9431E5842584103B05DF804FBDB
:10F97000D800002037B5002202AC094D44F8042D10
:10F980002146A86CFBF77EFA019B33B995F8362027
:10F990001AB92146686CFBF775FA019803B030BDBF
:10F9A000D8000020064B10B5DB68A020984704461D
:10F9B00018B1A022002108F00AFB204610BD00BFAC
:10F9C000D800002070B5044690B1D0F88000094DF1
:10F9D00008B12B699847D4F8980020B101F092FA49
:10F9E0000023C4F898302B692046BDE870401847C2
:10F9F00070BD00BFD80000201FB50E4C0190E06C18
:10FA0000FBF772FC024638B903A9E06CFBF73AFA3F
:10FA100010B10398FFF7D6FF002301A91A46E06C46
:10FA2000FBF7D6F820B94FF4B4710348F2F7C4FCE1
:10FA300004B010BDD8000020D3D60108F8B50423C7
:10FA4000437003780546032B0ABF144B0469DC6B33
:10FA5000FFF7A8FF0646B0B940F277111048F2F759
:10FA6000ABFC104B104A4FF4BC710D4808F038F94C
:10FA700031466868A0473046FFF7A4FFFA20FCF73C
:10FA8000BFF83846F8BD01272B7807704370002C6B
:10FA9000EED1FFF7B1FF2046F4E700BFD800002009
:10FAA000D3D6010873D6010849D70108F8B5037801
:10FAB0000646032B08BF154B0F460CBFDC6B0469D1
:10FAC000FFF770FF0546B0B94FF4C8711048F2F760
:10FAD00073FC104B104A40F291110D4808F000F9E8
:10FAE00029467068A0472846FFF76CFFFA20FCF70C
:10FAF00087F80120F8BD0223037033784760437014
:10FB0000002CEDD1FFF778FF2046F3E7D800002066
:10FB1000D3D6010873D6010865D7010808B5104A85
:10FB200010B1002382F8083192F82230BBB192F86C
:10FB3000083192F809118B4211D95B1A92F80A1117
:10FB400093FBF1F201FB12334BB900F0C5FC30B965
:10FB500000F0D0FC18B9BDE8084000F0DBBC08BDDF
:10FB6000D8000020094B93F822206AB1027A42F0B3
:10FB70000102027293F8082193F809319A4282BF78
:10FB8000037A43F002030372704700BFD8000020DD
:10FB900070470000064A1378FD2BDFBF0078054947
:10FBA000C8540133DABF012013700020704700BF32
:10FBB000A5510020A650002038B10078032803D0BA
:10FBC000431F58425841704701207047052307B52D
:10FBD00002A800F8013DFFF7DDFF0348FFF7DAFF59
:10FBE00003B05DF804FB00BFA4500020037A70B599
:10FBF0001B09D61804460F2E00F10C0015461844B8
:10FC000009DC08F0C0F90120237A05EB131565F330
:10FC10000713237270BDC3F10F0208F0B4F9237A01
:10FC2000002043F0F0032372F4E7000037B5114CD5
:10FC30000546227822B11049FFF7D8FF0023237030
:10FC40000E4C94F806213AB1082302A901F8043DAC
:10FC500001222846FFF7CAFF94F8073143B140F26A
:10FC6000011302A921F8043D02222846FFF7BEFF36
:10FC700003B030BDA5510020A6500020D8000020C0
:10FC80000122044B00F00F0083F80D0183F80621D8
:10FC9000704700BFD80000202DE9F04F17461E46E0
:10FCA0004FF000088BB0CDE901019DF85050C04CD9
:10FCB000A84502D30BB0BDE8F08F16F8083006EB6C
:10FCC000080A013B1F2B00F2CE81DFE813F0200071
:10FCD000CC012C006601DC00C0001E016001660141
:10FCE0004701CC017901940092019501CC01CC012E
:10FCF000CC01CC01CC01CC01CC01CC01CC01CC019C
:10FD0000CC01CC01CC01CC01CC01CC01B701A5EBDD
:10FD10000803DBB2012B4FF0000920D084F80791D3
:10FD20004FF002091BE04FF00009A5EB080B5FFA4A
:10FD30008BFB8DF81C9009F104035B4503DA1AF87C
:10FD40000930032B0DD0B9F1000F08D003230AA806
:10FD500000F8083DFFF71EFF07A8FFF71BFFC1448F
:10FD60008AE00AEB09014B7809F102001A095044B4
:10FD700003F00F03059104920393F8F754FC0599DF
:10FD8000049A097909F10509062AC1F3021C5FFAF0
:10FD900089F901F00F01039B21D90F2A05D19DF8A4
:10FDA0001C2042F002028DF81C205A1E062A19D986
:10FDB0000F2B05D19DF81C3043F004038DF81C3047
:10FDC00009B184F80B11BCF1000F0ED100F06EFCEC
:10FDD0009DF81C3043F001038DF81C30ABE784F82C
:10FDE000FC20DCE784F8FD30E4E7BCF1060FA2D18B
:10FDF0004FF6FF70EAE7A5EB0803DBB2052B40F2F4
:10FE00002F810AF10100F8F704FC9AF9053000216E
:10FE1000002B18DB62A3D3E9002312184B41914653
:10FE20009A46002394F80D2119EB02004AEB0301D6
:10FE3000022F02D1013041F10001019BC3E91C01F5
:10FE40004FF006098BE758A3D3E90023E5E7062323
:10FE50000AA800F80C3DFFF79DFE029B0DF1280952
:10FE600003F01F0309F8083D5248FFF793FE484688
:10FE7000FFF790FE08F101095FFA89F9C8453FF4E0
:10FE800019AFC84614E7A5EB0803DBB2042B40F218
:10FE9000E780DAF80120DFF824910892D2B2C2F3A9
:10FEA000021384F8FE3099F80030C2F30302052AE9
:10FEB00043F0040394BF43F002036FF341030DF1D9
:10FEC000210098BF84F8FF2089F800304FF0640AC1
:10FED000F8F7A1FB0AFB00FA5046F9F76DF878B184
:10FEE00099F80030C4F800A143F00103012289F819
:10FEF0000030314B1A70FFF769FE4FF005092EE70D
:10FF000099F8003060F30003F0E7A5EB0803DBB2DB
:10FF1000052B40F2A580534653F8010F9AF80310C1
:10FF20001A799AF80430090241EA03419AF802303A
:10FF30000890194364239AF8010059438DF824204E
:10FF400000F04CFB07238DF818000AA800F80C3DC0
:10FF5000FFF720FE06A8FFF71DFE71E7A5EB0803DB
:10FF6000DBB2042B7CD96421DAF80100030A59437F
:10FF7000C0B200F065FB0A238DF81C000AA800F847
:10FF8000083DFFF707FE07A8FFF704FEB5E79AF85C
:10FF9000010000F00F00FFF773FE08F102096BE7A4
:10FFA0006E3DD512000000006F3DD512000000002C
:10FFB000D8000020E4010020A5500020A45000201B
:10FFC000A5EB0803DBB2012B4AD001239AF80120EC
:10FFD0000AA8110902F00F0203FA01F1934084F814
:10FFE0000A310C2384F8091100F8083DFFF7D2FD0F
:10FFF00096E608F103093FE7A5EB0803DBB2012B06
:020000040801F1
:100000002ED0A3689AF8019098470122174B8DF8DB
:100010001C20C3E900014FEA19130A3302FA03F363
:10002000C4F8183109F00F03C4F81C310F230AA8D3
:1000300000F8083DFFF7AEFD07A8D7E7A5EB0803DA
:10004000DBB2012B0CD09AF801300BB1022B07D197
:1000500094F833209A423FF463AE84F833305FE67D
:100060004FF000097BE6C14608E700BFE801002029
:1000700030B585B003910446174B30B91B7803B3F4
:1000800005B0BDE83040FFF7A1BD00259DF90E1079
:100090009DF80F201D70FFF78FFD90B10F48237A58
:1000A00090F822502DB113F0010518BF012580F8FA
:1000B00005511B0907D0009304F10C032046FFF7FC
:1000C000EBFD05B030BD637F002BFAD1237F002B01
:1000D000F7D00093A36EF1E7A5500020D8000020D0
:1000E00010B5044678B1836A012B0CD1C36A1BB9E1
:1000F00010210648F2F760F9E36A587802288CBFAD
:100100000020012010BD0020FCE700BF42D80108FC
:100110002DE9F04F054689B018B10378033B012B58
:1001200003D92221C148F2F747F96B690BB11B785B
:100130001BB12321BD48F2F73FF90027BC4C94F8CE
:10014000FF3094F8FD800393D4F8003194F8FCB0AC
:10015000029394F8FEA000F0AFF900F0B5F908AAF8
:1001600042F80C7DB3494046FCF748FF064620B9EB
:100170002846FFF763FC01260AE0059BA3B1FCF7C4
:1001800001FF0599042907D92846FFF78FFC3E4651
:10019000304609B0BDE8F08FA74841434FF47A706C
:1001A000B1FBF0F0FBF72CFDAB6894F82020013395
:1001B000102AAB602DD1012B09D1D4F8F0300133D6
:1001C000C4F8F0309D4B5B699847A4F8E800B4F898
:1001D000E8300133A4F8E830002707AB019306AB01
:1001E0000093314641F2707341F28832686994F8A5
:1001F000FF90069784F8FF70FFF754FA0646A8B9F7
:100200002846FFF71BFC069800F07CFE84F8FF9060
:10021000B1E7112A05D1636989489847A4F8E80035
:10022000DAE750218148F2F7C7F8D5E7069A84F853
:10023000FF9012B11378012B06D02846FFF7FEFB82
:10024000069800F05FFEA3E794F82030102B40F0F2
:10025000A0801023002784F85030069BDA6862657E
:1002600003F15302002F00F0A3801121DFF8D4C165
:1002700084F8501003F1630E674610685168083225
:1002800003C77245BC46F7D1DFF8BCC103F12302B6
:1002900003F1330E674610685168083203C7724590
:1002A000BC46F7D1DFF8A4C103F1330203F1430EDA
:1002B000674610685168083203C77245BC46F7D1DB
:1002C000DFF88CC103F1430203F1530E6746106857
:1002D0005168083203C77245BC46F7D1544F9A683B
:1002E000BA631A7CC2F3030287F8FF201A7CC2F3B8
:1002F000021287F8FE20587CFFF7C2FC0022069805
:1003000097F83110437C1230012B98BF87F80621F3
:1003100011F0FD0F18BF87F83120C7E93D22C7F85B
:10032000F02087F8322087F8332000F0E1F9FCF75D
:1003300029FE012384F83530FFF734FB802207467D
:100340006969183007F01FFE0023069AC7F880304D
:10035000C7F8982094F835207B723A753B709DF869
:100360000C202B78FA737B70029AE36B87F80CB041
:1003700087F80D8087F80EA03A61002B52D03946DD
:10038000686898476420FBF73BFC3846FFF71AFB88
:10039000FEE6112B07D192F82270002F3FF459AFDF
:1003A00084F8503059E77D212048F2F705F854E7EA
:1003B0001021DFF890C084F8501003F1630E6746F7
:1003C00010685168083203C77245BC46F7D1DFF8A0
:1003D00078C003F1230203F1330E674610685168B9
:1003E000083203C77245BC46F7D1DFF860C003F19D
:1003F000230203F1330E674610685168083203C7C1
:100400007245BC46F7D1DFF848C003F1230203F17F
:10041000330E674610685168083203C77245BC4600
:10042000F7D15BE73846FFF7E7FAB1E642D80108B3
:10043000D8000020E100010840420F003CC701083D
:1004400030010020B0010020A00100209001002018
:1004500080010020437882781B02007843EA02433F
:1004600003430A20B3FBF0F07047000038B50446A0
:1004700081B10D7884B1A36A012B0DD1E36A1BB958
:100480005D210648F1F798FFE36A5878431B58420C
:10049000584138BDFF25EDE70020FAE7D0D8010824
:1004A000044B93F8252083F8FF209A6AC3F80021B3
:1004B000704700BFD8000020024B93F8242083F837
:1004C000FD207047D8000020024B93F8232083F8CA
:1004D000FC207047D8000020054B93F8242093F8A7
:1004E000FD1091423ABF012083F8FD2000207047A3
:1004F000D8000020064A92F8FC3092F82310994266
:100500003DBF03F1FF33012082F8FC30002070472B
:10051000D800002010B5FFF7C3FF0120FCF7F4FE60
:100520005023164C01212370002322461448637087
:10053000FCF78CFE18B932211248F1F73DFF502329
:100540000121114A1148A370E170FCF77FFE18B930
:1005500036210C48F1F730FF5023237102230C4A57
:1005600001210C486371FCF771FE28B9BDE8104009
:100570003A210448F1F720BF10BD00BF0456002007
:10058000043F0D00D0D8010806560020CC3F0D00D6
:100590000856002094400D00836A10B5012B0446D4
:1005A00008D1C36A1BB94B210348F1F705FFE36A81
:1005B000587810BD0020FCE7D0D8010807B502A983
:1005C00001F8010D0448FCF7EFFC08B1FCF710FE40
:1005D00003B05DF804FB00BF6D0401082DE9F04194
:1005E0004FF47A769046B1FBF6F6C8F30317052F61
:1005F000044630468CBF002701274FF00005FCF76A
:10060000BBFD18B10F2C8CBF0020012067F3000543
:1006100060F3410505F00303032B0CD12046FFF7DF
:10062000CDFF064B012103EB4402547003F8148004
:100630003046FCF70BFE2846BDE8F081045600204A
:100640000F282DE9F04105460F461FD8164B03EB46
:1006500040035C78231A5C425C414FF47A78B7FB24
:10066000F8F0FCF789FD4FF0000360F3000364F33A
:10067000410303F00303032B064609D04FF00000AB
:1006800066F3000064F34100BDE8F0810024E4E774
:100690002846FFF793FF044A012102EB450208FBBD
:1006A00007F0FCF7D3FDE9E704560020002373B5FB
:1006B000044602AD0D4E05F8013D9DF807300F2BA5
:1006C00001D902B070BD29463046FCF76DFC18B167
:1006D000E30708D5FCF772FD9DF807306408013385
:1006E0008DF80730E9E7FCF74FFDF5E76D040108E9
:1006F00038B504460320FFF761FF0420FFF75EFFD3
:100700000520FFF75BFF0620FFF758FF0720FFF7E4
:1007100055FF2046FFF79EFE0546FCF72DFD48B12C
:100720005023294A0121937103230632537028462E
:10073000FCF78CFDE01CFFF78DFE0546FCF71CFD69
:1007400048B15023204A0121137204230832537008
:100750002846FCF77BFDA01DFFF77CFE0546FCF755
:100760000BFD48B15023184A0121937205230A3228
:1007700053702846FCF76AFD04F10900FFF76AFE92
:100780000546FCF7F9FC48B150230F4A01211373C9
:1007900006230C3253702846FCF758FD04F10C0078
:1007A000FFF758FE0446FCF7E7FC58B15023064A11
:1007B000204693730723D3730121BDE838400E32DE
:1007C000FCF744BD38BD00BF045600200738C0B256
:1007D00005289ABF014B185C0820704785D801088E
:1007E00006289ABF014B185C002070478BD801087F
:1007F000052804D90628034818BF0020704702487E
:10080000704700BF90D0030048E80100072810B5EA
:10081000044604D940F243110348F1F7CDFD034BE0
:1008200013F9240010BD00BFD0D8010894D80108E6
:10083000142810B5044613DD4FF4A4711148F1F7E4
:10084000BBFD062C14DD082C14DD0A2C14DD0C2C49
:1008500014DD0E2C14DD152CB4BF0020082010BDB3
:10086000022803DD0428ECDC0620F8E70720F6E781
:100870000520F4E70420F2E70320F0E70220EEE78A
:100880000120ECE7D0D8010808B50F280DD8DFE823
:1008900000F0181818081A1A1A0A0A0C0C0C0C0C7A
:1008A0000C0A732008BD0020FCE74FF4C171074813
:1008B000F1F782FD064B074A40F28311034807F027
:1008C0000FFA3320EEE7DE20ECE700BFD0D80108B6
:1008D000DDB80108B4D801082DE9F0468DB0924684
:1008E00099462A4A149B074693420C4608D0284A48
:1008F000934203D0A6212748F1F75EFD002600E0D1
:100900000126254DEB6A98472046EB689847012F52
:100910004FF0000422D108230A22CDE90132AB694D
:1009200031460B93CDE90877CDE90644CDE904447F
:10093000039400943B464A4602200B9EB047214652
:10094000FF20F8F79FF80820F8F792F834213920B3
:100950002B6C0B930DB0BDE8F04618474FF47A634B
:100960000127CDE907430823CDE90173EB69CDE900
:1009700005440B93CDE9034722465146CDF800903C
:10098000334602200B9CA0473946D9E790D003009C
:1009900048E8010015D901083CC701082DE9F341D9
:1009A0000446104615460E469846FFF721FF0746B7
:1009B0002846FFF715FFC5B21DB9C5210948F1F753
:1009C000FBFC64B94046FFF721FF024600972B4627
:1009D00031462046FFF780FF02B0BDE8F0810022DB
:1009E000F4E700BF15D901080A68036853400360A3
:1009F0004A684368534043608A6883685340836011
:100A0000CA68C3685340C36070470B6810B5146868
:100A10006340036054684B686340436094688B682C
:100A200063408360CB68D2685340C36010BD000050
:100A3000A1F11003DBB2102B2DE9F0470C4615464F
:100A400008D84FF0010909FA03F303F0013323F04A
:100A500080732BB90023FF2085F8F030BDE8F087C4
:100A60000A460146284607F08EFA04F11C0E4FEAAA
:100A70008E0E5FFA8EFE4FEA1E13013B85F8F030B2
:100A800023462749B3FBF4F204FB1232E81812F0B4
:100A9000FF0210F804AC10F803CC10F8027C10F838
:100AA000016C32D111F80C804FEAD91289EA08089A
:100AB00011F807C08F5D11F80A604FEA420A5244EC
:100AC000C24602EBC20282EA49025FFA82F91A1BAD
:100AD000D2B215F802802A448AEA080A05F803A06F
:100AE00092F8018004338CEA080C80F801C092F877
:100AF00002C0DBB287EA0C078770D2789E4586EA8F
:100B00000206C670BED80020A8E7182CDFD9102A2C
:100B100001BF11F80AA011F80CC0CF5D8E5DD6E7B9
:100B200057DB01082DE9F04F92F8F030A1B01A918F
:100B30001892002B00F05D8101461CA8FFF765FFAD
:100B40004FF00108AC4CAD4DAD4E189B9DF875E0D3
:100B500003EB081319939DF870309DF87AA0009369
:100B6000009A9DF87F90A05C9DF8742014F80A10FC
:100B70000192019F9DF87920E75D02920697029FFE
:100B80009DF87E20E75D03920797A25C9DF8787040
:100B9000049208979DF873209DF87D70059214F8D3
:100BA000093014F80EC0A25C09979DF872700A977C
:100BB000E75D0B979DF877700C97E75D0D97089FA1
:100BC000E75D0E97099FE75D0F979DF87C70109782
:100BD0009DF8717011979DF876701297E75D1397E5
:100BE0009DF87B701497E75D1597109FE75D16974A
:100BF000119FE75D1797189F97F8F07047453ED80B
:100C00008DF870009DF818008DF872108DF8740042
:100C10009DF82C109DF838008DF87A108DF878002A
:100C20009DF810109DF858008DF876108DF87C0016
:100C30009DF84C109DF81C008DF87E108DF8750005
:100C40009DF854109DF83C008DF87F108DF87900C8
:100C50009DF834109DF85C008DF87B108DF87D00B8
:100C60008DF877201A98199A1CA98DF871C08DF803
:100C70007330FFF7CAFE002021B0BDE8F08F81EA93
:100C800003071B97009F434015F807B01B9F80EA9E
:100C90000C008BEA070716F80EB081EA0C0187EA10
:100CA0000B078DF8707015F80E707B4016F80A70FF
:100CB0007B408DF8713015F80A30584016F809302D
:100CC0005840009B8DF8720016F803C0049B8CEA14
:100CD000010115F809C0534081EA0C018DF8731029
:100CE00001991CA8695C4B400299715C4B408DF8DE
:100CF0007430069B5A40029BEB5C5A40039BF35CAA
:100D00005A408DF87520DDE906325340039AAA5CFB
:100D10005340059AB25C53408DF87630079A049B95
:100D20005340019AB25C5340059AAA5C53408DF837
:100D300077300D9A0B9B5340089AAA5C5340099A4E
:100D4000B25C53408DF87830DDE90D325340099A9A
:100D5000AA5C53400A9AB25C53408DF87930DDE9C1
:100D60000E3253400A9AAA5C53400C9AB25C53402C
:100D70008DF87A300B9B0F9A5340089AB25C53401F
:100D80000C9AAA5C53408DF87B30159A139B534004
:100D9000109AAA5C5340119AB25C53408DF87C3093
:100DA000DDE915325340119AAA5C5340129AB25CA5
:100DB00053408DF87D30DDE916325340129AAA5C1B
:100DC0005340149AB25C53408DF87E30179A139BAF
:100DD0005340109AB25C5340149AAA5C199953403C
:100DE0008DF87F30FFF700FE08F101035FFA83F80A
:100DF000ABE6FF2040E700BF57DB010857D90108E9
:100E000057DA01080068704782B0034660B16A464D
:100E100059680068013B03C207221DF8021012F155
:100E2000FF3203F8011FF8D202B070470FB404B0CC
:100E30007047000030B585B06D4685E80F00104C56
:100E400095E80F0084E80F0004F1100208A903C917
:100E500082E803000BB90B4BE360A3680BB9094BA5
:100E6000A36063680BB1236833B9A3680648984749
:100E7000064B6360064B23600123237605B030BD2B
:100E8000A85100202D0E0108CDDC0108197F0108B2
:100E9000097F01082DE9F041184D80462B7E0E4652
:100EA0001BB973211648F1F787FADE2E03D9742196
:100EB0001348F1F781FA2B6880209847044680B1E7
:100EC0008022002107F083F8B8F1000F12D08EB114
:100ED0002B6830469847074630B920466B689847DC
:100EE0003C462046BDE8F0813246414607F04BF8CB
:100EF0002677A76600236370F3E700BFA8510020A0
:100F000080DC010870B50A4C0546237E1BB98F2191
:100F10000848F1F751FA55B1A86E636810B19847C7
:100F20000023AB6663682846BDE87040184770BD73
:100F3000A851002080DC01082DE9F0479C4B1746A2
:100F40001A7E92B005460E4698461AB9A7219948CE
:100F5000F1F732FA032F01D80024D8E02A786B7811
:100F600043EA421333702B78022B02D0042B40F05B
:100F70008D800023042F8DF82630EDD06B687370C0
:100F80006B681B0AB370EB88F370EB7933716B6895
:100F9000CDF822309DF82630002B40F0C180052F7F
:100FA000DAD006242A7AC2F3400302F001019B0141
:100FB00043EAC11343EA1213C2F3800243EA421325
:100FC000737195F808904FEA1919631C9F42C3DDAD
:100FD0006A89DBB232556A890234120AF254D8F8AF
:100FE00010301A886B899A4204D040F24711714838
:100FF000F1F7E2F9D8F81420D8F8103011781B680E
:1010000010290A930DD902930DF1220301930123B4
:10101000297A009358320023090905F10C0000F0E9
:10102000E5FCB9F1000F0BD004EB090A574593DB3F
:1010300030194A4605F10C0106F0A5FF5FFA8AF463
:101040002B7F002B77D0BC4286D26B7F04F1010945
:1010500033556A7F5FFA89F9D8F81430002A68D1CD
:1010600058330693AB6E06A907932B7F06EB090056
:10107000ADF8203000F0ACFB4844C4B2A7425AD2CD
:1010800040F275114B48F1F797F965E7032B01D052
:10109000052B01D101236DE7002B3CD1082F7FF6F2
:1010A0005BAFD8F81440701C224652F8083FC6F8CF
:1010B000013053684360FFF7A7FE102F7FF64CAF57
:1010C000224652F8103F06F10900C6F8093053686D
:1010D0004360FFF799FE122F7FF63EAFB4F89830C9
:1010E00006A97374B4F8983005A81B0AB3741323C7
:1010F0002834CDE90646ADF8203000F033FB162F3A
:101100007FF62AAF1724059BC6F813306B6620467E
:1011100012B0BDE8F087D8F80C30274898471BE795
:1011200040F23D112348F1F747F94FF0000905243B
:101130004BE7883395E7E31C9F427FF70DAFD8F864
:1011400014301A78102A0DD1783306A905A8CDE9F4
:101150000636ADF8204000F06CFA059B335104349C
:10116000E4B2D4E7112A1DD103F1780268330B935E
:101170000DF122030F930A9B0BA91093B5F87A3057
:1011800005A8ADF8443095F87C300C928DF84630C7
:1011900095F87D300D968DF84730ADF8384000F069
:1011A00080FADAE74FF4CB710248F1F705F9AEE7C0
:1011B000A851002080DC010857DC01082DE9F04F20
:1011C0008F4DA3B02B7E06460F46904623B940F2C2
:1011D000A3118C48F1F7F0F8022F2CD92B6880204E
:1011E0009847044630B9EB6887489847204623B0B3
:1011F000BDE8F08F8022002106F0E9FE33785B091C
:1012000023703278072B02F00302627003D1EB687F
:101210007E4898470CE0B8F1000F00F0EF81012BF9
:1012200040F0C581AB687A48F3E742467948984771
:101230006B68204698470024D8E701F18802A0E1B6
:10124000F3465068227A4FEADC1E6EF300024FEA42
:101250005C1E6EF382024FEA1C1E6EF3C3026CF337
:101260000712227282B24A454FEA104C84BF0CF139
:10127000010C1FFA8CFC09EB0C4906EB0800CDF8B9
:101280003090FFF7BFFD0DF1880A68314AF8681DFC
:101290006066514607A800F0CCF9079B626E934246
:1012A00004D0EE685C495D48B047C1E72A6909F19E
:1012B0000101BBF1000F2CD05160227A04F10C0324
:1012C000049313091A4606F108010498059306F0E1
:1012D0005AFE6A69117810290CD90DF12A01019181
:1012E0000021CDF8089000915B46DDE904015832F9
:1012F00000F07CFB237A1B0903F10C0297422DD9E5
:1013000003F10D02974206D1002345482377EB688D
:101310006BE79160D1E70933A8EB0300617FC0B2AE
:1013200020776A6961B958321E4408920996ADF86F
:1013300028002B689847A06620B9EB68394868E711
:101340008832F1E7514600F043FA00283FF74EAFEC
:10135000EB68354898476B68A06E5AE700232377FF
:10136000A36643E7212F01D101232AE1EB682F482F
:101370004FE79DF83F30043F09EB0700DB09FFF71B
:1013800041FD6E696066A3B30DF1580A0021302259
:10139000504606F01CFEFF2332468DF8583052F8B6
:1013A000083F0DF15900CDF8593053683836CDF863
:1013B0005D30FFF729FDB6F860303A468DF86130B0
:1013C00049461B0A0DF163008DF8623006F0DBFD23
:1013D000CDE9086A08F1070808A907A8ADF8288030
:1013E00000F0C0F9636E079A9A4223D0EB68104868
:1013F0000FE72836CDE90869A8F10408ECE700BF3B
:10140000A851002080DC0108FADC010812DD010887
:1014100040DD01088FDD01086EBA0108CADD010850
:101420000FDE010843DE010875DE01089BDE0108BE
:101430000DDF01089DF837609DF83630360446EA26
:1014400003269DF835300DF13B001E4366609DF884
:101450003A709DF839303F0447EA03279DF8383049
:101460001F43A760FFF7CEFCE0609DF83F20237C80
:10147000D10961F3C713110961F3061362F3030382
:1014800023749DF84030637494F8213003B322AB89
:1014900033F8472D9B786282237522AB33F8442DB5
:1014A0009B78A4F81520E37522AB33F8412D9B7887
:1014B0002283A37622AB33F83E2D9B78A4F81B2021
:1014C000637722AB33F83B2D9B78E28384F820309E
:1014D0006D6994F9102005F1280C002AB5F89810D0
:1014E00004F1230004F15303CDF858C016AA12DA10
:1014F00005F11807ADF868100092083504F14302B1
:1015000004F13301CDE91776199500F0FCF90123B8
:1015100084F822306AE6ADF864101946CDE9176701
:1015200000F0B0F90023F3E7EB68394871E6701C6E
:10153000FFF768FC804501466060EB687FF475AE9C
:101540004146344898470023052F6377A7F10408E4
:1015500007D9737903F00F0308339845C4BFF35CD0
:101560006377F37996F8069096F805C049EA03295F
:10157000637FA4F80A906969002B7FF45EAE01F1E5
:1015800058024FF0010E0878CDE90826626810284D
:10159000CDF82A20ADF828808DF82EE02A6902D9EE
:1015A000002B7FF44DAE90684FF0000B4AE6032B02
:1015B000BDD0052BBBD0012BB6D1112F7FF4D2AEFD
:1015C000002384F821306B691FFA87F828330893C9
:1015D000731C099308F1FF33ADF82830337808A95C
:1015E0000DF135008DF8343000F0D4F800280DF1FD
:1015F00034093FF7BEAEEB6807480AE6032B01D07B
:10160000052BD8D1701CFFF7FDFB60609BE700BF86
:1016100042DF01085FDD0108EADE01080022FFF772
:10162000CDBD0B0A017043700B0C090E8370C170A5
:10163000704770B51025CEB00C462A4606460021EC
:10164000684606F0C4FC49238DF80030A37BD4F82B
:101650000A100DF106008DF80530FFF7E2FF216951
:101660000DF10A00FFF7DDFF238908A88DF80F3080
:1016700000F000FA216808A800F00CFA2A46694632
:1016800008A800F00DFA2289616808A800F008FA9D
:1016900008A90DEB050000F06EFA049B33604EB014
:1016A00070BD492370B500250C460646CEB08DF8B6
:1016B00000300B8BCDE901558DF801301B0A8DF8F8
:1016C00002308B7E03958DF80330CB7E0DF1060042
:1016D0008DF804300B691968FFF7A3FF61690DF1FC
:1016E0000A00FFF79EFFA38908A88DF80F308DF838
:1016F0000E5000F0BFF9216808A800F0CBF9694648
:1017000008A8102200F0CCF9A289A16808A800F06E
:10171000C7F908A904A800F02EFABDF8103008A8EF
:1017200033808DF804508DF803508DF802508DF8F9
:10173000015000F09FF9616808A800F0ABF9694614
:1017400008A8102200F0ACF9A289A16808A800F04E
:10175000A7F908A904A800F00EFABDF810307380AC
:101760004EB070BD30B50C46CBB0054604A800F0B5
:1017700081F9216804A800F08DF92289616804A824
:1017800000F08EF904A9684600F0F5F9009B2B6083
:101790004BB030BD70B50C89BEB006460D46A4B145
:1017A00014F00F0411D101AA10212868FFF740F9A5
:1017B0002889A04201DC3EB070BD68683119204420
:1017C00001AAFFF7AFF91034F2E74FF0FF30F2E76C
:1017D0002DE9F0430F89C7B081460D46002F4ED04A
:1017E000012410224FEA1718002117F00F0701A853
:1017F00018BF08F1010806F0EAFBAB7BD5F80A1028
:101800000DF10A008DF809308DF80440FFF709FF4B
:1018100029690DF10E00FFF704FF6E68013E444593
:1018200003DD288947B0BDE8F08309AA10212868A4
:101830008DF81340FFF7FCF809AA05A901A8FFF7E6
:1018400071F9444510DB002F14BF3B46102330468E
:101850004A464B440DF1130C934207D80134A4B20D
:1018600009F110091036DAE71023F0E710F801EF5C
:101870001CF8011F81EA0E0102F8011BECE74FF092
:10188000FF30CFE770B5C2B0144606460D46F122D0
:10189000002105A806F09BFB0023CDE90333636814
:1018A00010218DF805301A0A1B0C8DF80730A3683B
:1018B0008DF806208DF808301A0A1B0C8DF80A30B6
:1018C000A3898DF809208DF80B301B0A8DF80C3098
:1018D000012305AA20688DF80430FFF7A9F805AAAE
:1018E000314601A8FFF71EF9022305AA102120683E
:1018F0008DF80430FFF79CF805AA294601A8FFF7E8
:1019000011F942B070BD2DE9F0431025C3B04A9CD7
:1019100080460F4616460021F12205A8994606F09A
:1019200056FB2A46002101A806F051FBA268294671
:101930008DF80520130AEA408DF80720E2688DF83B
:101940000630D37920688DF8083093798DF8093006
:1019500053798DF80A3013798DF80B30D3788DF8E0
:101960000C3093788DF80D3053788DF80E30137855
:1019700005AA8DF80F30238A8DF810301B0A8DF8D8
:10198000113001238DF80430FFF752F805AA4146C3
:1019900001A8FFF7C7F8022305AA294660688DF859
:1019A0000430FFF745F805AA494601A8FFF7BAF841
:1019B000032305AA294620688DF80430FFF738F87C
:1019C00005AA394601A8FFF7ADF8042305AA294660
:1019D00020688DF80430FFF72BF805AA314601A8DE
:1019E000FFF7A0F843B0BDE8F0830000F0B50F2981
:1019F000C7B004460D4616461F4604D94FF4A171E0
:101A00001B48F0F7D9FC0123002F019318BF0223D4
:101A10008DF808309DF830310DF10A0083F0010394
:101A20008DF809304D9B1968FFF7FBFD4E990DF1BC
:101A30000E00FFF7F6FD4FF4807309AA102130461F
:101A400005AEADF81230FEF7F3FF09AA314601A842
:101A5000FFF768F80023601EDAB2954201D847B05C
:101A6000F0BD10F8012FF15C01334A400270F3E73A
:101A70007CDF010810B5102204460021F13006F089
:101A8000A6FA00212046C4F81411F022BDE8104047
:101A900006F09DBA0B46024610211846FEF7C8BF55
:101AA0002DE9FF470446D0F814010E46154604F20E
:101AB000011920B3C0F110089045474628BF1746CA
:101AC00048443A4606F05FFAD4F814313B440F2BF1
:101AD000C4F814311ED9A8451CD204F1F1031946EB
:101AE00013F8012BD87B4B4582EA000203F8012C46
:101AF000F6D122460846FFF715F83E44ED1B0DF1DE
:101B0000100A102D09D82A463146484606F03BFAFD
:101B1000C4F8145104B0BDE8F08704F1F002731E5C
:101B200006F10F0013F8017F12F8011F834281EACA
:101B300007011170F6D16A4604F1F1039846174681
:101B40009446186859680833ACE803004B45624670
:101B5000F6D1224639463846FEF7E4FF43463A4678
:101B600003CA524518605960174603F10803F6D1BD
:101B70001036103DC5E7F0B50C4689B010220021A3
:101B80000546684606F023FA224669466846FEF78F
:101B9000C9FF9DF900306A46002B0DF10F0140DAB4
:101BA000137812F8010F5B005BB243EAD013914245
:101BB00002F8013CF4D19DF80F305B0083F08703FD
:101BC0008DF80F30D4F81431102B39D1002304F2E2
:101BD000011211781DF8030001334140102B02F867
:101BE000011BF6D104F1F102134604F2011712F8B9
:101BF000011BD07B974281EA000102F8011CF6D15B
